:0200000480007A
:100000009715000093850586732510FC6B10B500CD
:10001000EF001005130510006B00050017850100A7
:10002000130545B1178601001306C6B43306A64072
:1000300093050000EF30501D174500001305858D16
:10004000EF30D007EF309012EF0080006F301009D2
:10005000130101FE2328210123263101232441011C
:10006000232E1100232C8100232A910013098000E4
:10007000130A000093091000130409009304000000
:100080006306390D1305F4FFEF00800E1304E4FF3F
:10009000B384A400E3C889FE93771900B384970062
:1000A0001309E9FF330A9A00E31809FCB7870180B6
:1000B00003A907B083A947B0130509009385090078
:1000C000EF00404393040500375501801384050079
:1000D00013061A009305900013050542EF00901DCA
:1000E000B787018003A587B083A5C7B01386040036
:1000F00093060400EF10005EEF308048EF3080364A
:10010000130705003755018013060900938609007F
:100110009387050013054543EF00D019375501803B
:1001200013058544EF00101D8320C10103248101C4
:1001300083244101032901018329C100032A81008D
:1001400013050000130101026780000093041000F2
:100150001389E9FF6FF01FF593070000638807001C
:1001600037450080130505916F30407567800000AA
:100170009307100063DEA736130101F59307E5FF2F
:100180001307D5FF232AF10293F7E7FFB307F740E0
:10019000232E31092326110A2324810A2322910ABE
:1001A0002320210B232C4109232A510923286109EB
:1001B0002326710923248109232291092320A109DF
:1001C000232EB107232AE1009305F5FF2326F10230
:1001D0002322010093091000138B05006386352745
:1001E0009387F5FF232CF1009382D5FF2324010090
:1001F000832781016386372F1308EBFF93F7E2FF14
:10020000130BCBFFB307FB40232201032328F1028A
:1002100023260100130A0800630A381D9307F8FF1C
:10022000232EF1009303D8FF232801008327C10167
:100230006380372B1309EAFF93F6E3FF130ACAFF23
:1002400023242103B306DA40930D000013040900B0
:10025000630A39151306F9FF930AD9FF93070000C3
:10026000630C36251305A4FF13F7EAFF130DE4FF13
:100270003307E5401303C4FF930E0D001304B4FFCE
:100280002320E102138E0A009308000013850E005C
:10029000638A3E0D130C0400930B0E00930C0000B8
:1002A00063823B231307E5FF9374ECFF1305C5FF3F
:1002B000930F0700B3049540130F000013850F0040
:1002C0002326E1062324C1072322D1072320610628
:1002D000232EC104232CD104232A710423280105D1
:1002E000232651042324B1042322E10523201105F0
:1002F000232EF102232CF103EFF09FE7832F8103DC
:10030000032F41048327C103938FEFFF8328010448
:10031000832581048322C104032801058323410529
:10032000832681050326C10503230106832E41068A
:10033000032E81060327C106330FAF00E390F4F9C3
:1003400013751C00330FE50113050700B38CEC0196
:10035000938BEBFF130CECFFE3C4E9F4137513006C
:1003600033059501032701021303E3FFB388A800B7
:10037000130EEEFF938EEEFF1304E4FFE31867F015
:1003800013F71A00B308170113040D00B387170100
:100390001306E6FF938AEAFFE3C4A9ED13741A007B
:1003A0003304F4001309E9FFB38D8D00130AEAFF4B
:1003B000E39E26E993F71300B38DB701832701016C
:1003C000032A81029383E3FFB387B7012328F10057
:1003D0008327C1019387E7FF232EF100E3C849E596
:1003E00083270101137A1B00330AFA008327C10017
:1003F0001308E8FF130BEBFFB38747012326F10037
:1004000083270103E39807E10327C10093F7120054
:10041000B387E70003278100032B41029382E2FFA9
:10042000B307F7002324F100832781019387E7FFB7
:10043000232CF100E3CE69DB8327410113FB170076
:1004400083278100330BFB00832741009385E5FF61
:10045000B38767012322F100832741019387E7FFD8
:10046000232AF1008327C102E398B7D683274103EB
:100470008320C10A0324810A93F5170083274100D2
:100480008324410A0329010A8329C109032A810916
:10049000832A4109032B0109832BC108032C8108FE
:1004A000832C4108032D0108832DC1073385F500F6
:1004B0001301010B6780000093081000130DE4FF87
:1004C0006FF09FEC130F10001307E5FF6FF0DFE7ED
:1004D0009307EAFF930D10002324F1026FF01FEE43
:1004E0001307EBFF930710002322E1026FF09FF246
:1004F00067800000130101FE232C8100232A910054
:100500002328210123263101232E11009304050005
:1005100013840500EF00C009B787018003A707B364
:100520009307F0FF9309050013890500630AF7029A
:100530001386040013850400930604009305040049
:10054000EF205068631E0500138504009305040026
:100550001306000093060000EF1090236344050289
:100560008320C101032481018324410113850900F3
:10057000930509008329C100032901011301010228
:1005800067800000EF30C0349307100213060000AC
:10059000930600002320F50093850600130506004E
:1005A000EF10401393090500138905006FF05FFBFE
:1005B000130101FF3707F07F2324810023229100DC
:1005C000232611003376B700938405001304050039
:1005D0006308E62093060500635CB01413D645411A
:1005E0009387050063000618370710009305F7FF8F
:1005F000B3F7B700B3E7E700930416C013971700EB
:1006000013F6140093D7F601B307F70013971600FB
:10061000630A06001357F70193971700B387E700A3
:100620001397260093D4144093056001130E000025
:1006300093060000370620003385C6001358F701E3
:100640009385F5FF63C8A700B387A740B306C5002D
:10065000330ECE0093971700B307F8001317170057
:1006600013561600E39A05FC13030000130500025D
:10067000370600806F004002638ED7121358F701CF
:10068000939717001305F5FFB3870701131717009A
:1006900013561600630605043308B600E3DEF6FCC5
:1006A000B305C80093880600634E080EB387D74091
:1006B000B3360701B387D740330707411358F70113
:1006C000939717001305F5FF3303C30093860800C3
:1006D000B38707011317170013561600E31E05FA18
:1006E000B3E7E7006394070E1355130093571E40BA
:1006F0003707E03F137E1E00B387E70063060E0056
:10070000370700803365E500939444011304050026
:10071000B384F4008320C100130504000324810086
:1007200093850400832441001301010167800000C8
:100730009397150093D71700B3E7A700E38C07FC46
:1007400013060000639C050C13D7B6001306B6FE13
:100750009307070093965601E30807FE9355470158
:100760006394050E93050000370810009397170057
:1007700033F707011385050093851500E30807FE8D
:100780009308000213880600B388B8401387070057
:10079000B396B600B35718013306A640B3E7E70097
:1007A0006FF09FE493C8F5FF93D8F801B388160162
:1007B0006FF0DFEFE36407EDB305C800E34408FE24
:1007C00093880700930700006FF01FEF9307F0FF77
:1007D0006308F30613051300135515006FF01FF19E
:1007E0001306050093860500EF1050091306040058
:1007F00093860400EF00C035130405008320C10078
:1008000013050400032481009384050093850400EC
:1008100083244100130101016780000013060500D5
:1008200093860500EF20000013060500938605005F
:10083000EF00506A13040500938405006FF09FEDEC
:10084000130E1E006FF09FEA138806009308000243
:100850001305F0FF6FF01FF4130500006B00050097
:10086000732500FC6B000500977101009381010F57
:1008700017F1FF7E1301017993050040732610CC18
:10088000B385C5023301B140F32630CC6386060040
:10089000130500006B000500678000006308052059
:1008A000130101F52324810A232E31092326110A7D
:1008B0002322910A2320210B232C4109232A5109A9
:1008C00023286109232671099309050003450500C2
:1008D000138419006308051CB7340000B75A01805F
:1008E000138A05001309500293849480938A4A4521
:1008F00063042505EF00C02303450400130B140017
:1009000013040B00E31605FE330534418320C10AAE
:100910000324810A8324410A0329010A8329C10986
:10092000032A8109832A4109032B0109832BC1086A
:100930001301010B67800000130504009306D0002B
:100940001306100003470500130B1500930707FE5D
:1009500093F7F70F63E8F600B317F600B3F79700C5
:10096000639207109307A002630AF7001306A00022
:1009700093050104EF30C03A032B010483470B00B9
:100980001307E00213051B006382E70E938747FB02
:1009900093F7F70F1307E0026364F70293972700BA
:1009A000B387570183A707006780070003471B0031
:1009B00093078006630AF708130B0500130515005B
:1009C0002300210533058540635AA00893070400DE
:1009D000130711043306A40083C60700938717008A
:1009E00013071700A30FD7FEE398C7FE13051500E2
:1009F00093070108B387A70093060A0013060104B2
:100A00009305001013050100238007FCEF304036EA
:100A100013040100B30BA100635AA00003450400B6
:100A200013041400EF00C010E39A8BFE03451B0073
:100A300013042B00E31E05EA6FF01FED03471B00B4
:100A40009307C006E31AF7F613053B0023002105C0
:100A500033058540130B2B00E34AA0F61305100065
:100A60006FF01FF913050B006FF0DFED03471B005C
:100A70009307A002631AF70083472B0013053B007E
:100A8000130B2B006FF09FF01306A00093050104D9
:100A9000EF300029032B010483470B0013051B00D3
:100AA0006FF0DFEE130510006FF05FE61305F0FF47
:100AB00067800000130101FC130341022322B102ED
:100AC00093050300232E11002324C1022326D10203
:100AD0002328E102232AF102232C0103232E1103F0
:100AE00023266100EFF09FDB8320C1011301010485
:100AF00067800000130101FF2324810023261100D9
:100B00001304050003450500630C050013041400DD
:100B100013041400EF00C0010345F4FFE31A05FEBF
:100B20008320C100032481001301010167800000BC
:100B3000976201009382826283A20200732320CC19
:100B4000131303013363A30023A062006780000036
:100B5000130101FE232E1100232C8100232A910072
:100B6000232821012326310123244101F3292000D8
:100B7000B70810009388F8FF33F7B80013D4450185
:100B800093D4F50193D5460193173700B3F8D800F5
:100B90001357D5011374F47F93F5F57F3367F7008E
:100BA00013D3F601931735009356D6019398380066
:100BB0003305B44013183600B3E6160113060500DA
:100BC000639E64426358A0146390050633E50601F2
:100BD000631805009306F07F631ED6366F00C002CF
:100BE0001305F6FF631E05003308F800B306D700AF
:100BF000B337F800B386F600130610006F00000A42
:100C00009308F07F63181605B366F700E3820610B9
:100C1000B7064000B376D700130400006396062899
:100C2000930500016F0040281306F07F6310C40293
:100C3000B366F700E384060EB7064000B376D7002C
:100C4000638806161306F07F6F00C03037068000F9
:100C5000B3E6C600130680036348A60A1306F00134
:100C6000634AA606130600023306A640B358A8003E
:100C7000B395C6003318C800B3E515013338000139
:100C800033E8050133D5A6003308F8003305E50045
:100C9000B337F800B306F50013060400B707800069
:100CA000B3F7F60063860708130616009307F07F74
:100CB000630EF630370780FF1307F7FF93571800CE
:100CC00033F7E6001378180033E807019317F701AC
:100CD0006F00C027930505FE93080002B3D5B60048
:100CE0001306000063081501130600043305A6402F
:100CF0003396A600336806013338000133E8050156
:100D0000130500006FF05FF833E806013338000187
:100D10006FF01FFF630005143386854063160406D9
:100D20003365F700631E05009307F07F630EF6023C
:100D30001387060093070800630406526F008021A2
:100D40009308F6FF639E0800B387070133B80701D5
:100D5000B306D700B3860601138807006FF0DFE9FA
:100D60001305F07F6310A606B3E70601638E077ACA
:100D7000B7074000B3F7F60013870600639A077AB7
:100D8000930708006FF0DFE91305F07F6396A50273
:100D9000B3E7060163880774B7074000B3F7F600AE
:100DA0001387060063980774930708001306F07F03
:100DB000130400006FF0DFE6370580003367A700FB
:100DC0009308060013068003634016091306F0011A
:100DD0006342160513050002330515413316A700BB
:100DE00033D31701B397A70033666600B337F0001B
:100DF000B367F60033571701B38707013307D700EE
:100E0000B3B60701B306D7001388070013860500A1
:100E10006FF0DFE8138608FE130300023356C700A5
:100E200013050000638868001305000433051541AD
:100E30003315A700B367F500B337F000B367F600CA
:100E4000130700006FF05FFBB367F700B337F000E4
:100E50006FF01FFF130614001375E67F6318050C6F
:100E60003365F700631004066300056233E606018C
:100E70006308063E33880701B337F8003307D7000D
:100E80003307F700B7078000B377F7006380076088
:100E9000B70780FF9387F7FF3377F70093050000CC
:100EA000930708001306100093F677006394060E6C
:100EB000630A047493F615006386067493E52500AF
:100EC0006F0040741306F07F6318C404630E057E40
:100ED000370640003376C700133616001316460057
:100EE000639485709305060033E60601630A0600E5
:100EF0003706400033F6C600631406009305000170
:100F00006316056E1387060093070800130400009C
:100F10001306F07F6FF05FF96396C500930500003C
:100F20006FF09FFC930500006FF09FFD9305F07F2D
:100F30006306B60233880701B337F8003307D700DA
:100F40003307F7009317F70113581800B3E70701A9
:100F500013571700130400006F00C05D6388090079
:100F6000930730006398F900639C04001306F07F38
:100F70006F00C006930720006394F900E39804FE15
:100F8000130400001307F0FF9307F0FF1306E07F40
:100F9000930550009306200093E515006384D96003
:100FA00093063000638AD95E6390096093F6F70078
:100FB00013054000638AA65E93864700B3B7F60028
:100FC0003307F700938706006F00005E638809000F
:100FD00093073000639CF9006392045213070000EA
:100FE00093070000930550006F00C0619307200035
:100FF0006396F950E39404FE6FF09FF8635AA00ED5
:10100000639E050833E50601E30605BC1305F6FFFC
:10101000631E050033880741B306D740B3B7070105
:10102000B386F640130610006F0040059308F07F6A
:10103000E30C16BD130680036346A60A1306F001EF
:101040006348A606130600023306A640B395C60001
:10105000B358A8003318C800B3E5150133380001B0
:1010600033E80501B3D6A60033880741B306D7405D
:10107000B3B70701B386F6401306040037098000B2
:10108000B3F72601E38607CA1309F9FF33F92601EE
:10109000130A0800130406006F0040311306F07FA6
:1010A000E308C4B837068000B3E6C6006FF09FF8C7
:1010B000930505FE93080002B3D5B60013060000A1
:1010C00063081501130600043306A6403396C600D4
:1010D000336806013338000133E805019306000048
:1010E0006FF09FF833E80601333800016FF01FFFFF
:1010F0006300051433868540631404063365F700E6
:10110000631805009307F07F930403006FF01FC27C
:101110009308F6FF63900802B307F8403338F800ED
:10112000B386E640B38606419304030013880700A4
:101130006FF05FEF1305F07F6312A606B3E70601B9
:10114000638E073EB7074000B3F7F600138706002B
:10115000639C073E93070800930403006FF05FACA5
:101160001305F07F6396A502B3E706016384073E8B
:10117000B7074000B3F7F600138706006392073EF7
:10118000930708001306F07F930403006FF05FC21B
:10119000370580003367A700930806001306800315
:1011A000634216091306F001634416051305000295
:1011B000330515413316A70033DE1701B397A70097
:1011C0003366C601B337F000B367F6003357170133
:1011D000B307F8403387E640B336F800B306D7408C
:1011E0001388070013860500930403006FF01FE9BE
:1011F000138608FE130E00023356C70013050000C5
:101200006388C80113050004330515413315A70091
:10121000B367F500B337F000B367F60013070000BB
:101220006FF01FFBB367F700B337F0006FF01FFFDD
:10123000130614001376E67F63120614B368F700F2
:1012400033E50601631A040C63900808631405244F
:101250009384E9FF93B41400130700009307000080
:10126000B3E6E7006382063293D6F7011314170042
:101270003304D4009396170013F67600930500000C
:10128000630A0602130620006380C9241306300097
:10129000638EC92093051000639E090013F6F600C3
:1012A000130540006308A60093B6C6FF93C6160058
:1012B0003304D40013548401134414001374140031
:1012C000130600006FF05FBEE30C05F8B38507411D
:1012D00033B5B7003306D7403306A6403705800044
:1012E0003375A600630E0500B307F8403387E64068
:1012F0003338F80033070741930403006FF05FF6BB
:10130000B3E7C500639E07189384E9FF93B4140004
:10131000130700006FF0DFF41306F07F6312C402BE
:1013200063880838370640003376C7001336160046
:101330001316460063948538930506006F00C000BD
:10134000639AC50293050000630A05003706400052
:1013500033F6C60063140600930500016392083655
:101360006308052013870600930708009304030011
:101370006FF0DFB9930500006FF05FFE338A07411D
:1013800033B647013309D7403309C94037068000D7
:101390003376C90063020608330AF840B386E64094
:1013A000333848013389064193040300630C09066E
:1013B00013050900EF20C04B130685FF9307F001CA
:1013C00063CAC70693060002B386C6403317C90036
:1013D000B356DA00B3E6E6003318CA00634C860859
:1013E00033068640130716009307F00163CCE70429
:1013F000130600023306E640B397C6003355E800F3
:101400003316C800B3E7A7003336C000B3E7C70000
:1014100033D7E6006FF0DFE4B3672A01E39807F8FB
:101420006FF09FEE13050A00EF20804413050502BC
:101430006FF09FF8930685FDB316DA0013080000DD
:101440006FF0DFF9130616FE9305000233D6C600CF
:10145000930700006308B70093070004B387E740D1
:10146000B397F600B367F800B337F000B367F60040
:101470006FF01FEAB70780FF9387F7FF3306C4407A
:10148000B3F6F6006FF0DF8A1387060093070800B3
:101490006FF01FDD13870600930708006FF0DFE58C
:1014A00013070600938705006FF09FDB9385040008
:1014B000E39204E093B686FF93C616003304D4008B
:1014C000930510006FF01FDF93051000E38404DE26
:1014D00093B686FF93C616003304D40093850400A8
:1014E0006FF05FDD130700001306F07F9305000027
:1014F0006F004011930708006FF0CFF41307F0FF5F
:101500009307F0FF1306E07F130400006FF05FA85D
:1015100013070000930700006F00C00E13070000C0
:10152000930700006FF05FFC130700006FF01FFCD3
:1015300093070800930500006FF01F971307000042
:10154000930403006FF09FFA9307080093040300CD
:101550006FF05FFE130700001306F07F6FF05FFE71
:10156000930708001306F07F930403006FF09F9E1B
:101570009307000093040000370740001306F07F34
:10158000930500016F000008130700009307000097
:10159000130600006FF09FF56398040093868700A0
:1015A0006FF0DFA1E39C04FEE31A04906F00800556
:1015B000930700006384090213073000639AE9006F
:1015C000638E04009307F0FF1306E07F6F000001B5
:1015D00013072000E398E9FEE38604FE93E5550037
:1015E000138707006F00400493050600B3E6060169
:1015F000E38E069093040000370740009307000035
:101600001306F07FB7068000B376D700638E06001E
:10161000130616009306F07FE30CD6F8B70680FF9A
:101620009386F6FF3377D70013D537009306F07F04
:101630009317D701B3E7A70013573700631ED600EF
:10164000B3E7E700130700006388070037070800C7
:101650009307000093040000B706F07F13164601BD
:101660001317C7003376D6001357C7003367E60059
:101670009394F401B36697001387070093870600DD
:101680006384050073A015008320C1010324810138
:1016900083244101032901018329C100032A810018
:1016A00013050700938507001301010267800000FE
:1016B000E38A85C8930500006FF09FCA9305060072
:1016C000E30605846FF01FF3E38A85849305000029
:1016D0006FF05F83130101FD23248102232A51014E
:1016E0002322910123261102232291022320210388
:1016F000232E3101232C410123286101232671016E
:101700002324810113040500930C0600938A06002C
:101710007329200013DB4501939BC500137BFB7FDE
:1017200093DBCB0013DAF501630A0B029307F07F1A
:101730006308FB081357D501939B3B00B36B7701FC
:10174000B7078000B3EBFB0093193500130B1BC0E8
:10175000130C0000930400006F00C008B3E7AB0057
:10176000638E070E63800B0413850B00EF2040107F
:10177000130755FF9307C00163CCE7029306D0011E
:10178000930985FFB386E640B39B3B01B356D40073
:10179000B3EB7601B31934019305D0C0338BA54068
:1017A0006FF01FFBEF20C00C130505026FF05FFC0C
:1017B000930B85FDB31B7401930900006FF0DFFDEF
:1017C00033E4AB006306040AB7070800B3F7FB0075
:1017D00093090500130BF07F130C300093040001F4
:1017E000E39A07F61395CA001354C50013D54A01AE
:1017F0009375F57F93870C0093DAFA0163840508EB
:101800001307F07F6386E50E93D7DC0113153400D0
:1018100033E5A700370480003364850093973C00CC
:10182000138515C01307000093162C00B3E6E600DD
:10183000B305AB409386F6FF1305E00033465A012B
:101840006362D51037550180939626001305055124
:10185000B386A60083A6060067800600930B0000EF
:1018600093090000130B0000130C10006FF09FEEA3
:10187000930B000093090000130BF07F130C200062
:101880006FF05FEDB3679401638607086302040499
:1018900013050400EF10D07D93050500938655FFD6
:1018A0009307C00163CED7021307D001938785FF4A
:1018B0003307D7403315F40033D7EC003364A70067
:1018C000B397FC001307D0C03305B7406FF09FF506
:1018D00013850C00EF10D079930505026FF01FFC03
:1018E000138585FD3394AC00930700006FF09FFDD6
:1018F00033669401630A0602370708003377E40071
:101900001305F07F631C07021307300093040001E6
:101910006FF09FF11304000093070000130500000F
:10192000130710006FF05FF013040000930700002E
:101930001305F07F130720006FF01FEF130730002F
:101940006FF09FEE6366740163968B2E63E4F92E4D
:101950001395FB0113D719009396F90193DB1B0034
:10196000B369E5001315840013D887013368A80014
:101970001355050133DEAB02131F0801135F0F017E
:101980009398870093D70901B3FBAB0213030E00B2
:101990003307CF03939B0B01B3E7770163FEE700A7
:1019A000B38707011303FEFF63E8070163F6E7004F
:1019B0001303EEFFB3870701B387E740B3DEA70247
:1019C0001397090113570701B3F7A70293890E0074
:1019D000330EDF03939707013367F700637EC70178
:1019E000330707019389FEFF636807016376C70128
:1019F0009389EEFF3307070113130301B369330122
:101A000037030100930EF3FF93D2090193DF08011E
:101A10003307C74133FED901B3FED801B307DE0354
:101A20003384D203338ECF03B3038E0013DE07015A
:101A3000330E7E00B382F20363748E00B3826200C1
:101A4000B703010013530E019383F3FFB302530056
:101A500033737E0013130301B3F777003303F300EE
:101A600063685700138409006314570463F2660423
:101A7000B3861601B3B71601B38707013307F70022
:101A80001384F9FF6366E8006314E80263E2160357
:101A900063665700639EE20063FC6600B38616012E
:101AA000B3B71601B38707011384E9FF3307F700C3
:101AB0003383664033075740B3B666003307D740D9
:101AC0009307F0FF6304E812B352A7029357030190
:101AD0003377A70293860200330E5F0213170701C4
:101AE00033E7E700637EC701330707019386F2FF00
:101AF000636807016376C7019386E2FF3307070136
:101B00003307C741335EA7029317030193D7070139
:101B10003377A702330FCF031317070133E7E7002B
:101B200093070E00637EE701330707019307FEFF6B
:101B3000636807016376E7019307EEFF3307070148
:101B400093960601B3E6F6009397060193D7070133
:101B500013D30601338E6F023307E741B38FFF02C1
:101B6000338FFE02B30ED30393570F01B38FDF0100
:101B7000B387F70163F6D70137050100330EAE00D6
:101B800013D307013303C301370E0100130EFEFF09
:101B900033F5C70113150501337FCF013305E50187
:101BA000636867006312673E93870600630005045D
:101BB0003307E8009387F6FF6364070363666700F3
:101BC0006312673C63F0A8029387E6FF93961800C0
:101BD000B3B816013388080133070701938806005C
:101BE000631467006384A80093E717001388F53F28
:101BF000635C001913F77700630A070A13072000D4
:101C000093E414006302E90A130730006308E9084B
:101C1000631E090813F7F700930640006308D7080E
:101C200013874700B337F7003304F4009307070026
:101C30006F00C0079385F5FF930600006FF09FD2F9
:101C400013060A0013840B009387090013070C0086
:101C500093063000630ED730930610006304D7302C
:101C600093062000E314D7F86F00000113860A00E2
:101C70006FF01FFE93E4840013050000930700003B
:101C80001307F07F6F000006370408009307000079
:101C900013060000130730006FF09FFB6318060067
:101CA000138787006FF01FF8E31C06FE370700015B
:101CB0003377E400630A0700370700FF1307F7FFD5
:101CC0003374E400138805401307E07F634E070771
:101CD00013D737009317D401B3E7E7001355340047
:101CE0001307080013174701B706F07F1315C50047
:101CF0003377D7001355C5003365A7001316F601D7
:101D00003367C5009305070013850700638404004B
:101D100073A014008320C1020324810283244102A2
:101D2000032901028329C101032A8101832A410178
:101D3000032B0101832BC100032C8100832C410064
:101D4000130101036780000093072000630AF90272
:101D500093073000630AF900631A09009307000033
:101D60001307F07F6F000001E30A06FE9307F0FF00
:101D70001307E07F93E45400138507006FF09FF68C
:101D8000E31E06FC6FF09FFE1307100063100806A9
:101D900093F677001307040063840604930620007B
:101DA00093E41400630CD902930630006302D90255
:101DB0006318090293F6F700130540006382A60238
:101DC00013B7C7FF13471700330787006F004001A1
:101DD0006318060013B787FF6FF0DFFEE31C06FEF3
:101DE00013578701134717001377170013051000C7
:101DF000330505419306800363CEA60E9306F001DA
:101E000063C2A6069385E54133D8A700B316B40094
:101E1000B397B700B3E60601B337F000B3E7F600B7
:101E20003355A40093F677006380060893062000DC
:101E300093E414006308D90693063000630ED904B6
:101E40006314090693F6F70093054000638EB60409
:101E500093864700B3B7F6003305F5009387060075
:101E60006F008004930610FEB386064193080002BB
:101E7000B356D40013080000630615019385E543AB
:101E80003318B400B367F800B337F000B3E7F600D7
:101E9000130500006FF01FF9631806009386870092
:101EA0006FF05FFBE31C06FEB7068000B376D5003B
:101EB000638E060093E414001305000093070000EE
:101EC00063160702130710006FF0DFE193D63700A7
:101ED0009317D501B3E7D70013553500E30407E0A6
:101EE00013F71400E30007E01307000093E4240055
:101EF0006FF05FDFB3E7870063840702930720007A
:101F000093E41400630EF902930730006302F902B0
:101F100093071000631409009307500093D737000C
:101F200093E4240013050000130700006FF09FDB0B
:101F300093079000E30406FE930710006FF01FFE66
:101F400093079000E31C06FC6FF01FFF37050800A5
:101F5000930700001307F07F1306000093040001AD
:101F60006FF05FD813050000930700006FF0DFFBF0
:101F700037050800930700001307F07F13060000E1
:101F80006FF05FD693860700938706006FF0DFC57A
:101F90009307050073272000370710001307F7FF8A
:101FA00013D84501B378B700130305001378F87F01
:101FB00013D5F501930EF07F93D546013377D70003
:101FC000130E060093F5F57F93D6F601631CD80136
:101FD000B3EEF800638C0E08736018001305200040
:101FE000678000006396D501B36EC700E3960EFECE
:101FF00063100808B3E7F80093B71700639605006D
:102000003366C700630C0604639C07006314D500A5
:1020100063D00503630005041305F0FF678000002B
:102020001305F0FF638A0600138506006780000031
:102030006356B800E30205FE67800000E36C17FDFD
:102040006392E802E3686EFCE366C3FF13050000D9
:10205000678000001305100067800000E39807FE0A
:102060006FF05FFBE3E8E8FC6FF05FFEE38E05F7DF
:10207000E39E05F8930700006FF09FF8130101FD40
:1020800023248102232A51012322910123261102B4
:102090002322910223202103232E3101232C4101ED
:1020A00023286101232671012324810113040500E3
:1020B000930C0600938A06007329200093DB4501E8
:1020C0009399C50093FBFB7F93D9C90013DBF501FE
:1020D000638A0B029307F07F6388FB089357D5014F
:1020E00093993900B3E93701B7078000B3E9F900E4
:1020F000131A3500938B1BC0130C000093040000CF
:102100006F00C008B3E7A90063800710638009046B
:1021100013850900EF10C075130755FF9307C00121
:1021200063CCE7029307D001130A85FFB387E7402A
:10213000B3994901B357F400B3E93701331A4401A5
:10214000930BD0C0B38BAB406FF01FFBEF1040720E
:10215000130505026FF05FFC930985FDB319340187
:10216000130A00006FF0DFFD33E4A9006308040ADE
:10217000B7070800B3F7F900130A0500930BF07FC7
:10218000130C300093040001E39A07F613D54A01BB
:102190001394CA001375F57F93870C001354C40081
:1021A00093DAFA01630605081307F07F6306E50E6C
:1021B00093D7DC011314340033E48700B7078000A1
:1021C0003364F400130515C093973C001307000017
:1021D00093162C00B3E6E600B38BAB009386F6FFB4
:1021E0001306E000B3455B0113851B00636CD61634
:1021F00037560180939626001306C654B386C60050
:1022000083A606006780060093090000130A0000F9
:10221000930B0000130C10006FF05FEE93090000A9
:10222000130A0000930BF07F130C20006FF01FEDDA
:10223000B367940163840708630004041305040072
:10224000EF100063930655FF9307C00163CED702DA
:102250001307D001930785FF3307D7403314F400E9
:1022600033D7EC0033648700B397FC001307D0C06A
:102270003305A7406FF09FF513850C00EF10405F0A
:10228000130505026FF01FFC130485FD33948C00C9
:10229000930700006FF09FFD33669401630A060206
:1022A000370708003377E4001305F07F631C07024B
:1022B00013073000930400016FF09FF11304000036
:1022C0009307000013050000130710006FF05FF084
:1022D00013040000930700001305F07F130720008C
:1022E0006FF01FEF130730006FF09FEE3704080008
:1022F000930700001307F07F93050000930400018B
:1023000013174701B706F07F1314C4003377D700C3
:102310001354C4009395F501336487003367B40008
:1023200013850700930507006384040073A014005D
:102330008320C10203248102832441020329010274
:102340008329C101032A8101832A4101032B010151
:10235000832BC100032C8100832C41001301010356
:1023600067800000B70E0100138EFEFF13570A01AD
:1023700093D80701337ACA01B3F7C70133884803FA
:10238000B3864703330FF7023303E80113D806017E
:1023900033086800330617036374E8013306D60177
:1023A000935F08013378C801B3F6C601935E040158
:1023B000337EC401131808013308D800330FC70354
:1023C000B306CA03338A4E033303EA0113DA060164
:1023D000330A6A003307D7036376EA013703010043
:1023E0003307670013530A013303E3003707010083
:1023F000130FF7FF337AEA01B3F6E60113D40901AC
:10240000131A0A01B3F9E901338F3703330ADA00EB
:10241000B38F4F01B3863803B307F402B382880247
:10242000B388F60093560F01B386160163F4F600E5
:10243000B382E200370701009307F7FF337FFF0005
:1024400093D80601B3F6F600B387C9039396060145
:10245000B386E601B3885800330EC403B3893E0344
:10246000338F8E02B389C90113D40701B309340134
:1024700063F4C901330FEF00370E0100130EFEFFA6
:1024800033F7C901B3F7C701131707013306F60184
:102490003307F700333A4601330767003304470137
:1024A0003306D600B336D600330E1401B30EDE0069
:1024B000333767003334440133648700B3B6DE003A
:1024C00093D90901B3381E0133043401B3E6D800AF
:1024D0003304D4003304E40193D77E011314940031
:1024E0003364F40093179600B3E70701B337F000A5
:1024F0001356760137070001B3E7C700939E9E008D
:102500003377E400B3E7D7016300070A13D7170056
:1025100093F71700B367F7001317F401B3E7E70069
:10252000135414001308F53F635A001113F7770092
:10253000630807081307200093E414006300E90808
:10254000130730006306E906631C090613F7F7005A
:10255000930640006306D70613874700B337F7009A
:102560003304F400930707006F00800593050B0008
:102570001384090093070A0013070C009306200038
:102580006300D728930630006304D7289306100011
:10259000E31AD7F813040000930700006F0000242B
:1025A00093850A006FF09FFD13850B006FF09FF776
:1025B00063980500138787006FF05FFAE39C05FEC0
:1025C000370700013377E400630A0700370700FF8D
:1025D0001307F7FF3374E400130805401307E07F87
:1025E000634E070113D737009317D401B3E7E70011
:1025F00013543400130708006FF09FD09307200096
:10260000630AF90293073000630AF900631A0900AC
:10261000930700001307F07F6F000001E38A05FEB7
:102620009307F0FF1307E07F93E45400138407003F
:102630006FF01FCDE39E05FC6FF09FFE13071000A7
:102640006310080693F677001307040063840604FA
:102650009306200093E41400630CD9029306300023
:102660006302D9026318090293F6F70013064000CB
:102670006382C60213B7C7FF1347170033078700EB
:102680006F0040016398050013B787FF6FF0DFFE0E
:10269000E39C05FE135787011347170013771700B4
:1026A00093061000B386064113068003634ED60ED0
:1026B0001306F0016342D6061305E5413316A40064
:1026C00033D8D700B397A70033660601B337F000BD
:1026D000B367F6003354D40093F67700638006089E
:1026E0009306200093E414006308D9069306300093
:1026F000630ED9046314090693F6F700130640002D
:10270000638EC60493864700B3B7F6003304F40023
:10271000938706006F008004130610FE33060641FF
:10272000930800023356C4001308000063861601A4
:102730001305E5433318A400B367F800B337F0007E
:10274000B367F600130400006FF01FF963980500EB
:10275000938687006FF05FFBE39C05FEB706800061
:10276000B376D400638E060093E4140013040000D3
:102770009307000063160702130710006FF05FB89D
:1027800093D637009317D401B3E7D700135434001E
:10279000E30807B613F71400E30407B613070000B5
:1027A00093E424006FF0DFB5B3E78700638407028A
:1027B0009307200093E41400630EF902930730009E
:1027C0006302F90293071000631409009307500095
:1027D00093D7370093E4240013040000130700008C
:1027E0006FF01FB293079000E38405FE930710007B
:1027F0006FF01FFE93079000E39C05FC6FF01FFF36
:1028000013040000930700001307F07F6FF05FAF21
:1028100037040800930700001307F07F93050000BA
:102820006FF01FAE130101FE232E1100232C810037
:10283000232A910023282101232631012324410149
:10284000F3292000B70810009388F8FF33F7B80089
:1028500013D44501B3F8D80093D4F50193D54601BC
:102860009317370013D3F6011357D5019356D601AA
:10287000939838001318360093F5F57F1306F07F10
:102880003367F7001374F47F93173500B3E616012E
:102890006396C50033E60601631406001343130074
:1028A0003306B440631E93506358C016639A0506FE
:1028B00033E50601631605029306F07F130400005A
:1028C0006318D62EB366F700E3880620370440006D
:1028D0003374870013341400131444006F00402D28
:1028E0001305F6FF631E05003308F800B306D70092
:1028F000B337F800B386F600130610006F00400AE5
:102900009308F07F631A1605B366F700E39006FCA0
:102910001307000093070000130400006F00C0328B
:102920009305F07F6314B402B366F700E38C061AD4
:10293000B7064000B376D7001306F07F930500007A
:10294000639C063C130400016F008026B7058000DD
:10295000B3E6B60013050600130680036348A60A13
:102960001306F001634AA606130600023306A640CA
:10297000B395C600B358A8003318C800B3E51501D5
:102980003338000133E80501B3D6A6003308F80058
:10299000B386E600B337F800B386F60013060400EA
:1029A000B7078000B3F7F600638607081306160022
:1029B0009307F07F630EF63C370780FF1307F7FF9E
:1029C0009357180033F7E6001378180033E807012F
:1029D0009317F7016F008033930505FE93080002FB
:1029E000B3D5B600130600006308150113060004F2
:1029F0003306A6403396C60033680601333800011B
:102A000033E80501930600006FF05FF833E8060134
:102A1000333800016FF01FFF6302061433868540D0
:102A2000631804063365F700631E05009307F07F03
:102A3000630EF60213870600930708006304065E20
:102A40006F00402D9308F6FF639E0800B3870701CF
:102A500033B80701B306D700B38606011388070011
:102A60006FF09FE91305F07F6312A606B3E7060136
:102A700013070000638A071CB7074000B3F7F6008E
:102A800013870600E3960706930708006F00C0024D
:102A90001305F07F6396A502B3E70601E3880700FC
:102AA000B7074000B3F7F60013870600E396070068
:102AB000930708001306F07F930500006FF09FE86E
:102AC000370580003367A7009308060013068003CC
:102AD000634016091306F001634216051305000250
:102AE000330515413316A70033D31701B397A70059
:102AF00033666600B337F000B367F600335717014B
:102B0000B38707013307D700B3B60701B306D70071
:102B100013880700138605006FF09FE8138608FEF0
:102B2000130300023356C7001305000063886800D2
:102B300013050004330515413315A700B367F500ED
:102B4000B337F000B367F600130700006FF05FFBC8
:102B5000B367F700B337F0006FF01FFF13061400E0
:102B60001375E67F631405183366F70063100406D7
:102B70006300066E33E606016306064A33880701E2
:102B8000B337F8003307D7003307F700B7078000E3
:102B9000B377F7006380076CB70780FF9387F7FF71
:102BA0003377F70093050000930708001306100021
:102BB00093F677006392061A6388050893761400EB
:102BC00063840608136424006F0000081305F07F77
:102BD000631CA4026302067E37044000337487003E
:102BE00013341400131444006394A504B3E50601E0
:102BF00063800502B7054000B3F5B600639A05008F
:102C0000130400016F00C00013040000E380A5FE60
:102C1000631006021387060093070800930500005F
:102C20001306F07F6FF0DFF8130400006FF01FFC55
:102C3000B3E60601E38406FE930400003707400074
:102C4000930700001306F07FB7068000B376D70025
:102C5000638E0600130616009306F07F630CD67091
:102C6000B70680FF9386F6FF3377D70013D537007A
:102C70009306F07F9317D701B3E7A70013573700E8
:102C8000631ED600B3E7E700130700006388070060
:102C9000370708009307000093040000B706F07F91
:102CA000131646011317C7003376D6001357C70013
:102CB0003367E6009394F401B36697001385070029
:102CC0009385060063040400732014008320C1016F
:102CD0000324810183244101032901018329C100C7
:102CE000032A810013010102678000009305F07F31
:102CF0006308B60233880701B337F8003307D700FB
:102D00003307F7009317F70113581800B3E70701CB
:102D10001357170093050000130400006FF05FE9DC
:102D200063880900930730006398F900639C0400EE
:102D30001306F07F6F00C006930720006394F9002C
:102D4000E39804FE930500001307F0FF9307F0FFDC
:102D50001306E07F13045000930620001364140050
:102D60006384D96093063000638AD95E63900960FA
:102D700093F6F70013054000638AA65E938647002A
:102D8000B3B7F6003307F700938706006F00005EC5
:102D90006388090093073000639CF9006394045230
:102DA0001307000093070000130450006FF0DFE9E1
:102DB000930720006398F950E39404FE6FF09FF8A6
:102DC000635CC00E639E050833E50601E30605AEAD
:102DD0001305F6FF631E050033880741B306D7408D
:102DE000B3B70701B386F640130610006F00400525
:102DF0009308F07FE30A16B1130680036348A60A1E
:102E00001306F001634AA606130600023306A64025
:102E1000B395C600B358A8003318C800B3E5150130
:102E20003338000133E80501B3D6A60033880741E3
:102E3000B306D740B3B70701B386F64013060400C4
:102E400037098000B3F72601E38607BE1309F9FFAF
:102E500033F92601130A0800130406006F008031BD
:102E60009305F07FE302B4ACB7058000B3E6B6008B
:102E7000130506006FF05FF8930505FE9308000246
:102E8000B3D5B6001306000063081501130600044D
:102E90003306A6403396C600336806013338000176
:102EA00033E80501930600006FF05FF833E8060190
:102EB000333800016FF01FFF630E06123386854022
:102EC000631404063365F700631805009307F07F69
:102ED000930403006FF0DFB59308F6FF63900802D8
:102EE000B307F8403338F800B386E640B3860641AE
:102EF00093040300138807006FF01FEF1305F07FA2
:102F00006310A606B3E70601638A073EB7074000D1
:102F1000B3F7F600138706006398073E930708008F
:102F2000930403006FF05FB91305F07F6394A5026B
:102F3000B3E706016380073EB7074000B3F7F6002A
:102F4000138706006390073E930708001306F07F7F
:102F50006FF01FFD370580003367A7009308060058
:102F600013068003634216091306F0016344160535
:102F700013050002330515413316A70033DE170190
:102F8000B397A7003366C601B337F000B367F60006
:102F900033571701B307F8403387E640B336F800DC
:102FA000B306D74013880700138605009304030077
:102FB0006FF01FE9138608FE130E00023356C70098
:102FC000130500006388C80113050004330515418B
:102FD0003315A700B367F500B337F000B367F60009
:102FE000130700006FF01FFBB367F700B337F00063
:102FF0006FF01FFF130614001376E67F63140614A8
:103000003365F70033E60601631A040C6310050804
:10301000631606249384E9FF93B414001307000099
:1030200093070000B3E6E7006382063293D6F70108
:1030300093151700B385D5009396170013F6760005
:1030400013040000630A0602130620006382C924E9
:10305000130630006380C92213041000639E090028
:1030600013F6F600130540006308A60093B6C6FFEA
:1030700093C61600B385D50093D5850193C5150079
:1030800093F51500130600006FF09FB2E30C06F8ED
:10309000B385074133B5B7003306D7403306A640A2
:1030A000370580003375A600630E0500B307F840AE
:1030B0003387E6403338F8003307074193040300B1
:1030C0006FF05FF6B3E7C5006390071A9384E9FFDA
:1030D00093B41400130700006FF0DFF49308F07F3F
:1030E000631A14036304052C37044000337487000B
:1030F0001334140013144400639215056300060290
:10310000B7054000B3F5B600639A0500130400014B
:103110006F00C00013040000E38215FF6310050276
:10312000630A062013870600930708009304030030
:103130006FF0DFAE130400006FF05FFCE30006AE3B
:103140006FF09FAF338A074133B647013309D74049
:103150003309C940370680003376C9006302060888
:10316000330AF840B386E6403338480133890641D4
:1031700093040300630C090613050900EF00406F78
:10318000130685FF9307F00163CAC7069306000282
:10319000B386C6403317C900B356DA00B3E6E6007B
:1031A0003318CA00634C860833068640130716009E
:1031B0009307F00163CCE704130600023306E640F0
:1031C000B397C6003355E8003316C800B3E7A7002D
:1031D0003336C000B3E7C70033D7E6006FF09FE493
:1031E000B3672A01E39807F86FF05FEE13050A0052
:1031F000EF000068130505026FF09FF8930685FD48
:10320000B316DA00130800006FF0DFF9130616FE9C
:103210009305000233D6C600930700006308B70089
:1032200093070004B387E740B397F600B367F8004D
:10323000B337F000B367F6006FF0DFE9B70780FF40
:103240009387F7FF3306C440B3F6F6006FF08FFEA6
:1032500013870600930708006FF0DFDC1387060072
:10326000930708006FF09FE513070600938705009A
:103270006FF05FDB13840400E39004E093B686FFF5
:1032800093C61600B385D500130410006FF0DFDE7F
:1032900013041000E38204DE93B686FF93C6160083
:1032A000B385D500138404006FF01FDD1307000001
:1032B0001306F07F6FF04FE6930708001306F07FC8
:1032C0006FF05FA51307F0FF9307F0FF1306E07F91
:1032D000930500006FF01FA813070000930700007C
:1032E0006FF09F9613070000930700006FF05FFCDC
:1032F00093070800930500006FF09F8B13070000F1
:10330000930403006FF05F94930708009304030095
:103310006FF05FFE130700001306F07F93040300B5
:103320006FF08FDF930708001306F07F930403000C
:103330006FF05F9E93070000930400003707400082
:103340001306F07F130400016FF01F9013070000B5
:1033500093070000130600006FF00FDC6398040071
:10336000938687006FF0DFA1E39C04FEE39C058455
:103370006FF09F8D930700006384090213073000EC
:10338000639AE900638E04009307F0FF1306E07F61
:103390006F00000113072000E398E9FEE38604FEB6
:1033A00013645400138707006FF05F8CE38485D8A3
:1033B000130400006FF0DFD6E38885861304000055
:1033C0006FF05F8513070500F3272000B707100093
:1033D0009387F7FF33F8B70093D54501B3F7D700CC
:1033E00093F5F57F93D646011305F07F93F6F67FAC
:1033F0006396A5003365E800631405029308F07F27
:1034000013050000639E1605B3E8C7006394080027
:10341000678000006398D5023367E800630E0700F9
:10342000370708003378E800630608021307F07FC7
:10343000130510006396E60233E6C700130510007B
:103440006300060237070800B3F7E7001305100012
:103450006398070073601800130510006780000070
:1034600067800000130101FFD30705E02326110048
:10347000232481002322910023202101732720008F
:1034800093D4770193F4F40F1387140013949700E7
:103490001377E70F1354940013D9F701630A070455
:1034A0001385043893573400930400001314D40197
:1034B0009397C7001315450193D7C700B367F5006D
:1034C0001319F90133E727011305040093050700D9
:1034D0006384040073A014008320C10003248100CE
:1034E00083244100032901001301010167800000CA
:1034F00063940404630A040613050400EF004037D4
:103500009307A00063C2A7029307B000B387A74048
:1035100013075501B357F4003314E4001307903830
:103520003305A7406FF0DFF8930755FFB317F4009A
:10353000130400006FF09FFE630E0402B707400003
:10354000B377F40063940700130700019357340026
:10355000B70608001314D401B3E7D700930407009B
:103560001305F07F6FF0DFF49307000013050000F0
:103570006FF01FF493070000930400006FF05FFEEC
:103580007328200013D745019378F77F9397C500E0
:103590001387180093D797009356D5011377E77FC9
:1035A000B3E6F60093D5F50193173500630A0716C5
:1035B000138608C81307E00F635AC706630E081C7A
:1035C00093073000631CF8006388051C9307F0FF25
:1035D0001306E00F130700006F00C00193072000DF
:1035E000E316F8FE639A051A130700009307F0FF2D
:1035F0001306E00F930850009306200093E818008C
:10360000630AD822930630006300D822631A0800A8
:1036100093F6F700130540006384A60093874700E4
:103620006302071893E828006F00C0176340C00CBE
:10363000130790FE634EE60E370780001305E00186
:10364000B3E6E6003305C5401307F0016348A7065B
:10365000138728C833D5A700B397E700B337F00026
:10366000B396E600B3E6D700B367D5006388071AC0
:10367000139717009376770093080000638606027D
:10368000930620006300D810930630006302D80E22
:1036900093081000631A08009376F70013064000A1
:1036A0006384C600130747001357B7011347170079
:1036B00013771700130600006F0040051307E0FFA3
:1036C0003306C7401303000233D6C60013070000B9
:1036D00063066500138728CA3397E600B367F700CF
:1036E000B337F000B367F6006FF05FF813156500AD
:1036F0003335A0009396360093D7D701B366D50033
:10370000B3E7F600130700009308000093F6770074
:10371000E39406EE6308070813F718006FF05FF0F4
:10372000B3E7F600639A080013060000638C0706EF
:10373000930710006FF0DFF3638C070C9307F07FA3
:103740006394F802B7084000B3F8160193B8180064
:103750009398480093963600B7070002B3E7F60047
:103760001306F00F6FF09FFA930800006FF09FFEB2
:1037700093880500E39A05F2130787009308100069
:103780006FF09FF293081000E38005F213078700A3
:10379000938805006FF05FF1930700001306F00FA8
:1037A000930850003707000433F7E700630E070063
:1037B000130616001307F00F6302E608370700FC34
:1037C0001307F7FFB3F7E7001307F00F93D737009E
:1037D0006318E60063860700B70740009305000002
:1037E000131676013707807F939797003376E600AC
:1037F00093D79700B367F6009395F501B3E7B70049
:103800006384080073A01800538507F067800000E8
:10381000930800001306F00F6FF0DFF813060000A6
:10382000930800006FF01FF8E39C05DE9387870084
:103830006FF01FDFE38605DE6FF05FFF9307000088
:103840006304080213073000631AE800638E050062
:103850009307F0FF1306E00F6F000001130720002D
:10386000E318E8FEE38605FE93E858006FF0DFF505
:10387000B7070100637AF5029307F00FB3B7A7000B
:10388000939737003757018093060002B386F640BE
:103890003355F500930787583385A7000345050086
:1038A0003385A640678000003707000193070001B9
:1038B000E36AE5FC930780016FF0DFFC93050500E8
:1038C0009306000013060000130500006F00C0629D
:1038D000B787018003A547B267800000130101FF8D
:1038E0009305000023248100232611001304050002
:1038F000EF00406AB787018003A507B28327C5039D
:1039000063840700E780070013050400EFC0DFF4BD
:10391000130101FF23248100B777018037740180F0
:103920001304441593874715B387874023229100DA
:103930002326110093D42740638004029387C7FF96
:1039400033848700832704009384F4FF1304C4FFA7
:10395000E7800700E39804FE8320C1000324810070
:10396000832441001301010167800000130101FF5E
:1039700023248100232021013774018037790180BD
:1039800093070415130909153309F940232611007B
:1039900023229100135929406300090213040415DE
:1039A000930400008327040093841400130444004C
:1039B000E7800700E31899FE3774018037790180AA
:1039C00093070415130949153309F9401359294080
:1039D0006300090213040415930400008327040004
:1039E0009384140013044400E7800700E31899FE51
:1039F0008320C100032481008324410003290100A6
:103A000013010101678000001303F0001307050094
:103A1000637EC3029377F7006390070A63920508F9
:103A2000937606FF1376F600B386E6002320B700F0
:103A30002322B7002324B7002326B700130707016A
:103A4000E366D7FE6314060067800000B306C34038
:103A50009396260097020000B38656006780C60042
:103A60002307B700A306B7002306B700A305B700D6
:103A70002305B700A304B7002304B700A303B700CE
:103A80002303B700A302B7002302B700A301B700C6
:103A90002301B700A300B7002300B7006780000030
:103AA00093F5F50F93968500B3E5D5009396050140
:103AB000B3E5D5006FF0DFF693962700970200007C
:103AC000B386560093820000E78006FA93800200D6
:103AD000938707FF3307F7403306F600E378C3F612
:103AE0006FF0DFF3130101FF3753018023268100BC
:103AF00093020500938705001303936803C707002B
:103B0000138E0700938717003308E30083480800EB
:103B100093F88800E39408FE130807001307D00207
:103B20006306E8101307B002630CE806B70F0080C5
:103B300093CFFFFF13040000638006081307000102
:103B4000138F06006382E610B3F3EF0393080000BF
:103B50001305000013039000930E900133DEEF0372
:103B6000130708FD6378E3001307F8FB63E4EE0630
:103B7000130798FC6358D70663CA08049308F0FF3C
:103B8000636AAE006302AE08930810003305E503D4
:103B90003305A7009387170003C8F7FF6FF05FFC9A
:103BA000B70F008003C8070093CFFFFF93072E00D5
:103BB00013040000E39406F8130700036300E80C05
:103BC000130FA0009306A0006FF01FF89308F0FFFA
:103BD0006FF05FFC1307F8F963E6EE00130798FA3D
:103BE000E34CD7F863C60802630404003305A04021
:103BF00063060600639608042320B6000324C10070
:103C00001301010167800000E3C6E3F86FF0DFF7FE
:103C10001307200223A0E20013850F00E30006FE35
:103C20009385F7FF13850F006FF01FFD03C8070092
:103C3000B70F008093072E00130410006FF0DFEF22
:103C4000930F05006FF0DFFD13070003631AE80010
:103C500003C70700130580051377F70D6306A70058
:103C6000130F00016FF05FEE03C81700130F000180
:103C700093872700930600016FF01FED03C707002D
:103C8000930680051377F70DE300D7FE130F80002E
:103C9000930680006FF05FEB130710006388E60067
:103CA000130740026364D7006FF0DFE3130101FFE5
:103CB00023261100EFF0DFC18320C10093076001CC
:103CC0002320F500130500001301010167800000A7
:103CD000130710006304E602130740026360C70283
:103CE0003787018093070500032547B29306060036
:103CF00013860500938507006FF0DFDE130101FFD7
:103D000023261100EFF0DFBC8320C1009307600180
:103D10002320F50013050000130101016780000056
:103D2000130710006304E602130740026360C70232
:103D30003787018093070500032547B293060600E5
:103D400013860500938507006FF0DFD9130101FF8B
:103D500023261100EFF0DFB78320C1009307600135
:103D60002320F50013050000130101016780000006
:103D7000130101F8232C8106B7870180232E110639
:103D8000232A910603A447B263CE05089307802037
:103D9000231AF1002324A100232CA100638605042B
:103DA0009387F5FF9304F0FF93058100130504004A
:103DB0002328F100232EF100231B9100EF00C02FD8
:103DC000635695009307B0082320F40083278100F1
:103DD000238007008320C107032481078324410730
:103DE00013010108678000009304F0FF9305810030
:103DF0001305040023280100232E0100231B91003A
:103E0000EF00802B635695009307B0082320F40041
:103E10008320C1070324810783244107130101087C
:103E2000678000009307B0082320F4001305F0FF1B
:103E30006FF01FFE130101F8232C8106232E1106BB
:103E4000232A91069307060013040500634E060813
:103E5000138606009306070013078020231AE1004B
:103E60002324B100232CB100638407049387F7FF58
:103E70009304F0FF930581002328F100232EF10025
:103E8000231B9100EF004023635695009307B00871
:103E90002320F40083278100238007008320C107AB
:103EA0000324810783244107130101086780000070
:103EB0009304F0FF9305810023280100232E0100C5
:103EC000231B9100EF00401F635695009307B00835
:103ED0002320F4008320C1070324810783244107A2
:103EE00013010108678000009307B0082320F50044
:103EF0001305F0FF6FF01FFEB787018003A707B21D
:103F000083278714638C070403A747001308F00175
:103F1000634EE80613182700630605023383070182
:103F20002324C30883A88718130610003316E6005D
:103F3000B3E8C80023A417192324D3109306200044
:103F40006304D5021307170023A2E700B387070114
:103F500023A4B70013050000678000009307C7146F
:103F60002324F7146FF05FFA83A6C718130717000E
:103F700023A2E70033E6C60023A6C718B3870701CC
:103F800023A4B70013050000678000001305F0FFAD
:103F900067800000130101FDB7870180232C4101D8
:103FA00003AA07B2232021032326110203298A141E
:103FB0002324810223229102232E3101232A51013D
:103FC0002328610123267101232481016300090450
:103FD000130B0500938B0500930A10009309F0FF63
:103FE000832449001384F4FF634204029394240061
:103FF000B304990063840B0483A74410638077059E
:104000001304F4FF9384C4FFE31634FF8320C1023A
:104010000324810283244102032901028329C1016F
:10402000032A8101832A4101032B0101832BC10053
:10403000032C8100130101036780000083274900DE
:1040400083A644009387F7FF638E870423A20400AE
:10405000E38806FA8327891833978A00032C4900DE
:10406000B377F70063920702E78006000327490051
:1040700083278A1463148701E38427F9E38807F808
:10408000138907006FF0DFF58327C91883A544085B
:104090003377F700631C070013050B00E780060069
:1040A0006FF0DFFC232289006FF09FFA1385050073
:1040B000E78006006FF09FFB130101E12326111E2C
:1040C000232A511D2328611D2320A11D138B0500C8
:1040D000130D06002326D1002324811E2322911EC6
:1040E0002320211F232E311D232C411D2326711D2A
:1040F0002324811D2322911D232EB11B930A050029
:10410000EF50102883270500138507002320F104B2
:10411000EF70902A8357CB002328010E232A010E2B
:10412000232C010E232E010E93F70708232EA10244
:104130006388070083270B01639407006F10C05644
:10414000B75701809387077D232AF10083470D002D
:10415000930BC110B76901802322710F2326010E32
:104160002324010E23280100232C01002322010413
:10417000232C01022324010423260104232201000D
:1041800093880B009389C994638E072013040D0054
:1041900093065002638AD73C83471400130414002B
:1041A000E39A07FEB304A441630EA41F8326C10E45
:1041B0008327810E23A0A801B3869600938717005A
:1041C00023A298002326D10E2324F10E930670001B
:1041D0009388880063C2F63A0327410083470400AE
:1041E000330797002322E100638E071A83441400EB
:1041F000A303010C130414001303F0FF130A0000BF
:1042000013090000130CA005930C9000930DA0025D
:1042100013041400938704FE6364FC040327410124
:1042200093972700B387E70083A7070067800700FD
:10423000130A0000938704FD8344040093162A00A8
:10424000338A4601131A1A00338A4701938704FD03
:1042500013041400E3F2FCFE938704FEE370FCFCFD
:104260006382041423069114A303010C130C1000A1
:10427000930C1000130DC114930D000013030000E4
:1042800023260102232A010223280102937F290009
:1042900063840F00130C2C00137F49088327C10E81
:1042A00063160F0033088A41E34E006B8346710C9E
:1042B000638A06028326810E1306710C23A0C800B0
:1042C00093871700130610009386160023A2C800D8
:1042D0002326F10E2324D10E130670009388880044
:1042E0006340D65C638A0F028326810E1306810C1D
:1042F00023A0C8009387270013062000938616008A
:1043000023A2C8002326F10E2324D10E1306700029
:1043100093888800E346D67493060008E302DF48DA
:1043200033089341E34A005593760910E39E063221
:104330000327810EB387970123A0A8011307170055
:1043400023A298012326F10E2324E10E9306700088
:1043500063C2E66A938888001379490063060900FE
:10436000B3048A416348906A63548A01130A0C00BB
:1043700003274100330747012322E100E39C075A4A
:104380002324010E63880D0093850D0013850A0018
:10439000EF20900593880B00130D040083470D0058
:1043A000E39607DE8327C10E638407006F10903504
:1043B0008357CB0093F70704638407006F204042C4
:1043C0008320C11E0324811E032541008324411E36
:1043D0000329011E8329C11D032A811D832A411D32
:1043E000032B011D832BC11C032C811C832C411C1E
:1043F000032D011C832DC11B1301011F67800000C9
:1044000013850A00232E110123246100EF50407709
:1044100083274500138507002326F104EF70C07938
:104420009307050013850A00938407002324F104F1
:10443000EF50007583278500032381008328C10185
:10444000232CF102638404006F10800F8344040066
:104450006FF01FDC83440400136909026FF05FDB17
:104460001369090193770902638A07688327C100EA
:104470009387770093F787FF03A7470083AD070073
:10448000938787002326F100930C07006342076A95
:104490001307F0FF130C09006308E30033E79D01E5
:1044A000137CF9F7E300077663840C006F10804CEF
:1044B000130790006374B7016F10C04B938D0D0309
:1044C000A307B11B13090C00930C1000130DF11A74
:1044D0008347710C130C030063549301138C0C007D
:1044E00023260102232A010223280102930D000042
:1044F000E38E07D8130C1C006FF05FD91369090114
:10450000937709026384075C8327C10013877700D0
:10451000137787FF832D0700832C470093078700BD
:104520002326F100137CF9BF13070000A303010C3D
:104530009306F0FF6302D362B3E69D011379FCF7A3
:10454000E39E0640E314030CE312076C937C1C000B
:10455000130D011BE38E0CF693070003A307F11A5A
:10456000130DF11A6FF0DFF6B304A441E310A4C5F4
:10457000834704006FF05FC71306410E93050B00DD
:1045800013850A00EF708076E31405E293880B0030
:104590006FF09FC493778900638407006F108001D8
:1045A0008327C1001305010B232E11019387770088
:1045B00093F787FF83A5070003A64700938787002B
:1045C000232461002326F100EF0001728327010BF1
:1045D0008328C101032381002328F10E8327410B87
:1045E000232AF10E8327810B232CF10E8327C10B85
:1045F000232EF10E1305010F232E11012324610038
:10460000EF5000502326A10C9307200003238100C4
:104610008328C1016314F5006F10405B93071000FD
:104620006314F5006F10807A930710066394F4000A
:104630006F20000D930710046394F4006F10104571
:1046400013F7F4FD9307F0FF2324E1066314F3004E
:104650006F10900F930770046314F7006F20001918
:10466000032EC10F232A2107832E010F032F410F91
:10467000832F810F9367091063540E006F10D07D54
:10468000232E010613890700930D000003278106DE
:10469000930760046314F7006F10D01A9307500457
:1046A000232411036314F7006F20400C130C010B3B
:1046B0009307010D1307C10C930603001308C10DE6
:1046C0001306200093050C0013850A0023226102C3
:1046D0002328D10B2320D103232AE10B232EE10130
:1046E000232CF10B2328F101232EC10B2324C1011C
:1046F000EF40000F0327810693077004032E81000B
:10470000832F0101032FC101832E010203234102E4
:1047100083288102130D05006304F7006F20003524
:104720008327410793F71700638407006F20400336
:104730008327C10D0327C10CB387A7412328F100AC
:104740002328E10203278106930770046314F7000E
:104750006F10500103278106930760046314F7006C
:104760006F10102F83270103032781069305100480
:104770009387F7FF2326F10C93F6F40F130600003E
:104780006318B7009386F60093F6F60F1306100031
:10479000230AD10C9306B00263DA07000327010352
:1047A000930710009306D002B387E740A30AD10C09
:1047B0009306900063C4F6006F20801F1308310E2B
:1047C000130508001306A000130E3006B3E6C70257
:1047D00093050500138307001305F5FF9386060371
:1047E000A38FD5FEB3C7C702E3426EFE93870703CC
:1047F00013F6F70FA30FC5FE9387E5FF63E40701E8
:104800006F2040279306610D6F00800003C60700EC
:104810002380C6009387170093861600E39807FF4E
:104820009307510EB387B7401307610DB307F70025
:104830009306410DB387D7402322F1048326410418
:104840000327010193071000B38CE60063C4E7005F
:104850006F20801A8327C103B38CFC008327410794
:1048600013CCFCFF135CFC4113F9F7BF136909106B
:1048700033FC8C0123260102232A01022328010292
:104880008327C107639407006F1000759307D00258
:10489000A303F10C13030000130C1C006FF01F9F07
:1048A0001306410E93050B0013850A0023206102B5
:1048B000232EE1012324F101EF704043E3160508A4
:1048C0008327C10E03230102032FC101832F81001F
:1048D00093880B006FF01FA10326810E03270101AF
:1048E0009306100023A0A8019387170093041600D5
:1048F000938C8800E3D4E6329306100023A2D800FC
:104900002326F10E2324910E93067000E3CE963CED
:104910000327C1038326010493841400B387E700AF
:1049200023A0DC0023A2EC002326F10E2324910E09
:1049300093067000938C8C00E3CA963C8326010F8B
:10494000138814009305010A2328D10A8326410FF6
:104950001305010B232EF100232AD10A8326810F90
:10496000232401012320010A232CD10A8326C10F0D
:104970002322010A2324010A232ED10A2326010A15
:10498000EFC0D06D832701010328810093888C003C
:104990009386F7FF130608008327C101E304052A65
:1049A00013071D00B387D70023A0EC0023A2DC006F
:1049B0002326F10E2324010F13077000E34207772B
:1049C00013870C0113862400938C080093080700BA
:1049D000832641041307410D23A0EC00B387D700C1
:1049E00023A2DC002326F10E2324C10E130770003E
:1049F000E354C7961306410E93050B0013850A0076
:104A0000EF70C02E631205748327C10E93880B00CC
:104A10006FF09F94930600010327810E63C49600F4
:104A20006F101006B7660180938EC69313090001BC
:104A3000930C70006F00C000938404FF635A9904C4
:104A4000938707011307170023A0D80123A2280189
:104A50002326F10E2324E10E93888800E3DEECFC8C
:104A60001306410E93050B0013850A002324D10180
:104A7000EF70C027631A056C938404FF8327C10E6F
:104A80000327810E832E810093880B00E34A99FA55
:104A9000B38797001307170023A0D80123A298001B
:104AA0002326F10E2324E10E93067000E3DEE68A4E
:104AB0001306410E93050B0013850A00EF700023C7
:104AC000631405688327C10E6FF01F8A8326C10017
:104AD0009377090113874600E396072C937709041F
:104AE000639407006F10C02C8327C100930C000053
:104AF0002326E10083DD07006FF0DFA28326C100DB
:104B00009377090113874600E394072893770904F4
:104B1000639407006F10C0258327C1002326E1009E
:104B2000839D070093DCFD4113870C00E352079639
:104B30003337B001B3079041B38CE7401307D0027D
:104B4000A303E10C9306F0FFB30DB041130C090071
:104B500013071000E312D39E93061000E306D794C8
:104B6000930620006300D72C130D011B1396DC0164
:104B700093F67D0093DD3D0093860603B36DB60189
:104B800093DC3C00A30FDDFE33E69D0193050D0091
:104B9000130DFDFFE31C06FC93771C00638E072AB0
:104BA00093070003638AF62A9385E5FFA30FFDFEB2
:104BB0009307011BB38CB74013090C00138D05003C
:104BC0006FF01F918327C100A303010C03AD070001
:104BD0009386470063140D006F10C0089307F0FF21
:104BE000E308F32E130603009305000013050D00E0
:104BF000232ED1002326110123246100EF50D00C75
:104C0000032381008328C1008326C101930D050081
:104C1000631405006F10C05AB30CA5418347710C93
:104C200013CCFCFF135CFC412326D1002326010298
:104C3000232A01022328010233FC8C01930D00007A
:104C400013030000E398078A6FF04FE40327C100C5
:104C5000A303010C130C1000832707001307470060
:104C60002326E1002306F114930C1000130DC11448
:104C70006FF08FE0136C090193770C02E38E07024B
:104C80008327C10013877700137787FF9307870077
:104C9000832D0700832C47002326F1001307100003
:104CA0006FF0DF8883440400136909086FF04FD662
:104CB0008327C1003787FFFF1347078383AD0700B2
:104CC0002314E10C93874700375701802326F10016
:104CD0009307C779930C0000136C2900232CF10073
:104CE00013072000930480076FF05F848326C100C0
:104CF0009377090203A70600938646002326D10076
:104D0000E392070693770901E39607749377090402
:104D1000638407006F10C01713790920E30C097230
:104D200083274100130D04002300F7006FF00FE705
:104D3000834404009307C006E380F4121369090159
:104D40006FF00FCD8344040093078006E38EF412C6
:104D5000136909046FF0CFCB834404001369890001
:104D60006FF00FCB8327C1008344040003AA070020
:104D7000938747002326F100635C0AC8330A404149
:104D8000136949006FF0CFC8834404001369190008
:104D90006FF00FC88347710C83440400639A07C601
:104DA00093070002A303F10C6FF08FC68344040045
:104DB000136949006FF0CFC59307B0028344040024
:104DC000A303F10C6FF0CFC48344040093061400D6
:104DD0006394B4016F105047938704FD1384060059
:104DE0001303000063E8FCC283440400131823008B
:104DF00033086800131818003303F800938704FD84
:104E000013041400E3F2FCFE6FF0CFC09306100011
:104E10006314D7006F10501493062000130C090080
:104E2000E314D7D4130D011B8327810193F6FD00F2
:104E300093DD4D00B386D70003C606009396CC01E0
:104E4000B3EDB60193DC4C00A30FCDFEB3E69D019C
:104E5000130DFDFFE39A06FC9307011BB38CA741DA
:104E600013090C006FF0CFE693065006E3D696A622
:104E70008326010F9305010A1305010B2328D10A8C
:104E80008326410F232EF10023241101232AD10A66
:104E90008326810F2320010A2322010A232CD10A11
:104EA0008326C10F2324010A2326010A232ED10AB7
:104EB000EFC0D01A832881008327C101631A053C03
:104EC0000327810EB75601809386C67C23A0D800A5
:104ED00093871700930610001307170023A2D8002A
:104EE0002326F10E2324E10E930670009388880098
:104EF000E3C2E6460327C10C83260101635AD76249
:104F0000032701048326C1039388880023ACE8FEAD
:104F10000327810EB387D70023AED8FE13071700EF
:104F20002326F10E2324E10E9306700063CEE67271
:104F3000032701019304F7FF635090C29306000119
:104F40000327810EE3D89642930C0001130D7000E5
:104F50006F00C000938404FFE3DE9C409387070149
:104F60001307170023A0380123A298012326F10E6E
:104F70002324E10E93888800E35EEDFC1306410EC6
:104F800093050B0013850A00EF605056631E051A47
:104F90008327C10E0327810E93880B006FF09FFBC0
:104FA00033088A41635E00B7130600018326810E31
:104FB000635C0607130E0001930E70006F00C000C3
:104FC000130808FF63520E079387070193861600A4
:104FD00023A0380123A2C8012326F10E2324D10ED9
:104FE00093888800E3DEDEFC1306410E93050B0078
:104FF00013850A00232E010123246100EF60104F66
:10500000631405140328C101130E00018327C10E88
:10501000130808FF8326810E0323810093880B0069
:10502000930E7000E3420EFBB387070193861600D0
:1050300023A0380123A208012326F10E2324D10E38
:105040001306700093888800635CD6AC1306410E8B
:1050500093050B0013850A0023246100EF601049BB
:105060006314050E032381008327C10E93880B0070
:1050700033089341635A00AB130600018326810E67
:105080006358060713030001130E70006F00C00081
:10509000130808FF635E03059387070193861600D4
:1050A00023A0380123A268002326F10E2324D10E69
:1050B00093888800E35EDEFC1306410E93050B0027
:1050C00013850A0023240101EF605042631E050688
:1050D00003288100130300018327C10E130808FF72
:1050E0008326810E93880B00130E7000E34603FBAA
:1050F000B38707019386160023A0380123A2080175
:105100002326F10E2324D10E130670009388880005
:10511000635CD6A01306410E93050B0013850A00AD
:10512000EF60D03C631205028327C10E93880B0009
:105130006FF08F9F1306410E93050B0013850A0035
:10514000EF60D03A630E05A263840DA693850D002F
:1051500013850A00EF1050296FF08FA5130C09007A
:105160006FF09F9F37670180130600018326810E31
:10517000930EC793130E000193027000634806015B
:105180006F004008130808FF635E0E07938707014E
:105190009386160023A0D80123A2C8012326F10E6E
:1051A0002324D10E93888800E3DED2FC1306410E3F
:1051B00093050B0013850A002324D10323226102E7
:1051C00023200103232EE1012324F101EF6010329B
:1051D000E31C05F603280102130E00018327C10E0C
:1051E000130808FF8326810E832E810203234102C8
:1051F000032FC101832F810093880B00930270005D
:10520000E3460EF9B38707019386160023A0D80161
:1052100023A208012326F10E2324D10E13067000C9
:10522000938888006354D6881306410E93050B00BB
:1052300013850A0023206102232EE1012324F101BA
:10524000EF60D02AE31205F08327C10E0323010289
:10525000032FC101832F810093880B006FF00F850E
:105260001306410E93050B0013850A00232E6100DF
:105270002324E101EF609027E31805EC8327C10E9A
:105280000323C101032F810093880B006FF0CF88A7
:105290008325C10C635CB07C0327010383260101D5
:1052A0009304070063C2E634635690028326810E9E
:1052B000B387970023A0A8019386160023A2980025
:1052C0002326F10E2324D10E130670009388880044
:1052D000E34CD63693C6F4FF0327010393D6F64179
:1052E000B3F4D400B304974063489042032701030A
:1052F00093760940B304ED00639406488325C10CFE
:105300000327010163C6E50093761900E3820636A0
:10531000832601040327C1031306700023A0D800CD
:105320008326810EB387E70023A2E8009386160048
:105330002326F10E2324D10E93888800E342D64E13
:10534000832601013307DD003386B64033079740DB
:10535000930C06006354C700930C07006356900338
:105360000327810EB387970123A098001307170026
:1053700023A298012326F10E2324E10E9306700048
:1053800093888800E3CEE66813C7FCFF1357F74104
:1053900033F7EC00B304E640634490006FE0DFFBBA
:1053A000930600010327810E63D6967C930C0001BF
:1053B000130D70006F00C000938404FF63DC9C7ABF
:1053C000938707011307170023A0380123A2980130
:1053D0002326F10E2324E10E93888800E35EEDFC82
:1053E0001306410E93050B0013850A00EF601010A1
:1053F000E31C05D48327C10E0327810E93880B007D
:105400006FF09FFB631C038A13090C001303000059
:10541000930C0000130D011B6FF08F8B9375190017
:10542000639C05CC23A2D8002326F10E2324910EE1
:10543000130770006346974E1306260093880801F1
:105440006FF00FD96356D0D8130700016344D7001B
:105450006F10005F130D70006F000001938606FF50
:10546000E350D70C138814009387070123A03C0155
:1054700023A2EC002326F10E2324010F930408003D
:10548000938C8C00E35C0DFD1306410E93050B001D
:1054900013850A002324D100EF605005E31605CAE6
:1054A0008327C10E8324810E83268100938C0B00F9
:1054B000130700016FF09FFA8326C10093770C0158
:1054C00013874600639C070A93770C04E382070C5A
:1054D0008327C100930C00002326E10083DD070031
:1054E000130710006FF08F841306410E93050B0015
:1054F00013850A00EF60807FE31805C48327C10E7F
:105500008324810E938C0B006FF08FC01306410E25
:1055100093050B0013850A00EF60407DE31605C27A
:105520008327C10E8324810E938C0B006FF00FC173
:1055300013771900631407006FE01FE26FF05F9CA0
:105540008327810383440400639407006FE05FCCEA
:1055500083C70700639407006FE09FCB136909407E
:105560006FE01FCB83264100130D040093D7F64153
:105570002320D7002322F7006FE05FE22326E1001B
:1055800083AD0600930C0000130710006FE01FFAB4
:1055900083AD06002326E10093DCFD4113870C0058
:1055A0006FE0DFEE83AD0600930C00002326E100E0
:1055B0006FE05FF70327C100832707001307470049
:1055C0002326E10083A5070003A6470083A68700E2
:1055D00083A7C7002328B10E232AC10E232CD10E86
:1055E000232EF10E6FF00F8193840600E34090CCE0
:1055F0006FF05FCE130C09006FF00FE8B757018012
:105600009387C779232CF10093770902638A072EC9
:105610008327C10013877700137787FF832D070047
:10562000832C4700930787002326F1001377190086
:10563000630E070033E79D01630A070013070003A9
:105640002304E10CA304910C13692900137CF9BF16
:10565000130720006FE09FED8344140013690902D3
:10566000130414006FE0DFBA1306410E93050B001C
:1056700013850A00EF608067E31805AC8327C10E2D
:1056800093880B006FF0DF8A8344140013690920AC
:10569000130414006FE0DFB7B75701809387077BCF
:1056A000232CF1006FF05FF69305000413850A00C8
:1056B000EF40C05E2320AB002328AB00631405003D
:1056C0006F10003C93070004232AFB006FE05FA7E4
:1056D00013050D00232411012326D100EF60C04DD6
:1056E0008347710C134CF5FF135CFC412326010228
:1056F000232A01022328010283288100930C05003C
:10570000337C8501930D00001303000063840700C0
:105710006FE05FDE6FE09FB7130600018326810E06
:105720006356966C930C0001130870006F00C00064
:10573000938404FF63DC9C6A9387070193861600B9
:1057400023A0380123A298012326F10E2324D10E91
:1057500093888800E35ED8FC1306410E93050B0086
:1057600013850A00EF608058E310059E8327C10E61
:105770008326810E93880B00130870006FF05FFB87
:1057800003270101130E7000130800013307ED0019
:105790002324E10003274103630E070A0327C10204
:1057A000631E070A032781031307F7FF232CE10277
:1057B000032741031307F7FF232AE1028326C104CD
:1057C000032781049388880023ACD8FE8326810EAA
:1057D000B387E70023AEE8FE938616002326F10E7A
:1057E0002324D10E6344DE1603278103834607007A
:1057F00003278100938C0600330697406354D6003C
:10580000930C0600635890038326810EB38797019B
:1058100023A098009386160023A298012326F10E58
:105820002324D10E634CDE3603278103938888003E
:105830008346070013C6FCFF1356F641B3FCCC00A9
:10584000B38C964163449003B384D400032741038F
:10585000E31607F40327C102630C076E0327C10296
:105860001307F7FF2326E1026FF05FF58326810E11
:10587000634898016F00C005938C0CFF635A98052C
:10588000938707019386160023A0380123A20801FD
:105890002326F10E2324D10E93888800E35EDEFCDC
:1058A0001306410E93050B0013850A00EF600044B8
:1058B000E31C058813080001938C0CFF8327C10E9D
:1058C0008326810E93880B00130E7000E34A98FB29
:1058D000B38797019386160023A0380123A298016D
:1058E0002326F10E2324D10E6342DE7003278103A9
:1058F0009388880083460700B384D4006FF01FF5B7
:105900008326C10093770901138746006386072227
:1059100083AD0600930C00002326E1006FF01FD139
:105920001306410E93050B0013850A00EF60003C3F
:10593000E31C05800326810E8327C10E93084111C5
:1059400013061600938C0B006FF08F881306410E20
:1059500093050B0013850A00EF604039631605FEBE
:105960008327C10E93880B0013080001130E7000EB
:105970006FF09FE713790C4023280100130D011BE2
:105980006F0040031306A0009306000013850D006E
:1059900093850C00232E110123246100EFB0806851
:1059A000032381008328C10163840C48930D050003
:1059B000938C05001306A0009306000013850D00CC
:1059C00093850C00232E110123246100EFB0D02811
:1059D0008327010113050503A30FADFE938717006D
:1059E0002328F100032381008328C101130DFDFF4B
:1059F000E30A09F80327810383460700E394D7F8F5
:105A00001307F00FE380E7F863960C00930790000C
:105A100063F4B7C5832781048325C104232E1101B4
:105A2000330DFD401386070013050D00232461008C
:105A3000EF604021832781031306A0009306000036
:105A400003CE170013850D0093850C00333EC00173
:105A5000B387C701232CF102EFB0C05C03238100A0
:105A60008328C101232801006FF05FF48326810E93
:105A7000375601801306C67C23A0C8009387170001
:105A8000130610009386160023A2C8002326F10EE9
:105A90002324D10E1306700093888800634CD60629
:105AA0006392051E0327010193761900B3E6E60011
:105AB000639406006FE05F8A832601040327C10315
:105AC0001306700023A0D8008326810EB307F700C9
:105AD00023A2E800938616002326F10E2324D10E7C
:105AE000634ED642938888000327010193861600EF
:105AF00023A0A801B307F70023A2E8002326F10E94
:105B00002324D10E130770006344D7006FE09F84F5
:105B10006FE05FEE1306410E93050B0013850A003C
:105B2000EF60C01C631205E28325C10C8327C10E00
:105B300093880B006FF0DFF693770904638C0720DE
:105B40008327C100930C00002326E10083DD0700BA
:105B50006FF0DFAD1306410E93050B0013850A00AD
:105B6000EF60C018631205DE8327C10E93880B0017
:105B70006FF04FB823A0380123A29800B387970095
:105B8000130717002326F10E2324E10E930670005D
:105B900063C4E6006FE00FFC6FE0DFE51306410E23
:105BA00093050B0013850A00EF604014631E05D8AF
:105BB0008327810393880B001308000183C6070025
:105BC000130E70008327C10E6FF0DFC68327010F0D
:105BD0009305010A1305010B2328F10A8327410FBE
:105BE000232411012320010A232AF10A8327810F8C
:105BF0002322010A2324010A232CF10A8327C10F3F
:105C00002326010A232EF10AEFB0D06C83288100ED
:105C10006342055A8347710C13077004635097223F
:105C200037570180130D077923260102232A010229
:105C3000232801021379F9F7130C3000930D0000AB
:105C4000930C300013030000638407006FE09F8A09
:105C50006FE0CFE383274100130D04002320F700FA
:105C60006FE0CFF393076000930C030063EE671EB1
:105C700037570180138C0C002326D100130D477C6D
:105C80006FE08FDF832601040327C1031306700032
:105C900023A0D8008326810EB307F70023A2E800D3
:105CA000938616002326F10E2324D10E93888800B4
:105CB0006346D626E3DA05E2130600FFB304B040DC
:105CC000E3D8C524930C0001130870006F00C000D6
:105CD000938404FFE3DE9C229387070193861600DA
:105CE00023A0380123A298012326F10E2324D10EEC
:105CF00093888800E35ED8FC1306410E93050B00E1
:105D000013850A00EF50907E631005C48327C10EEF
:105D10008326810E93880B00130870006FF05FFBE1
:105D20001386140013878C00B387D70023A2DC00EE
:105D300023A03C012326F10E2324C10E93067000FC
:105D4000E3C0C6BE1306160093088700930C070035
:105D50006FE01FC893770920638007168327C1006F
:105D6000930C00002326E10083CD07006FF01F8C09
:105D700093770920638607128327C1002326E10059
:105D8000838D070093DCFD4113870C006FE00FF05B
:105D900093770C20638607148327C100930C0000BF
:105DA0002326E10083CD0700130710006FE00FF8F2
:105DB00093770920638C07108327C100930C0000A0
:105DC0002326E10083CD07006FE0CFF58327C10FC5
:105DD00063C407128347710C13077004635C974810
:105DE00037570180130D87796FF01FE4B387970051
:105DF0009386160023A0380123A298002326F10ED3
:105E00002324D10E13067000938888006350D6CEE9
:105E10001306410E93050B0013850A00EF50106D19
:105E2000631405B28327C10E93880B006FF00FCC6B
:105E300093079000E3ECB7B76FF00F8237570180FC
:105E4000130DC7786FF05FDE1306410E93050B004C
:105E500013850A00EF509069631805AE8327C10EC1
:105E600093880B006FF00FC7930C60006FF05FE03A
:105E7000832601013307DD003386B64033039740A4
:105E8000930C06006352C3D0930C03006FF0CFCF86
:105E900083274100130D04002310F7006FE00FD09B
:105EA0008327C1002326E10083AD070093DCFD4179
:105EB00013870C006FE08FDD8327C100930C000077
:105EC0002326E10083AD07006FF04FF68327C10062
:105ED000930C00002326E10083AD07006FE08FE400
:105EE0008327C100930C00002326E10083AD070047
:105EF000130710006FE08FE39307D002A303F10CA8
:105F00006FF09FED1306410E93050B0013850A00F9
:105F1000EF50D05D8357CB006FE0CFC91306410E21
:105F200093050B0013850A00EF50505C631E05A01B
:105F30008325C10C8327C10E8326810E93880B0015
:105F4000E3D405BA6FF05FD7130360006FE04FF141
:105F500003270101B306ED0063F296BA93840600AD
:105F60006FF0CFB9032701039307D0FF6344F70015
:105F7000635AE3009384E4FF93F7F4FD2324F106CE
:105F80006FE04FFE83270101032701036340F726DB
:105F900083274107930C070093F7170063860700D8
:105FA0008327C103B30CF7008327410793F707400A
:105FB0006386070083270103E342F00413CCFCFF50
:105FC000135CFC4133FC8C01930470062326010210
:105FD000232A01026FE0DF8A8347710C130300005C
:105FE000638407006FE00FD16FE04FAA1306410EE4
:105FF00093050B0013850A00EF50504F631605946C
:106000008327810393880B001308000183C60700D0
:10601000130E70008327C10EB384D4006FF01F836A
:106020001306410E93050B0013850A00EF50104C28
:10603000631C05908325C10C8327C10E93880B0038
:106040006FF00FB0130C010B930603009307010DC3
:106050001308C10D1307C10C1306300093050C0083
:1060600013850A0023241103232261022328D10B64
:106070002320D103232AE10B232EE101232CF10B52
:106080002328F101232EC10B2324C101EF204075E9
:106090008346050093070003032E8100832F01012F
:1060A000032FC101832E01020323410283288102B1
:1060B000130D0500930C010A6384F6088327C10CB5
:1060C000B3876700B306FD0093850C0013050C0031
:1060D000232ED10023281101232461002328D10B72
:1060E000232AE10B232CF10B232EC10B2320010AC1
:1060F0002322010A2324010A2326010AEFB0007695
:106100008326C101032381008328010193870600B0
:10611000631405006FE00FE28327C10D63E4D7002D
:106120006FE04FE19305000313861700232EC10C87
:106130002380B7008327C10DE3E8D7FE6FE08FDF30
:10614000930C010A93850C0013050C002324110302
:10615000232261022328D10B2320D103232AE10B20
:10616000232EE101232CF10B2328F101232EC10B57
:106170002324C1012320010A2322010A2324010A26
:106180002326010AEFB0806D032E8100832F0101C9
:10619000032FC101832E01020323410283288102C0
:1061A000E30E05F093071000B38767402326F10C38
:1061B0006FF01FF19307D002A303F10C6FF0DFA57E
:1061C0008347710C2326D10023260102232A0102D2
:1061D00023280102130C0300930C03001303000097
:1061E000638407006FE00FB16FE04F8A83270101DE
:1061F0000327C10393047006B38CE70083270103D0
:106200006350F07E8327410793F70740639A075E48
:1062100013CCFCFF135CFC4133FC8C016FF01FDBE3
:106220001306410E93050B0013850A00EF50102C46
:10623000630405006FE05FF18324C10C03270101B3
:106240008327C10E93880B00330697406FF0CF93DE
:10625000832741070327010393F71700B3E767007C
:106260006356E07A639C0772832C010393046006F3
:106270006FF05FF937570180130D47796FF0DF9AA0
:10628000B7660180938EC6936FE09F8093070003EB
:106290002304F10C9307800513672900A304F10C74
:1062A000232AE10693073006930D0000130DC11455
:1062B00063C2673C032EC10F93F7F4FD2324F1065C
:1062C000232E0106832E010F032F410F832F810FF1
:1062D0001369291063460E38930710066388F45A31
:1062E000930710046384F4006FE04FBA130C010BA2
:1062F00013050C0023261103232461022328D10B4C
:10630000232AE10B232CF10B232EC10BEFE090404D
:106310001306C10CEF50404E13860500930505008F
:1063200013050C00EFE0501C93070109938507004B
:106330002324F1008327010B930C010A13060108A3
:106340002328F1088327410B13850C002326C1065F
:10635000232AF1088327810B232001082322010827
:10636000232CF1088327C10B23240108232EF108D5
:10637000B707FC3F2326F108EFB0900A0328010A73
:10638000032E410A832E810A032FC10A93850C0034
:1063900013050C002328010B23220103232AC10B20
:1063A0002320C103232CD10B232ED101232EE10B5B
:1063B0002328E1012320010A2322010A2324010AC0
:1063C0002326010AEFB08049032F0101832EC1016A
:1063D000032E010203284102032381028328C10204
:1063E00063160500930710002326F10CB7570180B0
:1063F0009387077B2322F1069306F3FF93070D0093
:106400006F00400993850C0013050C002320C10682
:10641000232EF105232C5104232A71042328F1048F
:10642000232A1103232861022328710A23267102DB
:10643000232A510A23245102232CF10B2322F10396
:10644000232EC10A2320C1022320010A2322010A8C
:106450002324010A2326010AEFB040408326C1010C
:10646000032F0102832E4102032E81020328C10261
:106470000323010383284103832701059386F6FF45
:106480009303080093020E00938F0E0013060F0073
:10649000630E05100326810093850C00232AF10268
:1064A00013050C00B70703402328D1042328110348
:1064B00023266102232EF1082326E10B2320010B62
:1064C0002322C10B2324D10B23280108232A0108EE
:1064D000232C0108EFB0C074832E010B032E410B57
:1064E0000328810B0326C10B13050C002324D103C1
:1064F0002322C10323200103232EC100EFE0C04E5D
:10650000930505002328A10013050C00EFE0806827
:106510000326C101832E8102032E4102232EC108CE
:106520000326010B03280102832581002320C108D3
:106530000326410B13850C002328D1092322C1080F
:106540000326810B232AC109232C01092324C10816
:106550000326C10B2326C1080326C106EFC0101B6A
:106560000327410683270101832601058323010AAE
:106570003306F70083450600832741038322410A3F
:10658000832F810A0326C10A232CF1062380B7003A
:106590002328D1061307F0FF232ED1000323C102C5
:1065A0008328010393871700E39EE6E4B706FE3FC6
:1065B00093850C0013050C002320F102232E1101FA
:1065C000232461002328710A23287102232A510AF7
:1065D00023265102232CF10B2324F103232EC10A7D
:1065E0002322C1022320010A2322010A2324010AB3
:1065F0002326D10AEFB04039032381008328C1014B
:1066000083270102634EA00893850C0013050C003C
:10661000EFB0C024032381008328C1018327010236
:10662000631805000327010193761700639A060695
:10663000032701071306000393061700B386D7004C
:10664000635407006FE00F8F93871700A38FC7FE77
:10665000E39CD7FE6FE00F8E930D000013890700B7
:10666000B707008033CEC7019307D002232EF1066F
:106670006FF09FC69305130013850A0023281101AC
:1066800023246100EF30806103238100832801010E
:10669000130D050063000540930D05006FF09FC1C9
:1066A0000327810793860700232EE10C0327410669
:1066B00003C6F7FF8345F7006310B6021305000316
:1066C000A38FA6FE8326C10D1386F6FF232EC10CD1
:1066D00003C6F6FFE386C5FE930516001305900377
:1066E00093F5F50F6306A600A38FB6FE6FE08F84C7
:1066F000032741068345A700A38FB6FE6FE08F8373
:10670000930700032304F10C930780076FF0DFB8B1
:10671000B38797009386160023A0380123A2980020
:106720002326F10E2324D10E13067000635CD6BA23
:106730001306410E93050B0013850A00EF50005B12
:10674000630405006FE05FA08327C10E8326810EDE
:1067500093880B006FF04FB9130C09006FD01FD650
:10676000B3066D00930C010A6FF01F96930C130093
:10677000130C010B1308C10D9307010D1307C10C76
:1067800093860C001306200093050C0013850A0065
:10679000232261022328D10B2320D103232AE10BDA
:1067A000232EE101232CF10B2328F101232EC10B11
:1067B0002324C101EF20C002032E8100832F010199
:1067C000032FC101832E010203234102832881028A
:1067D000130D0500B3069D01930C010A6FF0DF8EC7
:1067E0009307F0FF2322F1006FD09FBD63040300E5
:1067F0006FD01FE7130310006FD09FE6930470065D
:10680000832781039306F00F2326010283C7070025
:10681000232A01026388D7040327010363D4E70412
:10682000B307F740032781032328F10283471700AA
:10683000638E07000326410313071700232CE10290
:1068400013061600232AC1026FF0DFFC0327C102E2
:10685000832781031307170083C707002326E1025C
:106860006FF05FFB0327C10283274103B387E70073
:1068700003278104B387E702B38C970113CCFCFF95
:10688000135CFC4133FC8C016FD09FFF130C010B98
:1068900013050C0023261103232461022328D10BA6
:1068A000232AE10B232CF10B232EC10BEFE0806692
:1068B0001306C10CEF4050741386050093050500C4
:1068C00013050C00EFE04042930701099385070090
:1068D0002324F1008327010B930C010A13060108FE
:1068E0002328F1088327410B13850C002326C106BA
:1068F000232AF1088327810B232001082322010882
:10690000232CF1088327C10B23240108232EF1082F
:10691000B707FC3F2326F108EFB080300328010AB7
:10692000032E410A832E810A032FC10A93850C008E
:1069300013050C002328010B23220103232AC10B7A
:106940002320C103232CD10B232ED101232EE10BB5
:106950002328E1012320010A2322010A2324010A1A
:106960002326010AEFA0906F032F0101832EC1019E
:10697000032E010203284102032381028328C1025E
:1069800063160500930710002326F10CB75701800A
:106990009387C7792322F1066FF01FA68327C103CF
:1069A00093046006B30CF700B38C6C006FF09F8506
:1069B0009306610D6318060093060003230BD10CA8
:1069C0009306710D1307011B938707033386E64077
:1069D0002380F6009307D60D2322F1046FD01FE623
:1069E000B38CFC40938C1C0013CCFCFF135CFC416B
:1069F00033FC8C016FF08FDD8327410793F717007D
:106A0000639407006FD09FE56FD0DFE4639A0700BF
:106A1000130C100093046006930C10006FF00FDB52
:106A20008327C10393046006938C1700B38C6C001A
:106A300013CCFCFF135CFC4133FC8C016FF00FD9CD
:106A4000138708006FF04FAE8327C10003A3070030
:106A500093874700635403001303F0FF834414003B
:106A60002326F100138406006FD08FFA930C0300E5
:106A70006FF05FD6930720002322F1046FD01FDC54
:106A80009307C00023A0FA009307F0FF2322F10030
:106A90006FD01F938357CB0013E7070493070700BA
:106AA0002316EB006FD01F91130101FE2326310145
:106AB000B7790180232C8100232A9100232821010A
:106AC00023244101232E1100138A05001309050018
:106AD0009389496FEF30D02B03A78900B7170000C7
:106AE0001384F7FE832447003304444193F4C4FF26
:106AF000330494001354C4001304F4FF1314C400AB
:106B0000634EF4009305000013050900EF40D048E0
:106B100083A78900B38797006308F502130509006E
:106B2000EF3050278320C1010324810183244101D8
:106B3000032901018329C100032A810013050000F4
:106B40001301010267800000B305804013050900AE
:106B5000EF4090449307F0FF630AF504B787018084
:106B6000938787B403A7070083A68900B384844072
:106B700093E41400330487401305090023A2960010
:106B800023A08700EF3010218320C101032481015D
:106B900083244101032901018329C100032A8100C3
:106BA0001305100013010102678000009305000027
:106BB00013050900EF40503E03A789009306F0003B
:106BC000B307E540E3DCF6F4B786018083A686B21E
:106BD00093E717002322F7003305D540B7860180DD
:106BE00023A4A6B46FF09FF3638A0512130101FF7B
:106BF00023248100232291001384050093040500BF
:106C000023261100EF30D0180328C4FF130784FF98
:106C1000B77501809377E8FF3306F7009385456FDA
:106C20008326460003A5850093F6C6FF630AC51AAE
:106C30002322D600137818003305D6006310080A03
:106C4000032384FF0328450037750180330767401D
:106C5000832887001305C56FB38767001378180072
:106C60006380A8140323C70023A66800232413010C
:106C70006304081E93E617002322D7002320F600A2
:106C80009306F01F63E8F60A93F687FF9386860063
:106C900003A54500B386D50003A6060013D8570008
:106CA00093071000B3970701B3E7A700138586FF8A
:106CB0002326A7002324C70023A2F50023A0E60073
:106CC0002326E600032481008320C10013850400ED
:106CD00083244100130101016F30D00B03254500CF
:106CE00013751500631E050237750180B387D70041
:106CF0001305C56F8326860093E817003308F70055
:106D00006388A6160326C60023A6C6002324D60041
:106D1000232217012320F8006FF09FF66780000000
:106D200093E61700232ED4FE2320F6009306F01FCF
:106D3000E3FCF6F493D6970013064000636CD60E7E
:106D400093D66700138896031386860313183800BA
:106D50003388050183260800130888FF6308D812CA
:106D600003A646001376C6FF63F6C70083A6860017
:106D7000E318D8FE03A8C600232607012324D70062
:106D8000032481008320C1002324E800138504002C
:106D90008324410023A6E600130101016F30807FA8
:106DA000631608148325C60003268600B387F60001
:106DB000032481002326B60023A4C50093E6170010
:106DC0008320C1002322D700138504003307F70076
:106DD000832441002320F700130101016F30807BE1
:106DE00013781800B387D70063100802032584FFC7
:106DF0003307A7408326C70003268700B387A70071
:106E00002326D60023A4C600B786018013E6170008
:106E100083A6C6B22322C70023A4E500E3E4D7EA91
:106E2000B787018083A5C7B313850400EFF0DFC7E0
:106E30006FF05FE9130640016374D6021306400544
:106E40006364D60693D6C7001388F6061386E60653
:106E5000131838006FF0DFEFB387D7006FF09FE9AA
:106E60001388C6051386B605131838006FF05FEE59
:106E700023AAE50023A8E5002326A7002324A700D2
:106E8000232217012320F8006FF0DFE303A545005C
:106E900013562640930710003396C7003366A600AA
:106EA00023A2C5006FF05FED13064015636CD6009A
:106EB00093D6F700138886071386760713183800D1
:106EC0006FF01FE913064055636CD60093D6270177
:106ED0001388D6071386C607131838006FF05FE7CC
:106EE0001308803F1306E0076FF09FE693E6170054
:106EF0002322D7002320F6006FF0DFDC9306450045
:106F0000930700001305A5013788FFFF6F00C0013C
:106F1000939717002390E600939707019386260026
:106F200093D70701630ED50203D706001376170027
:106F30006304060093E717001357170013F62700A2
:106F4000B3650701E30606FC939717002390B6008C
:106F5000939707019386260093D70701E316D5FC84
:106F600067800000930685011307000013052500C4
:106F70006F00C001131717002390F60013170701C5
:106F80009386E6FF135707016304D50483D70600F1
:106F90001396070113560641939717006354060092
:106FA000136717009397070193D7070113762700FC
:106FB00093E51700E30006FC131717002390B600B3
:106FC000131707019386E6FF13570701E310D5FC5B
:106FD00067800000130101FE370E0100231D010030
:106FE000231E0100938585019307C10113088100C9
:106FF000130EFEFF03D705009387E7FF9385E5FF98
:1070000063180702239F07FEE39607FF1306460057
:107010009306E10103D70700938727001306260094
:10702000231FE6FEE398D7FE1301010267800000EC
:107030003307A70283D8270003D30700B376C7011D
:10704000B38616011357070193D80601330767006B
:1070500033071701935807012391D7002390E700C6
:10706000239F17FFE39807F96FF05FFA03570500B6
:10707000835725006306070037870000B3E7E70062
:107080002399F50003572500B78700009387F7FF82
:107090006304F702930765009385050113058501D5
:1070A00003D70700938727009385E5FF2391E50029
:1070B000E398A7FE67800000930765001305A5010C
:1070C00003D7070093872700631A0702E39AA7FEF6
:1070D000138725019387050093872700239F07FEC9
:1070E000E31CF7FE83D72501378700001307F7FF5E
:1070F000B3E7E7002399F5006780000013870501D7
:107100009387050093872700239F07FEE31CF7FE64
:10711000B7C7FFFF2398F500B787FFFF93C7F7FFB7
:107120002399F5006780000083574500130101FF94
:1071300023229100232611002324810023202101F2
:1071400093040500639C070C0357650013040000BB
:107150009317070193D7074163C4070A9306A50154
:107160001306000A63180702938764006F0080000B
:1071700003D7070093872700239EE7FEE39AD7FEF5
:10718000239C040013040401630CC40603D76400A9
:10719000E30C07FC937707F06390070413858401E1
:1071A000938524009307000013070500835607000A
:1071B0001307E7FF13968600B3E7C7002311F70014
:1071C00093D78600E394E5FE03D76400130484009C
:1071D000937707F0E38807FC1309000A6F0040016A
:1071E00013041400EFF01FD8634C890003D7640028
:1071F000131707011357074113850400E35207FED5
:107200008320C1001305040003248100832441006E
:1072100003290100130101016780000013F707F043
:1072200013040000631007041309F0F66F00400117
:107230001304F4FFEFF09FCCE30424FD83D7440054
:1072400013850400E39607FE8320C10013050400A4
:10725000032481008324410003290100130101015B
:1072600067800000930645009305A5011307000001
:107270006F00800083D7060013D687003367C700EE
:10728000939787002390E6001397070193862600C3
:1072900013570701E390D5FE83D74400130480FF02
:1072A0006FF09FF8130101FE232C8100232A910027
:1072B000232E110023282101232631019384050068
:1072C0001304050063C4050A9307F0001386050044
:1072D00013054500930684019305F00063D49702DB
:1072E0009307050003D7270093872700239FE7FE16
:1072F000E39AF6FE231C0400130606FFE3C2C5FE54
:1073000093F4F4009307700063D897021307840185
:107310009305240093070000835607001307E7FF37
:1073200013968600B3E7C7002311F70093D78600B2
:10733000E394E5FE938484FF638A04009384F4FF5E
:1073400013050400EFF01FC2E39A04FE13050000CA
:107350008320C10103248101832441010329010108
:107360008329C1001301010267800000930710FF09
:107370003309B04063DEF5129305850193090000DF
:10738000930645001306F000035784019387050018
:10739000B3E9E90003D7E7FF9387E7FF2391E7000D
:1073A000E39AD7FE23120400130909FFE34E26FDDA
:1073B000130900FF130710FF3309994093070000DA
:1073C00063C6E40A3309F9009307700063CA27050E
:1073D0006302090C835784011309F9FF13050400A4
:1073E00093F71700B3E93701EFF05FB1E31409FE3B
:1073F0009397090193D707416396070813950901ED
:10740000135505018320C101032481018324410117
:10741000032901018329C1001301010267800000D3
:107420009399090193D90941834784019305A401E4
:10743000B3E9F9009399090193D909019307000071
:1074400003D706009386260013568700B3E7C700CC
:1074500013178700239FF6FE9317070193D70701A1
:10746000E390D5FE130989FF6FF09FF6937709FF2C
:10747000B307F0403309F90093077000E3DA27F50A
:107480006FF01FFA930910001395090113550501B8
:107490006FF05FF713850900639809001315050164
:1074A000135505016FF0DFEA130510006FF01FFFA1
:1074B000930790FF9309000093064500E3C6F5F695
:1074C0006FF05FF183572501378600001306F6FF42
:1074D00093D7F700B307F0402390F50083562501BA
:1074E0009307050113874500B376D6002391D50095
:1074F0006386C60213876500239205001305E5FF26
:1075000083D607009387E7FF13072700231FD7FEC3
:10751000E318F5FE239C0500678000000356250153
:1075200033F6C600631ED600130825019306050036
:1075300003D6060093862600631E0600E39A06FF24
:107540009385A50113072700231F07FEE39CE5FE93
:107550006780000013876500239205001305C5FFAF
:1075600083D607009387E7FF13072700231FD7FE63
:10757000E398A7FE6780000083572501130101FBF4
:107580002324810493C7F7FF2326110413971701BF
:1075900013840500631E0700930625019307050069
:1075A00003D7070093872700631C0708E39AD7FED9
:1075B0008357240193C7F7FF13971701630007064A
:1075C00093058100EFF01FF09305410213050400BD
:1075D000EFF05FEF8355810003554102630CB50660
:1075E0009307A100130761021306010283D6070067
:1075F000938727006398060A83560700130727001E
:107600006392060AE314F6FE130500008320C1040A
:10761000032481041301010567800000930704001F
:1076200003D707009306240193872700631A0700F6
:10763000E388D7F803D7070093872700E30A07FEFC
:107640008320C104032481041305E0FF1301010515
:10765000678000000356A1008356610213351500B0
:107660001307A10093076102131515001305F5FF19
:107670009305C1039387270013072700631ED600D5
:10768000E384B7F80356070083D6070013072700E3
:1076900093872700E306D6FEE3EAC6F63305A0404B
:1076A0006FF0DFF613051000E38205F61305F0FF17
:1076B0006FF0DFF5130101FE232C8100232A9100D6
:1076C00023282101232631012324410123225101B2
:1076D0001389060093840700232E1100130405006C
:1076E00093890500130A0600930A0700EFF0DFA351
:1076F000930700093309A94063DCA718B787000086
:107700009387E7FF63DA272163840A1E03A54400F9
:1077100083A70400630AF5061387A4019387440333
:1077200013072700231F07FEE31CF7FE93078003C0
:107730006300F53663D0A71893070004630EF52E97
:10774000930710076310F532B78700409387F7FF60
:107750001307A00023AAF400B787FFFF23A4E400C7
:10776000239CF40023A6E4009307A00037870000C1
:107770009387870093971700B387F4002395E7005A
:1077800023A0A4006358201D83A5840083D744014F
:107790001308F008139615003306C40003570600BB
:1077A000B376F700634AA8021308B0006346B80234
:1077B000930706009305840103D72700630407009D
:1077C00093E616002391070093872700E396F5FEC2
:1077D0000357060083D7440193C7F7FFB3F7E700C9
:1077E0002310F60083D7640133F7D7006300070640
:1077F0006392D7026398092083A7C40003D784014A
:1078000093971700B307F40083D70700B3F7E70097
:10781000638E070213862403930684019384C401B4
:10782000130700008357060083D506009386E6FF02
:107830001306E6FFB387B700B387E70013D7070146
:107840002391F60013771700E31E96FC635620176A
:1078500083574400639E0712B7870000231C04006F
:107860009387E7FF63C82709231124018320C101FF
:107870000324810183244101032901018329C100DB
:10788000032A8100832A410013010102678000005E
:107890006354090E930700F7635CF908930724000B
:1078A0001304A40193872700239F07FEE39C87FE10
:1078B0006FF0DFFB93078001630AF5149307500311
:1078C0006312F51A37170000B7070004930660002B
:1078D0009387F77F1307078023AAF40023A4D4001B
:1078E000239CE40023A6D400930760006FF05FE8B8
:1078F000231C0400B787FFFF93C7F7FF2311F40091
:107900009307440013048401239007009387270002
:10791000E31CF4FE6FF09FF5930724001304A40109
:1079200093872700239F07FEE39C87FE6FF01FF4D9
:107930009305090013050400EFF0DF9663040500CA
:1079400093091000638A0A0A03A5440083A7040070
:10795000E314F5DC930700096302F50883578401FB
:107960001305040093F71700B3E9F900EFF00FD9FE
:1079700003A544006FF05FE1E3800AEE03A5440035
:1079800083A70400E31AF5D8E34020E16FF09FFCE1
:1079900013050400EFF08FD6B78700001309190014
:1079A000231C04009387E7FFE3C627F5E35E09EA9B
:1079B000231104006FF09FEB930700096306F500A5
:1079C00013050400EFF00FDA83574400E39207FC3D
:1079D000231C0400E34E09FC6FF01FE903A684009A
:1079E00083D74401131616003306C400035706005C
:1079F000B3F6E7006FF05FDE231C040023110400E0
:107A00006FF0DFE6E3080AE06FF05FE4B70780009D
:107A10009387F70F1307400023AAF4009307001081
:107A200023A4E400239CF40023A6E4009307400071
:107A3000130700106FF0DFD39307700023A4F40046
:107A4000B70701809387F7FF23AAF400930710007C
:107A5000239CF4009307600023A6F4001307100092
:107A60006FF01FD19307C00023A4F400B707018073
:107A70009387F7FF23AAF40093071000239CF400D8
:107A80009307B00023A6F400130710006FF05FCE39
:107A9000B70780009387F70F1307600023AAF4004D
:107AA0009307001023A4E400239CF40023A6E40021
:107AB00093076000130700106FF09FCB130101FDC7
:107AC00023202103232E310113890500835925002A
:107AD000232611022324810223229102232C410117
:107AE0009304060023267101232A510123286101F2
:107AF00023248101232291012320A101930B05005E
:107B0000EFF08FE2035429009307050013050900E5
:107B1000B389F940138A4403EFF00FE13304A44022
:107B20001387E40493070A0093872700239F07FE27
:107B3000E39CE7FE63483409138B4B00930A49002A
:107B4000138CAB01130D290013870A0093070B0058
:107B500003D60700835607009387270013072700E3
:107B6000631AD60AE39687FF13868B0113078901F0
:107B70009306000083570700835506001307E7FFAD
:107B8000B387D740B387B74093D607012311F700D7
:107B900093F616001306E6FFE31EEDFC930C1000AF
:107BA00013050A00EFF00FBC83D7C4041304F4FFDD
:107BB00013050900B3E7FC002396F404EFF08FBA35
:107BC000E35434F993060400032481028320C102A4
:107BD0008329C101032A8101832A4101032B010169
:107BE000832BC100032C8100832C4100032D010055
:107BF000938704001305090083244102032901022D
:107C00001307000013060000930500001301010391
:107C10006FF05FAA930C0000E3E4C6F86FF0DFF4A6
:107C2000130101F723229108930405000355250150
:107C3000378700001307F7FF232481082320210939
:107C4000232C410723261108232E3107232A51070D
:107C50002328610723267107232481072322910704
:107C60003375A7001389050013040600138A060064
:107C7000631EE5009389240113870400035607005F
:107C800013072700631E0622E31A37FF0356290154
:107C9000B78700009387F7FFB375F6006394F5127A
:107CA00093062901130709008357070013072700CC
:107CB00063960722E39AE6FEB78700009387F7FFF3
:107CC0006304F5109307090003D707009387270083
:107CD0006318071CE39AF6FEB76501809385459803
:107CE00013850400EFF05F896308052003D52401A4
:107CF00003562901B78700009387F7FF3378F50013
:107D0000B375F600630AF81AB78700009387F7FF88
:107D10006390F514930629019307090003D7070020
:107D20009387270063160712E39AD7FE3787000070
:107D30001307F7FF9358F500930508009389240172
:107D40006304E80E0357090013092900631807327A
:107D5000E31AD9FE9357F600B3871741B337F00003
:107D60009397F7002319F4001307240193070400E5
:107D700093872700239F07FEE39CE7FE8357240198
:107D8000378700001307F7FFB3E7E7002319F40074
:107D90008320C108032481088324410803290108A2
:107DA0008329C107032A8107832A4107032B01077F
:107DB000832BC106032C8106832C41061301010984
:107DC000678000006316F5089389240193870400F7
:107DD00003D7070093872700631A072AE39AF9FE5F
:107DE000B76501809385459813050900EFF0CFF83A
:107DF0006304051003562901B78700009387F7FF36
:107E0000B375F6006380F51203D524013377F500CE
:107E10006310F7049387040003D7070093872700B4
:107E20006314072AE39AF9FE83D70400938424009D
:107E3000639A0724E39A34FF9358F50037870000CC
:107E40001307F7FFE398E5F0930629016FF09FEF22
:107E5000138504009305C100EFF0CFE6930581027E
:107E600013050900EFF00FE68354E1008359A102E6
:107E7000639E040A93070101930641026382D7229D
:107E800003D7070093872700E30A07FE1305C10005
:107E9000EFF08FA90357A102B304A0406F0040097F
:107EA00003D52401B78700009387F7FFB375F5006A
:107EB00013880500E392F5E6938924016FF09FF59E
:107EC0001387440183D704009384240013042400FF
:107ED000231FF4FEE398E4FE6FF09FEB13074401C9
:107EE000835709001304240013092900231FF4FEFB
:107EF000E318E4FE6FF0DFE91307040193070400C1
:107F000093872700239F07FEE39CE7FEB7C7FFFF89
:107F10002318F400B787FFFF93C7F7FF2319F40076
:107F20006FF01FE7930629016FF0DFD9138709006F
:107F3000138909009307C102930601046312070223
:107F4000638AF61603D7070093872700E30A07FE24
:107F500013058102EFF04F9D0357A1023389A94019
:107F60008357810293098A03231BEA02231AFA0228
:107F70001307EA04938709002390070093872700DB
:107F8000E31CF7FE130CCA04930B0000930A410292
:107F9000930C0101130B610403D50A00938AEAFFD5
:107FA000631C05088357CA0413070C00B3EBFB00DE
:107FB0000356E7FF1307E7FF2311C700E39AE9FE23
:107FC000231C0A02E39A9AFD13074A0393078102CE
:107FD0001306210483560700938727001307270001
:107FE000239FD7FEE318F6FEB7C6FFFFB384240134
:107FF0009386260093850B001305810293070A00E0
:1080000013070004B386D40013060000EFF08FEAD4
:10801000035781028357C1009305040013058102B1
:10802000B387E740B337F000B307F0402314F10201
:10803000EFF0CF836FF0DFD5130641049305810283
:10804000EFE05FF913050C00930500001306C1056E
:1080500083570500035706001305E5FF1306E6FFE7
:108060003307F7003307B700935507012311E500E5
:1080700093F51500E31E66FD6FF0DFF29307000035
:108080006FF09FCD930800006FF05FDBB7870000B3
:108090009387F7FFE388F5E803D524016FF09FD7B6
:1080A0009307440113042400231F04FEE31CF4FE81
:1080B0006FF01FCE9307440113042400231F04FE16
:1080C000E31CF4FE6FF0DFCC378800001308F8FFE4
:1080D0006FF09FC383572501130101F52324810A03
:1080E00093C7F7FF2322910A2320210B232E310966
:1080F0002326110A232C4109232A51092328610927
:108100002326710923248109232291092320A1090F
:10811000232EB10713971701930405001389050057
:108120001304060093890600631E070093062501C9
:108130009307050003D707009387270063120730D2
:10814000E39AD7FE8357290193C7F7FF13971701C7
:10815000631E0700930629019307090003D7070050
:1081600093872700631C072EE39AF6FE376A018087
:1081700093054A9813850400EFF00FC0630E052E97
:1081800003D6240183552901B78700009387F7FFA1
:108190003375F600B3F6F5006316F50A138824016B
:1081A0009387040003D70700938727006318070805
:1081B000E39A07FFB78700009387F7FF639AF62CCF
:1081C000930629019307090003D707009387270027
:1081D000631C0748E39AD7FE1307040193070400C2
:1081E00093872700239F07FEE39CE7FEB7C7FFFFA7
:1081F0002318F400B787FFFF93C7F7FF2319F40094
:108200008320C10A0324810A8324410A0329010A25
:108210008329C109032A8109832A4109032B010902
:10822000832BC108032C8108832C4108032D0108EE
:10823000832DC1071301010B67800000B787000081
:108240009387F7FF6380F626138504009305C10129
:10825000EFF04FA79305810313050900EFF08FA6F8
:10826000835AA1038354E10163860A2C232651011A
:10827000138604002324910093070102930641030F
:10828000631206026384F63A03D707009387270038
:10829000E30A07FE1305C101EFE01FE9B387A4401D
:1082A0002324F10003278103938A890393870A001B
:1082B00023AAE9029384E90493872700239F07FEFA
:1082C000E39C97FE13058103EFE05FC3035B21028C
:1082D00037090100130C0105131A0B01330A6A4117
:1082E000930CA1031309F9FF130DE106930D61052A
:1082F0008357C1030357E103930B090093970701C9
:10830000B387E7006368FA0033D56703931B050161
:1083100093DB0B01130641059305C10113850B0087
:10832000EFE05FCB1307C1039307810503D6070076
:108330008356070093872700130727006314D6226C
:10834000E396A7FF930700009306C10613060C00EF
:108350000357060083D506001306E6FF3307F740F0
:108360003307B740935707012311E60093F717002F
:108370009386E6FFE31E96FD23907A019307C103DF
:1083800003D7270093872700239FE7FEE39A87FF01
:1083900023180104938A2A00E39C54F51307000074
:1083A0009307C1031306210583D60700938727008F
:1083B0003367D700E39AC7FE9317070193D70741A6
:1083C00063840700130710009315070193D5050177
:1083D0001387490393078103835607009387270078
:1083E00013072700239FD7FEE318F6FE8327C1005B
:1083F00003278100B74600009386F6FFB38AE74063
:10840000130581039387090013070004B386DA007C
:1084100013060000EFF00FAA035781038357C10131
:108420009305040013058103B387E740B337F000D9
:10843000B307F040231CF102EFE05FC36FF05FDC95
:108440001387440183D70400938424001304240079
:10845000231FF4FEE398E4FE6FF09FDA130749014F
:10846000835709001309290013042400231FF4FE75
:10847000E318E9FE6FF0DFD893054A981305090069
:10848000EFF08F8FE31E05CE6FF01FD5E30E08DAF5
:108490009307440113042400231F04FEE31CF4FE8D
:1084A0006FF01FD6130800009306290193070900F7
:1084B00003D7070093872700E31A07FCE39AD7FE48
:1084C000B78700009387F7FF630AF5041356F60099
:1084D000835709001309290063900718E31AD9FE8E
:1084E00093D5F5006384C500378700002319E400A5
:1084F000930704001307240193872700239F07FE97
:10850000E39CE7FE83572401378700001307F7FF3A
:10851000B3E7E7002319F4006FF09FCE1385240121
:1085200083D7040093842400639C0712E39AA4FE7B
:108530006FF0DFF99307C103130C0105630EFC0C08
:1085400003D7070093872700E30A07FE130581037B
:10855000EFE09FBDB307A0400356E1012326F100E1
:108560006FF05FD1E3F0C6DE9387FBFF93980701BE
:1085700093D8080193060000130641031307C106B0
:1085800083570700835506001307E7FFB387D740DB
:10859000B387B74093D607012311F70093F616006F
:1085A0001306E6FFE31EB7FD1307C103930781051A
:1085B00003D6070083560700938727001307270079
:1085C0006318D600E396A7FF938B08006FF09FD740
:1085D000E3FCC6FE1385EBFF931B050193DB0B0148
:1085E00093060000130641031307C10683570700D3
:1085F000835506001307E7FFB387D740B387B7401B
:1086000093D607012311F70093F616001306E6FF31
:10861000E31EB7FD6FF01FD393074401130424003A
:10862000231F04FEE31CF4FE6FF09FBD0357C1013E
:10863000835781036304F700378600002319C400C1
:10864000130724019307040093872700239F07FE45
:10865000E39CE7FE6FF01FEB930500006FF09FE8CF
:10866000130600006FF0DFE6130810006FF01FE440
:10867000130101FD23248102232611021384050026
:10868000930741001307E10193872700239F07FE0B
:10869000E39CE7FE0356E5009317060193D70741D5
:1086A00063CA0706B78700009387F7FF231201000C
:1086B0003376F600630CF6069307E5002313C1003A
:1086C0001307A10083D6E7FF9387E7FF130727006F
:1086D000231FD7FEE318F5FE6312060223140100E0
:1086E0009305040013054100EFE05F988320C10269
:1086F0000324810213010103678000009307100027
:108700009305F0FF130541002314F100EFE09FB93A
:108710006FF01FFD9307F0FF2312F100B7870000F1
:108720009387F7FF3376F600E318F6F89307050012
:108730009306E50003D7070093872700631C07060D
:10874000E39AF6FE1307440193070400938727007A
:10875000239F07FEE39CE7FE130724019307040011
:1087600093872700239F07FEE31CF7FE835724010E
:10877000B78600009386F6FFB3E7D700939707010B
:1087800093D707012319F4008316E500E3D006F61A
:108790009306040003D6060093862600E31806F429
:1087A000E31AD7FE3787FFFFB3C7E7002319F400AA
:1087B0006FF0DFF31307040193070400938727008A
:1087C000239F07FEE39CE7FEB7C7FFFF2318F400D3
:1087D000B787FFFF93C7F7FF2319F4006FF01FF16E
:1087E00083A8C500130101E183AE050003AE450077
:1087F00003A38500232E1103832505049308F0FFAE
:1088000023201117930800092324811E232C411DC6
:108810002326111E2322911E2320211F232E311DCA
:10882000232A511D2328611D2326711D2324811D08
:108830002322911D2320A11D232EB11B2328D10308
:10884000232AC103232C6102232211172322C100F2
:108850002326D1002328E100232C0101130A05005F
:108860001384070063800502032745049307100063
:10887000B397E70023A2E50023A4F500EF10505CB6
:1088800023200A04130901069305090013050103B7
:10889000EFF01FDE03562107378700001307F7FFAD
:1088A000B375E600639EE5001307090093072107EF
:1088B0008356070013072700E3960646E31AF7FEE0
:1088C0001356F600032741002320C400930730000D
:1088D000E300F714930740012324F100E318074451
:1088E00003274116B78700009387F7FF232AE1008B
:1088F000639EF500930709009306210703D707003D
:1089000093872700E3120718E39AD7FE930700091D
:108910002322F1161307C107930709001306410725
:1089200083D607009387270013072700231FD7FE4E
:10893000E398C7FE0356E1082320010093170601C0
:1089400093D7074163CA0760376B0180130C4B98BC
:10895000930B4C01930600009307810913870B00CA
:10896000930DC10A6F00800083560700938727008C
:10897000239FD7FE13072700E398B7FF6308061469
:10898000B78700009387F7FFE30AF6568317C108FD
:10899000E3D8075E9305C10713850B00EFE0DFBD49
:1089A00063020514E34205108357E108E39A076662
:1089B0008317C108930400009309011663C40702DA
:1089C00013048C111306C107938609009305060052
:1089D00013050400EFF0CFA48317C1089384F4FFBC
:1089E000E3D207FE1304010D930A810E130704005E
:1089F0009307C1071306010983D607009387270051
:108A000013072700231FD7FEE398C7FE9306000035
:108A10009307810913870B006F00800083560700BE
:108A200093872700239FD7FE13072700E398B7FFFC
:108A3000930C8C02930DCC1237FDFFFF130C8C119D
:108A40006F00C000938D4D01938C4C019305040081
:108A500013850B00EFE05FB2930705009305040058
:108A600013850D006356F004EFE01FB19307050076
:108A700093860900130604009305040013850C0077
:108A800063C00702EFF0CF991306810993860900AE
:108A90009305060013850C00EFF08F98B384A401B2
:108AA0009357FD01338DA701135D1D40E39C8CF9A5
:108AB000130681099386090093850B0013050600B0
:108AC000EFF04FE1930C41126F0000039307C107D1
:108AD0009306E10803D7070093872700E31C07EA02
:108AE000E39AF6FE93040000930C411293090116D9
:108AF0001304010D930A810E9305040013058109E7
:108B0000EFE05F9C130781099307040083D60700F9
:108B10009387270013072700231FD7FEE39857FFEB
:108B2000930504001305C1072318010AEFE09F997C
:108B30009307C107035704001304240093872700F9
:108B4000239FE7FEE31854FF1305810913860900EC
:108B50009305C107231A0108EFE05FF60355C11A18
:108B60006314051C930B4109130DE1071304610BFA
:108B700093054B981305C107EFE01FA06306051A84
:108B80001307000093860B006F00C0011317170036
:108B90002390F600131707019386E6FF135707018A
:108BA0006384A60583D70600139607011356064172
:108BB00093971700635406001367170093970701F4
:108BC00093D707011376270093E51700E30006FC0F
:108BD000131717002390B600131707019386E6FFBB
:108BE00013570701E390A6FD1307410B9307C10735
:108BF00083D607009387270013072700231FD7FE7C
:108C0000E39877FF2316010C130700009306C10CAD
:108C10006F00C001131717002390F6001317070108
:108C20009386E6FF135707016384860483D7060003
:108C300013960701135606419397170063540600D5
:108C4000136717009397070193D70701137627003F
:108C500093E51700E30006FC131717002390B600F6
:108C6000131707019386E6FF13570701E39086FC6D
:108C7000130700009306C10C6F00C0011317170003
:108C80002390F600131707019386E6FF1357070199
:108C90006384860483D706001396070113560641A2
:108CA0009397170063540600136717009397070103
:108CB00093D707011376270093E51700E30006FC1E
:108CC000131717002390B600131707019386E6FFCA
:108CD00013570701E39086FC1306000093860B00F0
:108CE0001307C10C83D50600835707009386E6FF60
:108CF0001307E7FFB387B700B387C70013D6070191
:108D00002391F60013761600E31E87FC13058109F4
:108D1000138609009305C107EFE05FDA0355C11A16
:108D20009384F4FFE30605E48327010083264100D2
:108D300013073000B337F000B307F04093F7D700C4
:108D4000938707022302F112832781006394E600D0
:108D5000B38797001307A0022320F1006354F700A4
:108D60002320E1001307A0006306E54E1305050369
:108D70001307E002A302A1122303E11263CC071E32
:108D8000130C711213040000130D410B930D4109D4
:108D9000930AE107930B610B1306000093850D0006
:108DA0006F00C001131616002390F500131606017C
:108DB0009385E5FF135606016384550583D70500A7
:108DC0001395070113550541939717006354050048
:108DD000136616009397070193D7070113752600B2
:108DE00093E81700E30005FC131616002390150105
:108DF000131606019385E5FF13560601E39055FD12
:108E000013060D009307C10783D50700938727003A
:108E100013062600231FB6FEE398B7FF2316010CA6
:108E2000130600009305C10C6F00C0011316160055
:108E30002390F500131606019385E5FF13560601EE
:108E40006384750583D70500139507011355054104
:108E50009397170063540500136616009397070154
:108E600093D707011375260093E81700E30005FC6C
:108E70001316160023901501131606019385E5FFBE
:108E800013560601E39075FD130600009305C10C0F
:108E90006F00C001131616002390F500131606018B
:108EA0009385E5FF135606016384750583D7050096
:108EB0001395070113550541939717006354050057
:108EC000136616009397070193D7070113752600C1
:108ED00093E81700E30005FC131616002390150114
:108EE000131606019385E5FF13560601E39075FD01
:108EF0001305000093850D001306C10C83D80500EF
:108F0000835706009385E5FF1306E6FFB387170135
:108F1000B387A70013D507012391F500137515003A
:108F2000E31E76FD138609009305C1071305810929
:108F3000EFE0DFB80356C11A0327010093071C00B6
:108F40009305060313041400A38FB7FE634A870238
:108F5000138C07006FF05FE413161601B7070100CA
:108F6000135616019387F7FF2317C1082320F1003A
:108F70006FF09F9D0356C11A130C61129307711273
:108F800013074000635AC70413075000E308E602C2
:108F900003C7E7FF032601009386E7FF1377F70770
:108FA000634606029307E00213068003930500035D
:108FB000630EF776635AE67803C7F6FF2380B600A0
:108FC0009386F6FF1377F7076FF09FFE13071003E2
:108FD000238FE7FE93841400B76501801386040095
:108FE0009385859713050C00EF2090128357210776
:108FF000032741012328911693C7F7FF2322E11687
:1090000013971701630607188326010103474112CE
:109010009387140023A0F60093870C00630A0702CD
:109020009306E0026302D72003C717009387170057
:10903000E31A07FE9306500463E6FC006F0040014C
:109040006388970103C7F7FF9387F7FFE31AD7FEFB
:109050002380070093870C00930600021306D002BA
:1090600003C707006304D7006316C7009387170080
:109070006FF01FFF13840C006F00C00003C70700D0
:10908000138406002300E40093061400938717005E
:10909000E31607FE83264100930720000347F4FFF1
:1090A000638EF610832781009386070063D49700B0
:1090B00093860400930700036316F702B3079441F5
:1090C00063D2F602130600036F00800063DCE60043
:1090D0008347E4FFA30F04FE1304F4FF3307944116
:1090E000E386C7FE03274100930730006304F70EB1
:1090F0008327C10023220A04138697009307700177
:1091000063F4C710130710009307400093971700EC
:10911000938647019305070013071700E378D6FEEF
:109120002322BA0413050A00EF1000472320AA04E3
:1091300093850C0093040500EF20101D0327810187
:1091400063080700B3079441B387F4002320F700B6
:109150008320C11E0324811E0329011E8329C11DF2
:10916000032A811D832A411D032B011D832BC11C52
:10917000032C811C832C411C032D011C832DC11B3E
:10918000138504008324411E1301011F6780000022
:10919000930709009306210703D707009387270049
:1091A000631A075AE39AD7FE03270101B727000085
:1091B0009387F7702320F7006FF0DFE99307000330
:1091C000E318F7F2B307944193061000E3CCF6EEF0
:1091D0006FF01FF283278100B384970063CA044EA7
:1091E000832701010327C10083A70700B307F70006
:1091F0002326F1008327C10023220A0413863700A7
:1092000093077001E3E0C7F0930500006FF09FF152
:10921000032CC100232481019307A00263D287EDB0
:109220002324F1006FF0CFEB03C70700E30407E04E
:1092300003C7170093871700A38FE7FEE30C07DE31
:1092400003C7170093871700A38FE7FEE31207FEFB
:109250006FF05FDE13071003A302E1121307E002B1
:109260002303E112938414006358F02A9307000348
:10927000A303F11283270100130C81129387F7FFD8
:109280002320F1006FF01FB0930C4112B7650180ED
:109290009385C59713850C00B7240000EF20406725
:1092A0009384F4706FF09FD4130D410B13070D00DE
:1092B0009307C1071306010983D607009387270088
:1092C00013072700231FD7FEE398C7FEB747000008
:1092D0009387E7082313F10C93070001232EF10075
:1092E000B78700009387F7FF2322F102B7C7FFFF7C
:1092F000938727009304000013038C0C930C4112F6
:10930000930901161304010D930AA10A2324F10203
:1093100013050300938609001306810993050D00C8
:1093200023206102EFE01FDB032301021307C104C6
:109330009307810983D60700938727001307270027
:10934000231FD7FEE398B7FF832741028355E1052A
:1093500033F6F500832781023305F6006354A03805
:10936000130600093306A640130704009307C1043F
:1093700083D607009387270013072700231FD7FEF4
:10938000E39827FF6356C0069307F0001307040015
:1093900063DEC70293060008B386A64093D6460054
:1093A00013871600131717003307E4009307040010
:1093B00093872700239F07FEE31CF7FE1306000890
:1093C0003306A640939646003306D6409317160000
:1093D000B307FC008356070083D70723B3F7F600D3
:1093E0002310F7009395050193D5054163C6051435
:1093F000930781091307040003D60700835607006B
:1094000093872700130727006316D602E396FAFE18
:1094100013070D009307810983D607009387270060
:1094200013072700231FD7FEE398B7FF8327C10147
:10943000B384F4000327C101130343019307CC1243
:1094400013571700232EE100E314F3EC8357610C4C
:109450000357E1081306810CB387E70037C7FFFF06
:10946000130727F7B387E7002313F10C1307C1078E
:1094700093070D0083D60700938727001307270063
:10948000231FD7FEE398C7FE130700009307810947
:109490006F00800003D70B0093872700239FE7FE10
:1094A000938B2B00E398B7FF930A8C02B71D000043
:1094B000130C8C116F00000193DD1D0063848A275B
:1094C000938A4A0193050D0013050C00EFE0CF8A43
:1094D0001307050093050D0013850A006344E0247B
:1094E000EFE08F89E34AA0FC9386090013060D0084
:1094F00093050D0013850A00EFE0DFBD1306810917
:10950000938609009305060013850A00EFE04FF1EA
:10951000B384B4016FF05FFA130C7112E39E07AAD3
:109520006FF05F86130600006FF0CFB98327C1008C
:10953000138CF7FF6FF01FCE9307C10413070400CD
:109540006F00C0009306E105E384F6EA03D6070046
:10955000835607009387270013072700E304D6FEEE
:109560008357210E03274102B377F7006386E73C58
:109570009305C10E13850B0023206102EFD09FF4E9
:109580009305811013050400EFD0DFF30357C10EDC
:109590000356A110035EE10E1347F7FF13170701EF
:1095A000135707012316E10EB305CE400323010232
:1095B00093060600635EB00693850C009306811047
:1095C0009307011203D50600938626009385250094
:1095D000239FA5FEE398F6FE231E01129306811039
:1095E0009305C10E6F00800003D705009386260007
:1095F000239FE6FE93852500E398F6FE23100112D3
:109600001307C10E93870C001305C11383D60700FF
:109610009387270013072700231FD7FEE398A7FE91
:109620008356A110B305C64123120110138606000C
:10963000638E05322326D1029307F0F663CEF5063A
:109640001305C10E23206102EFD0DFC50323010201
:109650008326C102930505009307011213074110E9
:109660000355C10E035681106306C534130E000066
:109670001305A11003D60700835E07009387E7FF59
:109680003306C6413306D641135E06012391C70057
:10969000137E1E001307E7FFE39EA7FC13061000CE
:1096A000938709001307000413058110232061022A
:1096B000EFE04F800323010293050400130581109E
:1096C00023206102EFD09F9A032301026FF05FD243
:1096D000832701012302011213840C0023A0070039
:1096E0006FF05FB1930704001307410E93872700C3
:1096F000239F07FEE39CE7FE6FF0DFCE8327010088
:10970000930C4112638E0708B76501809385C59558
:1097100013850C00B7240000EF20801F9384F470A1
:109720006FF0DF8C930A810E6FF00FBD83C7F6FFD9
:10973000130780036370F70E9307100393841400DC
:10974000A38FF6FE6FF05F89130717002380E600F2
:109750006FF09F88130721076F008000E306E98AF6
:109760008357090013092900E38A07FE0327010133
:10977000B72700009387F7702320F7006FF09F8DC5
:10978000930C4112B76501809385459713850C00B2
:10979000B7240000EF20C0179384F4706FF01F858A
:1097A000B76501809385859613850C00B72400006A
:1097B000EF2000169384F4706FF05F8393058109A6
:1097C0001305C107232EF100EFD05F8A93054B9854
:1097D00013058109EFD05FDA8327C101631A05FA07
:1097E00003270100634A07FE03C7E7FF930627FD2F
:1097F00093B6160093C6F6FFB306DC0083C60600D8
:1098000093F61600638A06FC9386E7FF1377F70743
:109810006FF04FF993871700A38FF6FE6FF0CFFB21
:109820001304010D930504001305C107374D000013
:10983000EFD05FC993040000930A810E9309C10C15
:10984000930C210D130DEDFF8357810E93F77700D5
:10985000639A070C1307410B9307040083D6070094
:109860009387270013072700231FD7FEE39857FF8E
:109870001305410B2316010CEFD04FE81305410BE4
:10988000EFD0CFE7130600009386090013870A0084
:1098900083D50600835707009386E6FF1307E7FF8B
:1098A000B387B700B387C70013D607012391F6002B
:1098B00013761600E31E97FD8357610B0357810B48
:1098C00093873700231BF10A630007021305410B3E
:1098D000EFD0CFE28357610B0357810B93871700BB
:1098E000231BF10AE31407FE8357C10C639C070294
:1098F0008357610B6368FD02130704009307410B54
:1099000083D607009387270013072700231FD7FE5E
:10991000E39837FF2314010E9384F4FF930750FD5F
:10992000E394F4F29305C10713050400EFD00FF49C
:10993000930901166FF08F8B9307040003D707007C
:1099400093872700E31607AA1307210EE398E7FE83
:109950009307040003D7070093872700E31A07C083
:109960001307210EE398E7FE6FF09FA81307C110BD
:109970009307010F03DE07000355070093872700B5
:10998000130727006314AE0613056110E394A7FEC6
:109990000357C10E835781106302F7069307040033
:1099A0001307410E93872700239F07FEE39CE7FEE2
:1099B0006FF01FA413050000130EE10E83DE0700F5
:1099C000035607009387E7FF1307E7FF3306D60127
:1099D0003306A600135506012391C7001375150021
:1099E000E31EC7FD130600006FF09FCB6360C50543
:1099F00093070112130741106FF09FC6938706006B
:109A0000639606000317E110635A07081307A110B5
:109A1000930701128355070013072700639C050C69
:109A2000E39AE7FE2315C1106FF01FC913860C00DF
:109A3000130781109307011203550700130727002E
:109A400013062600231FA6FEE318F7FE231E0112AD
:109A5000130581101306C10E13074110035E0600A3
:109A60001306260013052500231FC5FFE318E6FE95
:109A700023100112130EC10E13860C001305C1131F
:109A8000835E060013062600130E2E00231FDEFF42
:109A9000E318A6FE231201106FF09FBC930601127B
:109AA0001305A1106F00C0012390E60093971700E3
:109AB000939707019386E6FF93D70701E38EA6BE2F
:109AC00003D7060013160701135606411317170094
:109AD0006354060093E71700131707011357070194
:109AE00013F6270093651700E30006FC2390B600E9
:109AF0006FF0DFFB138616002315C1106FF0DFBB7C
:109B0000032785008327C50003260500832645001B
:109B1000130101FC13050100930541012324E10019
:109B20002326F100232E11022320C1002322D1007D
:109B3000EFE01FB4835761021305000093C7F7FFDE
:109B400013971701631007029307410193066102FF
:109B500003D7070093872700631C0700E39AD7FE0B
:109B6000130520008320C103130101046780000056
:109B7000130510006FF01FFF1305050F678000002D
:109B80003775018013058567678000003775018090
:109B90001305856767800000130101FF232611006C
:109BA0002324810023229100630C0602B765018003
:109BB0009385C5BD1305060013040600EF10105D64
:109BC000B764018063120502138584BD8320C10040
:109BD00003248100832441001301010167800000F8
:109BE000B76401806FF05FFE938584BD13050400A8
:109BF000EF10D059E30A05FCB75501809385054560
:109C000013050400EF109058E30005FC1305000055
:109C10006FF0DFFBB777018003C5076B678000003B
:109C2000130101FF23261100232481002322910028
:109C3000638C050213840500B76501809385C5BD5B
:109C400013050400EF109054B764018063120502FD
:109C5000138584BD8320C100032481008324410037
:109C60001301010167800000B76401806FF05FFE9F
:109C7000938584BD13050400EF105051E30A05FCE1
:109C8000B75501809385054513050400EF1010506A
:109C9000E30005FC130500006FF0DFFB130101FD7D
:109CA000232E310123261102232481022322910233
:109CB00023202103232C4101232A51012328610160
:109CC0002326710123248101232291019387B5006A
:109CD00013076001930905006366F7069307000107
:109CE00063E6B71EEF00D00A9304000193078001DA
:109CF00013062000377901801309496FB307F90073
:109D000003A44700138787FF630AE42083274400E6
:109D10008326C4000326840093F7C7FFB307F4002B
:109D200003A747002326D60023A4C6001367170005
:109D30001385090023A2E700EF00D0051305840076
:109D40006F00801993F487FF63C2071863E0B418AB
:109D5000EF0010049307701F63F6974693D79400A3
:109D60006386071A13074000636CF73C93D76400BF
:109D7000138697031385870393163600377901807E
:109D80001309496FB306D90003A44600938686FFE2
:109D9000638686029305F0006F000001635C073262
:109DA0000324C400638C86008327440093F7C7FF15
:109DB00033879740E3D4E5FE130605000324090129
:109DC0009308890063081417032544009306F000E4
:109DD0001375C5FFB307954063CCF640232A1901DC
:109DE0002328190163D6073E9307F01F63EAA72EC5
:109DF000937785FF9387870083254900B307F90090
:109E000083A6070013555500130710003317A7004A
:109E10003367B700938587FF2326B4002324D4003B
:109E20002322E90023A0870023A68600935726401B
:109E300093051000B395F5006368B710B3F7E5001C
:109E400063940702939515001376C6FFB3F7E500F8
:109E500013064600639A070093951500B3F7E500D3
:109E600013064600E38A07FE1308F00013133600BA
:109E700033036900130503008327C500130E060092
:109E80006302F52E03A747001384070083A7C700CA
:109E90001377C7FFB30697406342D82EE3C206FE8E
:109EA0003307E40083264700032684001385090056
:109EB00093E616002322D7002326F60023A4C7002A
:109EC000EF00406D130584006F0000019307C00090
:109ED00023A0F900130500008320C102032481029E
:109EE00083244102032901028329C101032A81013C
:109EF000832A4101032B0101832BC100032C810024
:109F0000832C4100130101036780000093060020A9
:109F1000130600041305F0036FF05FE603A4C70007
:109F200013062600E39487DE0324090193088900C1
:109F3000E31C14E9032749009357264093051000BA
:109F4000B395F500E37CB7EE03248900832A44002F
:109F500013FBCAFF63689B00B3079B401307F00025
:109F60006346F714B7870180B78C018083AAC7B313
:109F700003A78CB29307F0FF330A6401B38A54013C
:109F8000630AF734B71700009387F700B38AFA0023
:109F9000B7F7FFFFB3FAFA0093850A0013850900AB
:109FA000EF10807F9307F0FF930B0500630CF528FB
:109FB00063684529378C0180130C8CB483250C0011
:109FC000B385BA002320BC00938705006304AA3A36
:109FD00083A68CB21307F0FF638CE63A338A4B41B9
:109FE000B307FA002320FC0093FC7B0063860C304F
:109FF000B7170000B38B9B4193858700938B8B0031
:10A00000B3859541B38A5B019387F7FFB3855541CB
:10A0100033FAF50093050A0013850900EF10C077A5
:10A020009307F0FF6300F53C33057541B30A450122
:10A0300083250C002324790193EA1A00B305BA00A2
:10A040002320BC0023A25B01630824359306F000A3
:10A0500063F866350327440093074BFF93F787FFA8
:10A06000137717003367F7002322E400130650002C
:10A070003307F4002322C7002324C70063EEF6361B
:10A0800083AA4B0013840B00B787018003A787B313
:10A090006374B70023ACB7B2B787018003A747B397
:10A0A0006376B71A23AAB7B26F00401A13E71400F9
:10A0B0002322E400B30494002324990093E71700BB
:10A0C0001385090023A2F400EF00C04C130584009F
:10A0D0006FF09FE08326C400032684006FF01FC446
:10A0E00093579500130740006372F714130740015C
:10A0F000636AF7229386C7059385B7059396360062
:10A10000B306D90083A70600938686FF6388F61CF2
:10A1100003A747001377C7FF6376E50083A787008F
:10A12000E398F6FE83A6C700032749002326D40040
:10A130002324F40023A4860023A687006FF01FCFFA
:10A14000130740016376F71213074005636AF71E91
:10A1500093D7C4001386F7061385E70693163600D7
:10A160006FF0DFC1130E1E0093773E0013058500CC
:10A17000638E07108327C5006FF09FD003268400ED
:10A1800093E514002322B4002326F60023A4C7007D
:10A19000B3049400232A99002328990093E716001A
:10A1A00023A6140123A4140123A2F4003307E4001E
:10A1B000138509002320D700EF00C03D130584005C
:10A1C0006FF09FD113D63400938784006FF09FB255
:10A1D0003307A400832747001385090093E717007E
:10A1E0002322F700EF00003B130584006FF0DFCE61
:10A1F00013E714002322E400B3049400232A9900F7
:10A200002328990013E7170023A6140123A414019F
:10A2100023A2E4003305A4002320F50013850900E0
:10A22000EF004037130584006FF01FCB9357650094
:10A230009386970393858703939636006FF05FECC0
:10A24000630E241103248900832A440093FACAFF71
:10A25000B3879A4063E69A001307F000E348F7E4F7
:10A2600013850900EF000033130500006FF0DFC60F
:10A270001386C7051385B705931636006FF01FB018
:10A28000832783001306F6FF6392671C93773600DB
:10A29000130383FFE39607FE0327490093C7F5FFE7
:10A2A000B3F7E7002322F90093951500E3EEB7C852
:10A2B000E38C05C833F7F500631A07009395150082
:10A2C00033F7F500130E4E00E30A07FE13060E00E7
:10A2D0006FF0DFB9938A0A016FF01FCC03254900A4
:10A2E00093D52540130710003317B7003367A70035
:10A2F0002322E9006FF09FE3B3855B01B305B04013
:10A300009395450113DA450193050A001385090069
:10A31000EF1080489307F0FFE318F5D0130A000010
:10A320006FF01FD1130740056362F7089357C5000C
:10A330009386F7069385E706939636006FF05FDC09
:10A34000130740156362F70893D7F4001386870755
:10A3500013857707931636006FF05FA2378C018064
:10A36000130C8CB483270C00B387FA002320FC0065
:10A370006FF01FC613174A01E31C07C403248900AA
:10A38000B30A5B0193EA1A00232254016FF0DFCF76
:10A3900023A47CB36FF05FC513840B006FF0DFCE96
:10A3A0009307100023A2FB006FF09FEB13074015EB
:10A3B0006362F7069357F5009386870793857707BF
:10A3C000939636006FF0DFD3130740556362F706AC
:10A3D00093D724011386D7071385C7079316360032
:10A3E0006FF0DF99938C8CFFB38A9A01B38A7A411C
:10A3F000130A00006FF0DFC3930584001385090082
:10A40000EFC08FFE0324890083250C00832A4400BB
:10A410006FF09FC7130740556364F70293572501F8
:10A420009386D7079385C707939636006FF05FCD65
:10A430009306803F1306F0071305E0076FF01F94A3
:10A440009306803F9305E0076FF09FCB8327490079
:10A450006FF09FE5B777018083A7C7666780070025
:10A4600063800502630206046388060483470600CE
:10A4700023A0F500034506003335A00067800000E7
:10A48000130101FF9305C10063040602638A0602FB
:10A490008347060023A0F500034506003335A000DE
:10A4A00013010101678000001305000067800000B0
:10A4B000130500006FF0DFFE1305E0FF678000006A
:10A4C0001305E0FF6FF0DFFD9377350093F6F50F8E
:10A4D000638A07029307F6FF630E06021306F0FF76
:10A4E0006F0080011305150013773500630E070018
:10A4F0009387F7FF6380C70203470500E314D7FE85
:10A500006780000093070600130730006366F702B8
:10A51000639607001305000067800000B307F5008D
:10A520006F00C00013051500E386A7FE0347050072
:10A53000E31AD7FE6780000093F5F50F9398850026
:10A54000B3E5B80093980501B3E8B8003708FFFEFB
:10A55000B78580801308F8EF938505081303300052
:10A560000327050033C7E800330607011347F7FF49
:10A570003377E6003377B700E31207FA9387C7FF14
:10A5800013054500E36EF3FCE39A07F86FF09FF8BC
:10A5900067800000678000008327C504130101FF66
:10A5A000232481002322910023261100232021014E
:10A5B0001304050093840500638E0702139524009D
:10A5C000B387A70003A5070063060504032705005A
:10A5D00023A0E70023280500232605008320C100CF
:10A5E0000324810083244100032901001301010198
:10A5F000678000001306100293054000EF2010133F
:10A600002326A40493070500E31A05FA13050000A6
:10A610006FF0DFFC1309100033199900130659007D
:10A62000131626009305100013050400EF201010E8
:10A63000E30E05FC23229500232425016FF09FF9EA
:10A640006380050203A745008327C504131727006D
:10A65000B387E70003A7070023A0E50023A0B70006
:10A6600067800000130101FE232A910083A40501E5
:10A6700037030100232C81002328210123263101E7
:10A68000232E11002324410113890500930905009D
:10A690001384060013884501930800001303F3FF99
:10A6A000832708001308480093881800B3F6670052
:10A6B000B386C60293D70701B387C702B386860065
:10A6C00013DE060133F76600B386C70193970601D0
:10A6D0003387E700232EE8FE13D40601E3C298FC7B
:10A6E000630204028327890063D0F4049387440043
:10A6F00093972700B307F90023A2870093841400DF
:10A70000232899008320C10103248101832441016E
:10A710008329C100032A81001305090003290101CF
:10A720001301010267800000832549001385090099
:10A7300093851500EFF05FE6130A0500630C05042E
:10A74000032609019305C9001305C5001306260059
:10A7500013162600EF2010110327490083A7C90410
:10A7600013172700B387E70003A707002320E9009A
:10A7700023A027019387440013090A009397270019
:10A78000B307F90023A287009384140023289900BB
:10A790006FF05FF7B766018037650180938686BEEC
:10A7A000130600009305500B1305C5BFEF20407141
:10A7B000130101FE232C8100232A9100232821016B
:10A7C0002326310123244101938906009307900039
:10A7D00093868600232E110023225101B3C6F60270
:10A7E0001309050013840500130A060093040700EB
:10A7F00063D8370D93071000930500009397170057
:10A8000093851500E3CCD7FE13050900EFF0DFD8E0
:10A8100093050500630A050A930710002328F50035
:10A82000232A95009307900063D64709930A940062
:10A8300093840A003304440183C604001306A00075
:10A8400013050900938606FDEFF0DFE19384140001
:10A8500093050500E39284FE13048AFF33848A0083
:10A8600063563A03B3894941B3093401834604006E
:10A870001306A00013050900938606FDEFF09FDE86
:10A880001304140093050500E39289FE8320C1019F
:10A890000324810183244101032901018329C1008B
:10A8A000032A8100832A4100138505001301010258
:10A8B000678000001304A400130A90006FF05FFA91
:10A8C000930500006FF05FF4B76601803765018083
:10A8D000938686BE130600009305E00C1305C5BFE2
:10A8E000EF20005E3707FFFF3377E5009307050091
:10A8F0001305000063160700939707011305000175
:10A90000370700FF33F7E7006316070013058500DC
:10A9100093978700370700F033F7E70063160700C7
:10A920001305450093974700370700C033F7E7004A
:10A9300063160700130525009397270063CA0700D5
:10A9400037070040B3F7E7001305150063840700DD
:10A950006780000013050002678000008327050060
:10A960001307050093F677006384060293F6170039
:10A9700013050000639E060493F627006388060A09
:10A9800093D717002320F7001305100067800000FD
:10A990009396070193D6060113050000638E060601
:10A9A00093F6F70F6380060693F6F70063820604BA
:10A9B00093F637006384060293F61700639C060043
:10A9C00093D71700130515006396070013050002BF
:10A9D000678000002320F7006780000093D72700DE
:10A9E00093F6170013052500E39606FE6FF05FFD52
:10A9F00093D7470093F6370013054500E39E06FA08
:10AA00006FF0DFFD93D7870093F6F70013058500FD
:10AA1000E39006FA6FF0DFFD93D7070193F6F70F87
:10AA200013050001E39206F86FF0DFFD93D72700CE
:10AA30002320F70013052000678000008327C5044A
:10AA4000130101FF232481002322910023261100FA
:10AA50001304050093840500638C070203A54700D7
:10AA6000630205060327050023A2E7008320C10037
:10AA70000324810093071000232A95002326050054
:10AA80002328F500832441001301010167800000A1
:10AA90001306100293054000EF2040492326A4042A
:10AAA00093070500E31C05FAB7660180376501804E
:10AAB000938686BE13060000930500141305C5BFD8
:10AAC000EF2000401306C001930510001305040099
:10AAD000EF20C045E30A05FC930710002322F50090
:10AAE000930720002324F5006FF05FF8130101FEA7
:10AAF000232821012326310103A905018329060109
:10AB0000232A910023244101232E1100232C8100AC
:10AB1000138A050093040600634C3901138709006A
:10AB20009384050093090900130A0600130907001E
:10AB300083A7840083A5440033842901B3A7870039
:10AB4000B385F500EFF05FA5630E051A1303450109
:10AB500093182400B30813019307030063781301CB
:10AB600023A0070093874700E3EC17FF13084A016F
:10AB7000131E2900938E440193952900330EC801BA
:10AB8000B385BE006376C81393875401130F40004A
:10AB900063F0F516370601001306F6FF6F0080011B
:10ABA00093DF0F0163980F08130848001303430055
:10ABB0006370C811832F0800B3F4CF00E38204FE52
:10ABC0009303030093820E001309000003A7020001
:10ABD00083AF030093834300B376C700B386960226
:10ABE0009357070133F7CF0093DF0F0193824200A1
:10ABF000B3879702B386E600B386260113D7060112
:10AC0000B3F6C600B387F701B387E70013970701D0
:10AC1000B366D70023AED3FE13D90701E3E8B2FA37
:10AC2000B307E30123A02701832F080093DF0F015F
:10AC3000E38C0FF6032703009302030093860E00B4
:10AC4000930407009303000083A7060093D904012F
:10AC50003377C700B3F7C700B387F70383A4420075
:10AC6000938242009386460033F9C400B3873701CC
:10AC7000B38777009393070133E7E30023AEE2FE47
:10AC800003D7E6FF93D707013307F70333072701FD
:10AC90003307F70093530701E3E8B6FAB307E3017C
:10ACA00023A0E7001308480013034300E364C8F13E
:10ACB000634880006F0080011304F4FF6308040000
:10ACC00083A7C8FF9388C8FFE38807FE8320C101DC
:10ACD00023288500032481018324410103290101E4
:10ACE0008329C100032A810013010102678000004B
:10ACF000338F9540130FBFFE137FCFFF130F4F000D
:10AD00006FF05FE9B766018037650180938686BE84
:10AD1000130600009305D0151305C5BFEF20401A98
:10AD2000130101FE232C8100232821012326310158
:10AD3000232E1100232A9100937736001304060076
:10AD40009309050013890500639E070A13542440E4
:10AD50006306040683A48904638A040C93771400B1
:10AD60006390070213541440630A040403A504000B
:10AD7000630605069304050093771400E38407FE39
:10AD8000138604009305090013850900EFF01FD610
:10AD9000630609060327490083A7C9041354144016
:10ADA00013172700B387E70003A707002320E90054
:10ADB00023A0270113090500E31A04FA8320C10127
:10ADC00003248101832441018329C1001305090063
:10ADD00003290101130101026780000013860400AA
:10ADE0009385040013850900EFF05FD023A0A40031
:10ADF00023200500930405006FF01FF813090500D8
:10AE00006FF05FF69387F7FF37670180130787C5F9
:10AE100093972700B307F70003A6070093060000E7
:10AE2000EFF05F84130905006FF05FF293051000E7
:10AE300013850900EFF04FF6930405006300050247
:10AE400093071027232AF500930710002328F50005
:10AE500023A4A904232005006FF05FF0B7660180EA
:10AE600037650180938686BE1306000093050014A3
:10AE70001305C5BFEF20C004130101FE23244101C7
:10AE800003AA050183A78500232631019359564063
:10AE9000338A4901232C8100232A91002328210190
:10AEA00023225101232E110013091A009384050057
:10AEB0001304060083A54500930A050063D8270103
:10AEC0009397170093851500E3CC27FF13850A009D
:10AED000EFF08FEC630C0510130845016354300349
:10AEE0009389590093992900330735019307080086
:10AEF0009387470023AE07FEE39CE7FE9389C9FED4
:10AF00003308380103A60401938744011373F40145
:10AF1000131626003386C7006304030A9305000254
:10AF2000B3856540930808009306000003A7070057
:10AF30009388480093874700331767003367D7002B
:10AF400023AEE8FE03A7C7FFB356B700E3E0C7FE92
:10AF50001387540193074000636AE600B3079640E5
:10AF60009387B7FE93F7C7FF938747003308F8002E
:10AF70002320D80063840600130A090003A74400B5
:10AF800083A7CA048320C10113172700B387E700F2
:10AF900003A70700232845010324810123A0E4001F
:10AFA00023A0970003290101832441018329C100C3
:10AFB000032A8100832A41001301010267800000F7
:10AFC00003A707009387470013084800232EE8FED5
:10AFD000E3F6C7FA03A70700938747001308480062
:10AFE000232EE8FEE3EEC7FC6FF05FF9B766018041
:10AFF00037650180938686BE130600009305901D79
:10B000001305C5BFEF10D06B0327050183A705010A
:10B01000130805003305F7406312F70493972700E0
:10B0200013084801938545013307F800B387F500FD
:10B030006F0080006374E8028326C7FF03A6C7FF82
:10B040001307C7FF9387C7FFE386C6FEB3B6C600E4
:10B050003305D0401365150067800000678000004D
:10B0600083A7050103270601130101FF23248100A3
:10B07000232291002320210123261100938405001F
:10B08000130406003389E7406394E71A93162700F8
:10B090009385450113074601B387D5003307D700D1
:10B0A0006F00800063FCF51803A6C7FF8326C7FF67
:10B0B0009387C7FF1307C7FFE306D6FE6360D61664
:10B0C00083A54400EFF04FCD6302051A03AE0401DF
:10B0D0008322040193844401931E2E00130844012B
:10B0E00093922200930F4501B70801002326250102
:10B0F000B38ED401B3025800138F0F0013830400E2
:10B10000930700009388F8FF0327030083250800B6
:10B11000130F4F00B3761701B386F600B3F715018E
:10B12000B386F64093D5050193570701B387B7401F
:10B1300013D70641B387E70013970701B3F616014B
:10B14000B366D70013084800232EDFFE1303430025
:10B1500093D70741E36A58FAB38582409385B5FED9
:10B160001304540193D525001307000063E4820003
:10B17000139725003387EF001308400063E6820031
:10B180009385150013982500B3840401B38F0F0134
:10B1900063FED405B708010013880F0093850400EF
:10B1A0009388F8FF03A7050013084800938545001E
:10B1B000337617013306F60093560641935707017D
:10B1C000B387D7009396070133761601B3E6C6001E
:10B1D000232ED8FE93D70741E3E6D5FD1387FEFF64
:10B1E000330797401377C7FF3387EF00639A060052
:10B1F0008327C7FF130EFEFF1307C7FFE38A07FE6F
:10B200008320C100032481002328C5018324410039
:10B2100003290100130101016780000093870400E6
:10B220001309100093040400138407006FF05FE912
:10B23000E34609FE130900006FF09FE89305000044
:10B24000EFF08FB5630205048320C1000324810061
:10B25000930710002328F500232A050083244100CA
:10B26000032901001301010167800000B766018016
:10B2700037650180938686BE13060000930500247F
:10B280001305C5BFEF10D043B76601803765018055
:10B29000938686BE13060000930520231305C5BFC1
:10B2A000EF101042B707F07FB3F5B700B707C0FC47
:10B2B000B385F5006358B0009307000013850700BD
:10B2C00067800000B305B04093D545419307300136
:10B2D00063C8B700B7070800B3D5B7406FF0DFFD0C
:10B2E0001387C5FE9306E001930500009307100045
:10B2F000E3C6E6FCB7070080B3D7E7001385070075
:10B3000067800000130101FE232A910083240501B8
:10B31000232C81001304450193942400B30494006A
:10B320002328210103A9C4FF23263101232441013D
:10B330001305090093890500232E1100EFF08FDA21
:10B3400013070002B307A74023A0F9009307A0004A
:10B35000138AC4FF63D0A708130555FF6370440523
:10B3600083A784FF63000504B306A74033D7D70043
:10B370003319A9003369E900138684FF3707F03FCA
:10B380003367E900B397A7006372C40203A644FFC2
:10B39000B356D600B3E7D7006F0040019307000013
:10B3A000631405063707F03F3367E9008320C101C6
:10B3B0000324810183244101032901018329C10060
:10B3C000032A81001385070093050700130101027A
:10B3D000678000009306B000B386A640B707F03F31
:10B3E0003357D9003367F7009307000063764401B1
:10B3F00083A784FFB3D7D700130555013315A900E0
:10B40000B367F5006FF09FFA3315A9003707F03FD7
:10B410003367E500930700006FF05FF9130101FD4A
:10B42000232A5101938A050093051000232021034C
:10B43000232E3101232C41012326110223248102D2
:10B440002322910213090600138A060093090700BC
:10B45000EFF08F9463080510B7071000935449016B
:10B460001386F7FF93F4F47F130405003376260167
:10B47000638404003366F6002326C10063880A084B
:10B480001305810023245101EFF04FCD0327C100A4
:10B49000930705006302050C032681009306000252
:10B4A000B386A640B316D700B3E6C6003357A7004D
:10B4B000232AD4002326E1003339E00013091900C0
:10B4C000232CE40023282401638404069384D4BC41
:10B4D000B384F4001305500323209A00B307F5400A
:10B4E00023A0F9008320C102130504000324810274
:10B4F00083244102032901028329C101032A810116
:10B50000832A410113010103678000001305C10074
:10B51000EFF0CFC4930710002328F4008327C10065
:10B5200013091000232AF40093070502E39004FA9C
:10B53000131729003307E400032507019387E7BCAD
:10B540002320FA00EFF00FBA131959003309A9406C
:10B5500023A029016FF01FF983268100232AD4003C
:10B560006FF09FF5B766018037650180938686BED0
:10B57000130600009305A0301305C5BFEF1050144B
:10B58000130101FD23202103138905009305810088
:10B59000232611022324810223229102232E31012A
:10B5A00093090500EFF01FD69304050013840500EE
:10B5B000130509009305C100EFF0DFD4032709014B
:10B5C00083A709018326C100B387E74003278100D1
:10B5D000939757003307D740B387E7001307050059
:10B5E000635EF002939747013384870093860500DA
:10B5F000138504009305040013060700EF608F8D88
:10B600008320C10203248102832441020329010211
:10B610008329C1011301010367800000939747014B
:10B62000B385F5406FF09FFC130101FF232021013A
:10B630002326110023248100232291009307700107
:10B640001309050063DAA70437870180832787B0D1
:10B650008325C7B037870180032407B1832447B10E
:10B66000138507001306040093860400EF601FA1F2
:10B670001309F9FF93070500E31409FE8320C100B5
:10B68000032481008324410003290100138507005E
:10B690001301010167800000B767018013193500AD
:10B6A000938787C533892701832709018320C10038
:10B6B00003248100832549018324410003290100DB
:10B6C000138507001301010167800000832606012E
:10B6D0009385F5FF93D55540938515009307460153
:10B6E0009396260093952500B386D700B305B50041
:10B6F00063F8D7021307050003A8070093874700E4
:10B7000013074700232E07FFE3E8D7FEB387C640A1
:10B710009387B7FE93F7C7FF938747003305F5007C
:10B720006378B50013054500232E05FEE36CB5FED6
:10B73000678000000327050113D655409306450195
:10B740006352C70293172700B387F60063F2F6042B
:10B7500003A7C7FF9387C7FFE30A07FE130510007F
:10B760006780000093172600B387F600E350E6FEDB
:10B7700093F5F501E38C05FC03A607001305100003
:10B780003357B600B315B700E302B6FC678000007C
:10B790001305000067800000130101FF23248100CE
:10B7A0002322910013040500B7840180138505004E
:10B7B0002326110023A004B4EF50806D9307F0FFFF
:10B7C000630CF5008320C100032481008324410021
:10B7D000130101016780000083A704B4E38407FE1E
:10B7E0008320C1002320F40003248100832441002E
:10B7F0001301010167800000130101FF2322910062
:10B80000B7040080232481002326110093C4F4FF91
:10B810001304060023200600B3F6B4003706F07FB9
:10B82000938705001307050063D0C606B3E8A6009A
:10B83000638C080433F6C5001388050093080000E4
:10B8400063120602B787018083A6C7B103A687B13A
:10B85000EF60DF821307050013880500B3F6B4001C
:10B860009308A0FC93D64641B70710809387F7FF53
:10B87000938626C03378F800B3861601B707E03FF9
:10B88000B367F8002320D4008320C1000324810083
:10B89000832441001305070093850700130101016C
:10B8A00067800000130101F6930EC108232AF108F6
:10B8B00037030080B707FFFF138E05001343F3FF24
:10B8C0002326D108938787209305810093860E0055
:10B8D000232E1106232AF1002328E108232C010935
:10B8E000232E11092324C101232CC101232E610021
:10B8F000232861002322D101EF800FFC83278100E0
:10B90000238007008320C1071301010A678000001C
:10B91000130E050037850180130101F6032545B29A
:10B92000930E8108232AF10837030080B707FFFF31
:10B930001343F3FF2324C1082326D10893878720CC
:10B940001386050093860E0093058100232E1106B1
:10B95000232AF1002328E108232C0109232E1109B1
:10B960002324C101232CC101232E6100232861005F
:10B970002322D101EF804FF4832781002380070029
:10B980008320C1071301010A678000003367B500F7
:10B990009303F0FF1377370063100710B7877F7F9B
:10B9A0009387F7F70326050083A60500B372F60018
:10B9B0003363F600B382F200B3E262006392721066
:10B9C0006316D6080326450083A64500B372F60029
:10B9D0003363F600B382F200B3E26200639E720C3E
:10B9E0006316D6060326850083A68500B372F6008B
:10B9F0003363F600B382F200B3E262006398720C24
:10BA00006316D6040326C50083A6C500B372F600EC
:10BA10003363F600B382F200B3E262006392720C09
:10BA20006316D6020326050183A60501B372F6004C
:10BA30003363F600B382F200B3E26200639C720AE1
:10BA40001305450193854501E30ED6F4131706014E
:10BA500093970601631EF7001357060193D706015B
:10BA60003305F7409375F50F63900502678000007A
:10BA70001357070193D707013305F7409375F50F67
:10BA800063940500678000001377F70F93F7F70FB3
:10BA90003305F740678000000346050083C60500B4
:10BAA00013051500938515006314D600E31606FEF2
:10BAB0003305D64067800000130545009385450097
:10BAC000E31CD6FC13050000678000001305850009
:10BAD00093858500E312D6FC130500006780000003
:10BAE0001305C5009385C500E318D6FA13050000B9
:10BAF000678000001305050193850501E31ED6F854
:10BB00001305000067800000B367B50093F73700A6
:10BB10006392070803A70500B7867F7F9386F6F731
:10BB2000B377D700B387D700B3E7E700B3E7D70011
:10BB30001306F0FF639EC706130605001308F0FF07
:10BB40002320E60003A74500938545001306460021
:10BB5000B377D700B387D700B3E7E700B3E7D700E1
:10BB6000E38007FF83C7050003C7150083C62500D0
:10BB70002300F600638A0700A300E60063060700BF
:10BB80002301D6006394060067800000A30106002D
:10BB9000678000009307050003C70500938717001F
:10BBA00093851500A38FE7FEE31807FE678000006A
:10BBB000130605006FF01FFB937735001307050090
:10BBC000639C0704B7867F7F9386F6F79305F0FFA3
:10BBD0000326070013074700B377D600B387D700C3
:10BBE000B3E7C700B3E7D700E384B7FE8346C7FFD8
:10BBF0000346D7FF8347E7FF3307A7406380060468
:10BC0000630A06023335F0003305E5001305E5FF4E
:10BC100067800000E38806FA8347070013071700D0
:10BC200093763700E39807FE3307A7401305F7FF25
:10BC3000678000001305D7FF678000001305C7FF6A
:10BC400067800000B3E7A50093F7370013070500EE
:10BC5000639807069307300063F4C7063703FFFEB7
:10BC6000B78880801303F3EF93880808130E300021
:10BC700083A60500B387660013C8F6FFB3F7070174
:10BC8000B3F71701639E07022320D7001306C6FFF0
:10BC90001307470093854500E36CCEFC93851500A0
:10BCA000930717006304060283C6F5FF1308F6FF27
:10BCB000A38FD7FE638E06001387070013060800C4
:10BCC0009385150093071700E31006FE67800000B8
:10BCD0003306C700630A080093871700A38F07FE87
:10BCE000E39CC7FE67800000678000008327860012
:10BCF000130101FD232A510123261102232481026D
:10BD00002322910223202103232E3101232C4101E0
:10BD1000232861012326710123248101930A06004F
:10BD200063880714130B05008329060003A505008B
:10BD300083A48500138405006F00400D8357C40061
:10BD400013F70748630A0708832644018325040183
:10BD50001307190093941600B386D40093D4F60108
:10BD6000330AB540B384D40093D414403307470159
:10BD70001386040063F6E40093040700130607002B
:10BD800093F707406386070A9305060013050B0027
:10BD9000EFD0DFF0130C0500630A050A83250401C8
:10BDA00013060A00EF10002C8357C40093F7F7B76F
:10BDB00093E707082316F40033054C01338A444106
:10BDC000232A940023244401232884012320A4004F
:10BDD00093040900130A090013060A0093850B0057
:10BDE000EF10003A032784000325040083A78A008C
:10BDF000B304974033054501232494002320A40075
:10BE00003389274123A42A016304090603A94900B1
:10BE100083AB0900138A040093898900E30809FEB3
:10BE2000E37E99F093040900130A09006FF0DFFA2A
:10BE300013050B00EF10C046130C0500E31E05F6BA
:10BE40008325040113050B00EFA01FDA9307C00040
:10BE50002320FB008357C4001305F0FF93E707047A
:10BE60002316F40023A40A0023A20A006F00C000D6
:10BE700023A20A00130500008320C10203248102CB
:10BE800083244102032901028329C101032A81017C
:10BE9000832A4101032B0101832BC100032C810064
:10BEA000130101036780000083D7C500130101ED72
:10BEB000232C411123286111232EB10F23261112A7
:10BEC000232481122322911223202113232E3111A6
:10BED000232A511123267111232481112322911128
:10BEE0002320A11193F707082326D100138A050008
:10BEF000130B0500930D06006386070083A7050159
:10BF0000E3800756B7670180930AC104938707D877
:10BF1000376C0180B764018023205105232401047C
:10BF20002322010413870A0023280100232201028F
:10BF3000232401022326010223240100232AF100E5
:10BF4000130CCCEE9384C4EF83C70D0063800720ED
:10BF500013840D00930650026386D738834714007C
:10BF600013041400E39A07FE3309B4416300B41FBD
:10BF700083268104832741042320B701B386260149
:10BF800093871700232227012324D1042322F104BD
:10BF9000930670001307870063CEF6348326810072
:10BFA00083470400B38626012324D1006380071A47
:10BFB00083461400930D1400A30D0102930CF0FFAF
:10BFC00013040000130D00001309A005930B90004B
:10BFD0009309A002938D1D00938706FE6364F90404
:10BFE0000326410193972700B387C70083A7070063
:10BFF0006780070013040000938706FD83C60D00C9
:10C0000093152400338485001314140033848700AF
:10C01000938706FD938D1D00E3F2FBFE938706FEDA
:10C02000E370F9FC638406122306D108A30D010214
:10C0300013091000930B10009309C108930C000022
:10C04000137F2D0063040F0013092900137E4D0890
:10C05000832781040326410463160E00B30624419E
:10C06000E348D0028346B103130516009305870009
:10C07000638006049306B103938717002320D7003B
:10C08000930610002322D7002324F1042322A104C5
:10C0900093067000E3CCA60C930F260093060701CD
:10C0A000130605001387050013850F00938506000E
:10C0B000630C0F029306C1032320D7009387270048
:10C0C000930620002322D7002324F1042322A10475
:10C0D00013077000E34AA70C130605001387050039
:10C0E0001305150093858500930600086300DE6044
:10C0F000B38C7C416344906BB387FB0023203701F2
:10C10000232277012324F1042322A10413077000C2
:10C110006340A77493784D0063860800B30B2441F5
:10C120006348701F6354240113040900032781002E
:10C13000330787002324E100639C077283C70D0047
:10C140002322010413870A00E39407E08327810474
:10C15000E39C074A8357CA0093F70704E392074E0C
:10C160008320C112032481120325810083244112FC
:10C17000032901128329C111032A8111832A411144
:10C18000032B0111832BC110032C8110832C411030
:10C19000032D0110832DC10F1301011367800000CF
:10C1A00013050B00232CE100EFD09F9D8327450052
:10C1B000138507002326F102EFF01FA09307050067
:10C1C00013050B002324F102EFD09F9B032785006A
:10C1D000832781022322E10203278101E3960716C8
:10C1E00083C60D006FF01FDF83C60D00136D0D02B7
:10C1F0006FF05FDE136D0D0193770D026382071EF2
:10C200008327C1009389770093F989FF83A64900AA
:10C2100083AB0900938789002326F100138E060063
:10C2200063C8061E9306F0FF13090D006388DC0047
:10C23000B3E6CB011379FDF76382067AE31A0E00A9
:10C2400093069000E3E6760193870B03A307F10EB4
:10C25000130D0900930B10009309F10E6F00C00637
:10C26000136D0D0193770D02638607148327C100B8
:10C270009389770093F989FF83AB090003AE4900E6
:10C28000938789002326F1001379FDBF93060000F0
:10C29000A30D01021306F0FF6380CC1A33E6CB0135
:10C2A000137DF9F76312065E63960C3E639C06727B
:10C2B000937B19009309010F63880B009307000318
:10C2C000A307F10E9309F10E13890C0063D47C01CE
:10C2D00013890B008347B103B337F0003309F9002A
:10C2E0006FF01FD63309B441E314B4C98347040087
:10C2F0006FF0DFCB1306010493050A0013050B0052
:10C30000EFF0DF9EE31805E413870A006FF01FC902
:10C31000930600010327410463D07607930C0001C4
:10C32000930970006F00C000938B0BFF63D67C05F0
:10C33000938707011307170023A0850123A2950106
:10C340002324F1042322E10493858500E3DEE9FC44
:10C350001306010493050A0013050B00EFF01F9963
:10C36000E31A05DE938B0BFF832781040327410427
:10C3700093850A00E3CE7CFBB38777011307170090
:10C3800023A0850123A275012324F1042322E104C3
:10C3900093067000E3D8E6D81306010493050A005B
:10C3A00013050B00EFF09F94E31605DA8327810451
:10C3B0006FF05FD70326C10093770D019306460007
:10C3C0006390077E93770D04E38607188327C100E7
:10C3D000130E00002326D10083DB07006FF0DFEA95
:10C3E0000326C10093770D019306460063960778F4
:10C3F00093770D04E38007148327C1002326D1001F
:10C40000839B070013DEFB4193060E00E3DC06E08E
:10C41000B3367001330EC041330EDE409306D002B6
:10C42000A30DD1021306F0FFB30B704113090D00E9
:10C4300093061000E394CCE613061000E380C6E0F8
:10C44000130620006382C6269309010F1316DE012E
:10C4500093F67B0093D73B0093860603B36BF600FD
:10C46000135E3E00A38FD9FE33E6CB01938509000E
:10C470009389F9FFE31C06FC937719006380072674
:10C4800093070003638CF6249385E5FFA38FF9FEE1
:10C490009307010FB38BB740130D09009389050073
:10C4A0006FF09FE28327C100A30D010283A907005B
:10C4B00093864700E38009049307F0FF232CE100F3
:10C4C0002326D1006382FC7813860C0093050000BC
:10C4D00013850900EFD05FFF8326C1000327810188
:10C4E000E30E0512B30B3541930C00006FF0DFDD56
:10C4F0008326C100A30D01021309100083A70600C3
:10C50000938646002326D1002306F108930B1000E2
:10C510009309C1086FF09FB28327C10013692D00F2
:10C52000B786FFFF83AB0700375D01809387470025
:10C5300093C606832326F1009307CD79231ED102EB
:10C54000130E00002328F100930620006FF05FD443
:10C550000326C10093770D028326060013064600CA
:10C560002326C1006390076093770D01639E0776D1
:10C5700093770D04E394070893780D20638608767B
:10C58000832781002380F6006FF01F9C83C60D0077
:10C59000136D0D086FF01FA483C60D0093851D0059
:10C5A000E386360B938706FD938D0500930C000000
:10C5B000E3E4FBA283C60D0093952C003383950121
:10C5C00013131300B30CF300938706FD938D1D0026
:10C5D000E3F2FBFE6FF05FA083C60D00136D4D000C
:10C5E0006FF05F9F9307B00283C60D00A30DF102A9
:10C5F0006FF05F9E8327C10083C60D0003A4070070
:10C60000938747002326F100E356049C33048040BF
:10C61000136D4D006FF01F9C83C60D00136D1D0040
:10C620006FF05F9B8347B10383C60D00E394079AC5
:10C6300093070002A30DF1026FF0DF9983C60D008E
:10C640009307C0066384F666136D0D016FF09F9823
:10C6500083C60D00930780066382F664136D0D0494
:10C660006FF05F9713690D019377090263840738B0
:10C670008327C100930610009389770093F989FFFF
:10C680009387890083AB090003AE49002326F1009C
:10C690006FF01FC013061000638AC67813062000CF
:10C6A00013090D00E392C6DA9309010F83270101F4
:10C6B00093F6FB009389F9FFB386D70003C6060003
:10C6C00093D74B009316CE01B3EBF600135E4E00EA
:10C6D0002380C900B3E6CB01E39A06FC9307010F60
:10C6E000B38B3741130D09006FF01FBEB306244111
:10C6F000E350D0A0130E0001635EDE72130F7000D2
:10C700006F00C000938606FF635EDE049387070117
:10C7100013061600232097002322C7012324F104C7
:10C720002322C10413078700E35ECFFC1306010434
:10C7300093050A0013050B00232CD100EFF00FDB4B
:10C74000E31A05A083268101130E000183278104CB
:10C75000938606FF0326410413870A00130F700017
:10C76000E346DEFA13061600130E8700B387D700E0
:10C77000232097002322D7002324F1042322C1047D
:10C7800013077000634CC752B38C7C41130516002D
:10C7900093058E0013070E00E350909713030001DA
:10C7A0006358935F130E70006F00C000938C0CFFF2
:10C7B000635A9305938707011306160023209700F9
:10C7C000232267002324F1042322C10413078700D6
:10C7D000E35ECEFC1306010493050A0013050B006B
:10C7E000EFF0CFD0E318059613030001938C0CFFF4
:10C7F000832781040326410413870A00130E700067
:10C80000E34A93FB1305160013068700B3879701CD
:10C8100023209700232297012324F1042322A1043B
:10C82000130770006340A7201307060013051500C7
:10C83000B387FB0023203701232277012324F1044F
:10C840002322A1041307700093058600E354A78CEC
:10C850001306010493050A0013050B00EFF00FC93E
:10C86000E31A058E8327810493850A006FF09F8A5F
:10C870001306010493050A0013050B00EFF00FC720
:10C88000E30E058A6FF01F8D13090D006FF0DFBAFC
:10C890009305000163D0D508930F00019302700047
:10C8A0006F00C000938606FF63D6DF0693870701FB
:10C8B00013061600232087012322F7012324F10405
:10C8C0002322C10413078700E3DEC2FC1306010420
:10C8D00093050A0013050B002320D102232EC1016A
:10C8E000232CE101EFF08FC0E316058683260102B9
:10C8F000930F000183278104938606FF03264104DA
:10C90000032EC101032F810113870A0093027000D7
:10C91000E3CEDFF8B387D700130616002322D70033
:10C92000232087012324F1042322C10493067000ED
:10C930001307870063D8C6F21306010493050A00A3
:10C9400013050B00232EC101232CE101EFF00FBAD8
:10C95000E31205808327810403264104032EC101CD
:10C96000032F810113870A006FF0CFEF1306010434
:10C9700093050A0013050B00232EC101232CE101AE
:10C98000EFF0CFB6631805FC03264104832781042A
:10C99000032EC101032F81019305410513051600E4
:10C9A00013870A006FF0CFF01306010493050A0005
:10C9B00013050B00232CC101EFF04FB3631C05F8E6
:10C9C0000326410483278104032E81019305410539
:10C9D0001305160013870A006FF00FF1E3960C861B
:10C9E000130D0900930C0000930B00009309010F35
:10C9F0006FF09F8D0326C1009377090193064600CF
:10CA00006396071893770904638407368327C10068
:10CA1000130E00002326D10083DB070093061000CD
:10CA20006FF01F871306010493050A0013050B001E
:10CA3000EFF0CFAB631005F2032541048327810497
:10CA4000930541051305150013870A006FF0CFEA1F
:10CA5000937709402320F102130D00009309010F81
:10CA60006F00400393050E001306A000930600001C
:10CA700013850B00232EE100232CC101EF40805AC7
:10CA8000032E81010327C10163080E30930B0500BB
:10CA9000138E050093050E001306A00093060000F8
:10CAA00013850B00232EE100232CC101EF40D01A87
:10CAB0008327010213050503A38FA9FE032E81011D
:10CAC0000327C1019389F9FF130D1D00E38C07F8BB
:10CAD0008327410283C60700E396A6F99307F00F68
:10CAE000E302FDF863160E0093079000E3F877BFAA
:10CAF000832781028325C102232EC101B389F94016
:10CB00001386070013850900232CE100EFF08F93B3
:10CB100003274102032EC1011306A000834517001D
:10CB20009306000013850B00B337B000B307F7007E
:10CB300093050E002322F102EF40C04E032781012E
:10CB4000130D00006FF09FF48327410283C60D0090
:10CB5000638207C883C70700638E07C6136D0D4045
:10CB60006FF04FC7032681009357F64123A0C600FC
:10CB700023A2F6006FF04FBD832B06002326D100C1
:10CB800013DEFB4193060E006FF08FE92326D100E0
:10CB9000832B0600130E0000930610006FF04FEF7A
:10CBA000832B0600130E00002326D1006FF0CFED7B
:10CBB00013090D006FF05FABB75701809387077BB8
:10CBC0002328F10093770D02638007068327C100B5
:10CBD0009389770093F989FF83AB090003AE49007D
:10CBE000938789002326F10013761D00630E06004B
:10CBF00033E6CB01630A060013060003230EC102CD
:10CC0000A30ED102136D2D001379FDBF93062000F2
:10CC10006FF00FE8B75701809387C7792328F10099
:10CC200093770D02E39407FA8325C10093770D01F2
:10CC3000138645006386070483AB0500130E0000CE
:10CC40002326C1006FF05FFA13850900EFE0DFF6DD
:10CC500003278101930B0500930C00006FF0CFE6D2
:10CC600093050004EFD08F832320AA002328AA0075
:10CC70006300052093070004232AFA006FF08FA8B1
:10CC800093770D04638A07088327C100130E000001
:10CC90002326C10083DB07006FF01FF583C61D004C
:10CCA000136D0D20938D1D006FF0CFB283C61D0054
:10CCB000136D0D02938D1D006FF0CFB113060104AB
:10CCC00093050A0013050B00EFF04F82631405C8AB
:10CCD00003264104832781049305410513051600AB
:10CCE00013870A006FF0CFC08327810023A0F600CE
:10CCF0006FF08FA593076000938B0C0063F497018E
:10CD0000930B6000B75E018013890B002326D100CE
:10CD100093894E7C6FF08FB293770D206386070C5A
:10CD20008327C100130E00002326C10083CB070018
:10CD30006FF09FEB93770D20638C07088327C1006A
:10CD40002326D100838B070013DEFB4193060E00E0
:10CD50006FF00FCD93770D20638207068327C10004
:10CD6000130E00002326D10083CB07006FF0CFD134
:10CD700093770920638807028327C100130E000000
:10CD80002326D10083CB0700930610006FF04FD00D
:10CD9000138605006FF09FA793079000E3E877CF15
:10CDA0006FF0DF938327C100130E00002326D1000C
:10CDB00083AB0700930610006FF08FCD8327C1006F
:10CDC000130E00002326D10083AB07006FF0CFCBFA
:10CDD0008327C1002326D10083AB070013DEFB416C
:10CDE00093060E006FF0CFC38327C100130E00001F
:10CDF0002326C10083AB07006FF01FDF832781006C
:10CE00002390F6006FF04F941306010493050A0077
:10CE100013050B00EFE09FED6FF0CFB3938B0C0089
:10CE20002326D100930C00006FF00FCA13090D00E8
:10CE30006FF08FC1138E0500130605006FF01F936E
:10CE40009307F0FF2324F1006FF08FB18327C10017
:10CE500083AC07009387470063D40C00930CF0FF6A
:10CE600083C61D002326F100938D05006FF08F9679
:10CE70009307C0002320FB009307F0FF2324F10059
:10CE80006FF00FAEB777018083A7876667800700D2
:10CE9000638405029307F00F63E8C7002380C50091
:10CEA00013051000678000009307A0082320F500F9
:10CEB0001305F0FF67800000130500006780000085
:10CEC000B787018003A747B2130101FF93870600CC
:10CED00013080600232611008328C70093060500C7
:10CEE000138705001386070063000802B7670180F7
:10CEF0009387C7F0B76501809385C5F11385080056
:10CF0000EF004011EF1090673758018093070845F4
:10CF1000130808456FF01FFE130101FF930606007A
:10CF20001306000023261100EFF09FF9B385C50218
:10CF3000130101FF2324810023261100EFC01FD617
:10CF400013040500630805020326C5FF130740020A
:10CF50001376C6FF1306C6FF6360C706930630014B
:10CF60009307050063E2C60223A0070023A207007F
:10CF700023A407008320C1001305040003248100BB
:10CF80001301010167800000232005002322050012
:10CF90009307B00163F0C70423240500232605008E
:10CFA00093070501E312E6FC23280500930785019A
:10CFB000232A05006FF05FFB93050000EF60DFA4FC
:10CFC0008320C10013050400032481001301010123
:10CFD00067800000930785006FF01FF9130101FCC3
:10CFE0001303C1022326D10293060300232E11004E
:10CFF0002328E102232AF102232C0103232E11030B
:10D0000023266100EF0010128320C10113010104E7
:10D0100067800000130E050037850180130101FCB5
:10D02000032545B2130381022324C1022326D10222
:10D03000138605009306030093050E00232E1100AE
:10D040002328E102232AF102232C0103232E1103BA
:10D0500023266100EF00100D8320C101130101049C
:10D0600067800000B3C7A50093F73700B308C50079
:10D07000639207069307300063FEC7049377350079
:10D08000130705006398070613F6C8FF930706FE0B
:10D09000636CF708637CC70293860500930707005B
:10D0A00003A80600938747009386460023AE07FF38
:10D0B000E3E8C7FE9307F6FFB387E74093F7C7FFA0
:10D0C000938747003307F700B385F50063681701BE
:10D0D0006780000013070500E37C15FF83C7050088
:10D0E0001307170093851500A30FF7FEE36817FFDA
:10D0F0006780000083C60500130717009377370089
:10D10000A30FD7FE93851500E38007F883C60500BB
:10D110001307170093773700A30FD7FE93851500E9
:10D12000E39A07FC6FF05FF683A6450083A2050033
:10D1300083AF850003AFC50083AE050103AE450193
:10D1400003A3850103A8C5012322D70083A60502F6
:10D15000232057002324F7012326E7012328D701A2
:10D16000232AC701232C6700232E07012320D7027F
:10D170001307470293854502E368F7FA6FF09FF1C2
:10D1800063F6A502B387C5006372F5023307C500D5
:10D19000630A060E83C6F7FF9387F7FF1307F7FFAF
:10D1A0002300D700E398F5FE678000009307F000A6
:10D1B00063E8C702930705009306F6FF630C060CAD
:10D1C00093861600B386D70003C705009387170020
:10D1D00093851500A38FE7FEE398D7FE67800000D4
:10D1E000B3E7A50093F737006390070A930806FF9B
:10D1F00093F808FF93880801330815011387050089
:10D20000930705008326070013070701938707018B
:10D2100023A8D7FE832647FF23AAD7FE832687FFAE
:10D2200023ACD7FE8326C7FF23AED7FEE31CF8FC52
:10D230001377C600B38515011378F600630E070453
:10D240001387050093880700130E3000032307009F
:10D2500013074700B306E84023A06800B386D50053
:10D2600093884800E364DEFE1307C8FF1377C7FF07
:10D270001307470013763600B387E700B385E50050
:10D280006FF09FF3678000009306F6FF9307050099
:10D290006FF01FF367800000130608006FF0DFF1E6
:10D2A000130101FD232021032326110223248102DF
:10D2B00023229102232E3101232C4101232A5101E3
:10D2C000232861012326710123248101130906000B
:10D2D0006386051C1384050093090500EFD04FAB4E
:10D2E0009304B9009307600163FE970E93F484FFE3
:10D2F0001387040063CE040E63EC240F8327C4FF5E
:10D30000930A84FF13FAC7FF338B4A01635EEA1264
:10D31000B7760180938B466F03A68B0083264B0064
:10D320006300661F13F6E6FF3306CB0003264600B4
:10D33000137616006316061493F6C6FF3306DA005A
:10D340006358E60E93F7170063940702032C84FFDB
:10D35000338C8A4183274C0093F7C7FFB386D700ED
:10D36000B38B460163DAEB34B30BFA0063D4EB2CD6
:10D370009305090013850900EFC05F9213090500AA
:10D38000630C05048327C4FF130785FF93F7E7FFAA
:10D39000B387FA006386E7281306CAFF93074002A3
:10D3A00063E6C7301307300183260400636EC7208D
:10D3B000930705001307040023A0D7008326470026
:10D3C00023A2D7000327870023A4E70093050400C6
:10D3D00013850900EF905F8113850900EFD08F9BC3
:10D3E0006F00C0019304000113070001E3F824F16A
:10D3F0009307C00023A0F900130900008320C10295
:10D4000003248102832441028329C101032A81016B
:10D41000832A4101032B0101832BC100032C8100CE
:10D4200013050900032901021301010367800000AD
:10D430008327CB0003278B00130A0600338BCA0017
:10D440002326F70023A4E70083A74A0033079A4066
:10D450009306F00093F7170063ECE606B367FA0053
:10D4600023A2FA0083274B0093E717002322FB0037
:10D4700013850900EFD00F92130904006FF01FF815
:10D4800093F71700E39607EE032C84FF338C8A4151
:10D4900083274C0093F7C7FF6FF01FED0324810231
:10D4A0008320C10283244102032901028329C1018F
:10D4B000032A8101832A4101032B0101832BC1002F
:10D4C000032C810093050600130101036FC00FFDBB
:10D4D000B3E7970023A2FA00B3859A0013671700F9
:10D4E00023A2E50083274B0093858500138509005F
:10D4F00093E717002322FB00EF900FEF6FF05FF729
:10D5000093F6C6FF3306DA00938504016350B60E26
:10D5100093F71700E39E07E4032C84FF338C8A41C2
:10D5200083274C0093F7C7FFB386D700338B4601A0
:10D53000E34CBBE28327CC0003278C001306CAFF11
:10D54000930640022326F70023A4E70013098C006A
:10D5500063ECC626930530010327040093070900F6
:10D5600063F2C5022324EC00032744009307B001B3
:10D570002326EC0063E2C7260327840093070C01EF
:10D580001304840023A0E7000327440023A2E7003C
:10D590000327840023A4E70033079C00B3079B40C4
:10D5A00023A4EB0093E717002322F70083274C0006
:10D5B0001385090093F71700B3E4970023229C001A
:10D5C000EFC05FFD6FF09FE32320D500832644006A
:10D5D0001307B0012322D500636EC716832684008B
:10D5E00013078400930785006FF01FDDB38A9A004C
:10D5F000B307964023A45B0193E7170023A2FA0028
:10D600008327C4FF138509001309040093F717004B
:10D61000B3E49700232E94FEEFC0DFF76FF01FDE18
:10D620008327C5FF93F7C7FF330AFA00338B4A01FC
:10D630006FF09FE18327CC0003278C001306CAFFFD
:10D64000930640022326F70023A4E70013098C0069
:10D65000330B7C0163E2C60E9305300103270400FF
:10D660009307090063F2C5022324EC00032744005A
:10D670009307B0012326EC0063E0C7100327840062
:10D6800093070C011304840023A0E7000327440040
:10D69000138A0B00930A0C0023A2E70003278400DF
:10D6A0001304090023A4E7006FF01FDA93050400B8
:10D6B000EFF01FAD6FF09FD18327CB0003278B00C6
:10D6C0001306CAFF930640022326F70023A4E700AF
:10D6D00003278C008327CC0013098C00330B7C01BB
:10D6E0002326F70023A4E70063E8C604930630016D
:10D6F0000327040093070900E3F8C6F82324EC008D
:10D70000032744009307B0012326EC00032784007D
:10D71000E3F8C7F62328EC000327C4009307400270
:10D72000232AEC00032704016304F60693078C0107
:10D73000130404016FF05FF593050400130509005D
:10D74000EFF01FA413040900138A0B00930A0C00C6
:10D750006FF09FCF032784002324E5000327C40034
:10D760002326E500832604016302F604130704015F
:10D77000930705016FF05FC4832784002328FC0012
:10D780008327C400232AFC0003270401E310D6FAF0
:10D79000232CEC000327440193070C02130484019B
:10D7A000232EEC00032704006FF01FEE2328D50082
:10D7B000832644011307840193078501232AD5009A
:10D7C000832684016FF05FBF9305040013050900F1
:10D7D000EFF01F9B6FF05FDC832784002328FC00A1
:10D7E0008327C400232AFC00032704016308D60012
:10D7F00093078C01130404016FF0DFD8232CEC0095
:10D800000327440193070C0213048401232EEC0028
:10D81000032704006FF01FD703A74506130101FD7E
:10D82000B727000023286101232611022324810247
:10D830002322910223202103232E3101232C410195
:10D84000232A51012326710123248101B3F7E70024
:10D85000130B06006388070A83278600832B0600C4
:10D860001389050093090500930AF0FF63880708F0
:10D8700003AC4B0003A40B00135A2C0063060A06EA
:10D88000930400006F00C00013044400630C9A046A
:10D89000832504001306090013850900EF10D050FA
:10D8A00093841400E31255FF1305F0FF8320C10297
:10D8B0000324810223240B0023220B008324410232
:10D8C000032901028329C101032A8101832A41011D
:10D8D000032B0101832BC100032C810013010103E1
:10D8E0006780000083278B00137CCCFFB3878741C0
:10D8F0002324FB00938B8B00E39C07F613050000A9
:10D900006FF0DFFAEF1010556FF05FFA0327860013
:10D91000630407006FF05FF0232206001305000088
:10D9200067800000130101ED232E3111232A5111CC
:10D93000232EB10F232611122324811223229112A8
:10D9400023202113232C4111232861112326711137
:10D9500023248111232291112320A1112326D100F8
:10D96000930A050093890500930D060063060500E0
:10D97000832785036380076E0397C900B7260000DD
:10D980009317070193D7070133F6D70063180602F0
:10D9900003A64906B367D7009397070137E7FFFF50
:10D9A00093D707411307F7FF3377E6002396F90073
:10D9B0009397070123A2E90693D7070113F787007E
:10D9C0006304073E03A709016300073E93F7A7011D
:10D9D0001307A000638AE73EB76701809304C10480
:10D9E0009387C7F4376C0180376901802320910445
:10D9F00023240104232201041387040023280100A7
:10DA000023220102232401022326010223240100F0
:10DA1000232AF100130C8C0B1309890C83C70D000A
:10DA2000638E072413840D0093065002638ED7443F
:10DA30008347140013041400E39A07FE330AB44129
:10DA4000630EB42383268104832741042320B70176
:10DA5000B306DA0093871700232247012324D10459
:10DA60002322F10413067000130787006350F602A7
:10DA7000E382063A130601049385090013850A0020
:10DA8000EFF09FD9631005201387040083268100DF
:10DA900083470400B38646012324D1006380071E18
:10DAA00083461400930D1400A30D0102930CF0FFA4
:10DAB00013040000130D0000130AA005930B90003F
:10DAC000130BA002938D1D00938706FE6364FA0476
:10DAD0000326410193972700B387C70083A7070058
:10DAE0006780070013040000938706FD83C60D00BE
:10DAF00093152400338485001314140033848700A5
:10DB0000938706FD938D1D00E3F2FBFE938706FECF
:10DB1000E370FAFC638406162306D108A30D010204
:10DB2000130A1000930B1000130BC108930C000094
:10DB3000937F2D0063840F00130A2A00832641047B
:10DB4000137F4D0883278104138616009305060072
:10DB500063160F0033084441E342001B0345B10341
:10DB600013068700630C05029306B1032320D70038
:10DB700093871700930610002322D7002324F10473
:10DB80002322B10413077000E348B70E9386050003
:10DB9000130706009385150013068600638E0F0495
:10DBA0009306C1032320D700938727009306200004
:10DBB0002322D7002324F1042322B1041307700089
:10DBC000E350B712E382072A130601049385090084
:10DBD00013850A00232CE101EFF01FC46314050A2A
:10DBE0008326410483278104032F81011306410505
:10DBF000938516001387040013050008630CAF6AB1
:10DC0000B38C7C4163489079B387FB002320670184
:10DC1000232277012324F1042322B1041307700087
:10DC20006352B702638A072613060104938509002D
:10DC300013850A00EFF05FBE631605048327810495
:10DC400013860400937E4D0063860E00B30B44419F
:10DC5000634070276354440113040A0003278100C2
:10DC6000330787002324E1006394077E83C70D00F8
:10DC70002322010413870400E39607DA8327810433
:10DC8000E39E076283D7C90093F70704E39607660C
:10DC90008320C112032481120325810083244112B1
:10DCA000032901128329C111032A8111832A4111F9
:10DCB000032B0111832BC110032C8110832C4110E5
:10DCC000032D0110832DC10F130101136780000084
:10DCD00013850A00232CE100EFB09FEA832745005B
:10DCE000138507002326F102EFD01FED93070500EF
:10DCF00013850A002324F102EFB09FE80327850073
:10DD0000832781022322E10203278101E390072E6A
:10DD100083C60D006FF01FDB83C60D00136D0D026F
:10DD20006FF05FDA136D0D0193770D0263820726A2
:10DD30008327C100138B7700137B8BFF83264B0057
:10DD4000832B0B0093078B002326F100138806001A
:10DD500063C806269306F0FF130A0D006388DC00F3
:10DD6000B3E60B01137AFDF7E38C060AE3140812FD
:10DD700093069000E3E0761393870B03A307F10E5D
:10DD8000130D0A00930B1000130BF10E138A0C00F5
:10DD900063D47C01138A0B008347B103B337F000CF
:10DDA000330AFA006FF0DFD89385090013850A0063
:10DDB000EF001066E312055483D7C9001307A000D3
:10DDC00093F7A701E39AE7C08397E900E3C607C08A
:10DDD000032481128326C1008320C11283244112AF
:10DDE00003290112032A8111032B0111832BC11076
:10DDF000032C8110832C4110032D011013860D007C
:10DE000093850900832DC10F8329C11113850A0051
:10DE1000832A4111130101136F009053136D0D01FB
:10DE200093770D02638007148327C100138B77005B
:10DE3000137B8BFF832B0B0003284B0093078B0076
:10DE40002326F100137AFDBF93060000A30D010203
:10DE50001306F0FF638ACC1833E60B01137DFAF743
:10DE6000631A066863940C3E6390067C937B1A00E9
:10DE7000130B010FE38C0BF093070003A307F10EC4
:10DE8000130BF10E6FF09FF0330AB441E31CB4BBE7
:10DE9000834704006FF09FC023220104937E4D004E
:10DEA00063860E72B30B4441635270731386040091
:10DEB0001307000183264104E3587743930C0001C4
:10DEC000130B70006F0080019385260013068600F7
:10DED00093060700938B0BFF63D87C05938707019C
:10DEE0001387160023208601232296012324F104A0
:10DEF0002322E104E35AEBFC6386073A130601048C
:10DF00009385090013850A00EFF01F91E31C05D6E5
:10DF100083264104938B0BFF83278104138604001F
:10DF200093851600E3CC7CFBB38777012320860121
:10DF3000232276012324F1042322B1041307700065
:10DF4000E35AB7D063840768130601049385090078
:10DF500013850A00EFF05F8CE31605D28327810456
:10DF60006FF05FCF0326C10093770D019306460043
:10DF7000E390070C93770D04E38E07228327C100FB
:10DF8000130800002326D10083DB07006FF09FEB0E
:10DF90000326C10093770D0193064600E39007081E
:10DFA00093770D04E388071E8327C1002326D10041
:10DFB000839B070013D8FB4193060800E3DC06D8D7
:10DFC000B3367001330800413308D8409306D002BD
:10DFD000A30DD1021306F0FFB30B7041130A0D001D
:10DFE00093061000E39ACCE613061000E380C6D82F
:10DFF000130620006386C626130B010F1316D801E3
:10E0000093F67B0093D73B0093860603B36BF60031
:10E0100013583800A30FDBFE33E60B0193050B000A
:10E02000130BFBFFE31C06FC93771A00638407269F
:10E03000930700036380F6269385E5FFA30FFBFE9D
:10E040009307010FB38BB740130D0A00138B050024
:10E050006FF0DFD3EF10003E6FF01F928327C100F7
:10E06000A30D010203AB070093864700E3040B10E6
:10E070009307F0FF232CE1002326D100E38CFC065C
:10E0800013860C009305000013050B00EFC0CFC3EF
:10E090008326C10003278101E30C0522B30B6541F0
:10E0A000930C00006FF09FCE8326C100A30D0102E8
:10E0B000130A100083A70600938646002326D1008A
:10E0C0002306F108930B1000130BC1086FF01FA675
:10E0D00083C60D009307C006E380F608136D0D019B
:10E0E0006FF05F9E83C60D0093078006E38EF604F3
:10E0F000136D0D046FF01F9D136A0D0193770A02D3
:10E10000638C07528327C10093061000138B77009E
:10E11000137B8BFF93078B00832B0B0003284B0093
:10E120002326F1006FF09FD283C60D00136D0D08FA
:10E130006FF05F998327C100136A2D00B786FFFF38
:10E1400083AB0700375D01809387470093C6068342
:10E150002326F1009307CD79231ED1021308000076
:10E160002328F100930620006FF05FCE0326C10044
:10E1700093770D0283260600130646002326C1006E
:10E180006394076893770D016390077E93770D047E
:10E19000E394070C937E0D2063880E7C8327810017
:10E1A0002380F6006FF09F878327C10083C60D0090
:10E1B00003A40700938747002326F100E35404904B
:10E1C00033048040136D4D006FF0DF8F83C60D0068
:10E1D000136D1D006FF01F8F8347B10383C60D00C1
:10E1E000E392078E93070002A30DF1026FF09F8D5B
:10E1F00083C60D00136D4D006FF0DF8C9307B002E6
:10E2000083C60D00A30DF1026FF0DF8B83C60D00F6
:10E2100093851D00E38E660F938706FD938D0500A1
:10E22000930C0000E3E2FB8A83C60D0013982C00D8
:10E230003308980113181800B30CF800938706FDF3
:10E24000938D1D00E3F2FBFE6FF01F881306100094
:10E25000E380C60A13062000130A0D00E39EC6D809
:10E26000130B010F8327010193F6FB00130BFBFF38
:10E27000B386D70003C6060093D74B009316C80198
:10E28000B3EBF600135848002300CB00B3E60B01B4
:10E29000E39A06FC9307010FB38B6741130D0A0045
:10E2A0006FF0DFAE930510009306000013860400A4
:10E2B0006FF05FC233084441E35400951305000139
:10E2C000E3520505130F0001930F70006F008001EA
:10E2D000138526001307870093060600130808FF1E
:10E2E00063500F0793870701138616002320270129
:10E2F0002322E7012324F1042322C104E3DACFFC23
:10E3000063840716130601049385090013850A0028
:10E31000232C0101EFF04FD0E3160596032881016D
:10E3200083264104130F0001130808FF832781048B
:10E330001387040013851600930F7000E3440FFB4E
:10E34000130F8700B387070123202701232207012A
:10E350002324F1042322A104130770006354A74669
:10E360006380076C130601049385090013850A0076
:10E37000EFF08FCAE318059083264104B38C7C41EB
:10E380008327810413064105938516001387040033
:10E39000E35C908713050001635A9567130300013E
:10E3A000130F70006F00800193852600130787000C
:10E3B00093060600938C0CFF635C9305938707011B
:10E3C0001386160023202701232267002324F1044B
:10E3D0002322C104E35ACFFC638407061306010419
:10E3E0009385090013850A00EFF00FC3E31C05882D
:10E3F0008326410413030001938C0CFF83278104BF
:10E400001387040093851600130F7000E34893FBF5
:10E4100093068700B38797012320270123229701C2
:10E420002324F1042322B10413077000634CB71AAC
:10E430009385150013868600138706006FF0CFFCC6
:10E440009305100093060000138704006FF09FF6F9
:10E45000130601049385090013850A00EFF0CFBB72
:10E46000E30605806FF01F8213051000930600007D
:10E47000138704006FF09FE66382072013060104F0
:10E480009385090013850A00232EE101232CF10155
:10E49000EFF08FB8631805FE8326410483278104BB
:10E4A000032FC101832F81011306410593851600B7
:10E4B000138704006FF08FEE639A072C0347B103B4
:10E4C000631E0756638E0F1A9307C1032326F104B8
:10E4D000930720002328F10413064105930510003B
:10E4E0001307060093860500938516001306870020
:10E4F0006FF08FF0130A0D006FF01FAF930500014E
:10E5000063D0055F93020001930370006F00C001A8
:10E51000138526001307870093060600130808FFDB
:10E5200063D802071386160093870701232087010B
:10E53000232257002324F1042322C104E3DAC3FC7D
:10E54000638E0706130601049385090013850A00EC
:10E5500023200103232EE101232CF101EFF0CFABA7
:10E56000631205F20328010283264104930200018D
:10E57000130808FF83278104032FC101832F810122
:10E58000138704001385160093037000E3CC02F98F
:10E59000B387070123208701232207012324F104E5
:10E5A0002322A10493067000E3C8A6F01307870096
:10E5B00093051500930605006FF04FDA93060000EF
:10E5C00013051000138704006FF05FF563544401D6
:10E5D00013040A0083278100B38787002324F100F6
:10E5E0006FF0CFE8638407321306010493850900B6
:10E5F00013850A00EFF04FA2631605E88325410456
:10E6000083278104130641059385150013870400B1
:10E610006FF08FDF23220104138704006FF00FC710
:10E62000639C0CF4130D0A00930C0000930B000084
:10E63000130B010F6FF08FF50326C10093770A01CA
:10E6400093064600639A071893770A046380073A93
:10E650008327C100130800002326D10083DB0700B5
:10E66000930610006FF08FFE13064105930510000E
:10E6700093060000138704006FF00FD863920F1CFD
:10E68000930600001306410593051000138704004C
:10E690006FF08FD693770A402320F102130D00000C
:10E6A000130B010F6F004003930508001306A00031
:10E6B0009306000013850B00232EE100232C01019B
:10E6C000EF205016032881010327C1016304083499
:10E6D000930B050013880500930508001306A0009E
:10E6E0009306000013850B00232EE100232C01016B
:10E6F000EF2090568327010213050503A30FABFEFD
:10E70000032881010327C101130BFBFF130D1D001B
:10E71000E38C07F88327410283C60700E396A6F936
:10E720009307F00FE302FDF86316080093079000CB
:10E73000E3F277B7832781028325C102232E0101EB
:10E74000330BFB401386070013050B00232CE1005D
:10E75000EFD04FCF032741020328C1011306A000C9
:10E76000834517009306000013850B00B337B000F4
:10E77000B307F700930508002322F102EF20900A67
:10E7800003278101130D00006FF09FF413060104AD
:10E790009385090013850A00232EE101232CF10142
:10E7A000EFF08F87631005CE832641048327810411
:10E7B000032FC101832F8101138704009385160065
:10E7C0006FF0CFB99305150013068F00930605006F
:10E7D00013070F006FF0CFC22326D100832B060052
:10E7E00013080000930610006FF04FE683274102E4
:10E7F00083C60D00638807AC83C70700638407AC3A
:10E80000136D0D406FF00FAC032681009357F64156
:10E8100023A0C60023A2F6006FF04FA0832B0600B2
:10E820002326D10013D8FB41930608006FF04FD286
:10E83000832B0600130800002326D1006FF08FE021
:10E840009307C1032326F104930720002328F10432
:10E8500013074105930610006FF01FC9B7570180D9
:10E860009387077B2328F10093770D0263840706C3
:10E870008327C100138B7700137B8BFF832B0B0047
:10E8800003284B0093078B002326F10013761D000D
:10E89000630E060033E60B01630A0600130600034D
:10E8A000230EC102A30ED102136D2D00137AFDBFFA
:10E8B000930620006FF08FD9130A0D006FF01F84AC
:10E8C000B75701809387C7792328F10093770D020A
:10E8D000E39007FA8325C10093770D011386450065
:10E8E0006386070483AB0500130800002326C100DC
:10E8F0006FF0DFF913050B00EFD00FAC0327810198
:10E90000930B0500930C00006FF04FC81307100025
:10E9100093870B00232661052328710523247105A5
:10E920002322E104130641056FF0CFB193770D0464
:10E930006380070A8327C100130800002326C10053
:10E9400083DB07006FF09FF483C61D00136D0D205D
:10E95000938D1D006FF00F9783C61D00136D0D0280
:10E96000938D1D006FF00F968327810023A0F60082
:10E970006FF0CF8A93076000938B0C0063EC970BCA
:10E98000B7580180138A0B002326D100138B487CD3
:10E990006FF0CF9993770D20638607108327C1000E
:10E9A0002326D100838B070013D8FB419306080070
:10E9B0006FF00FBA93770D20638C070C8327C1008B
:10E9C000130800002326D10083CB07006FF08FC708
:10E9D00093770D206384070A8327C1001308000082
:10E9E0002326C10083CB07006FF05FEA93770A20EC
:10E9F000638A07068327C100130800002326D1007D
:10EA000083CB0700930610006FF04FC493060600F7
:10EA10006FF05FA093079000E3EC77CB6FF09F87D8
:10EA200013064105930510009306000013870400A8
:10EA30006FF00F9D930B60006FF09FF49307B1038D
:10EA40002326F104930710002328F104130641053F
:10EA5000930510006FF08F93832781002390F600B9
:10EA60006FE0DFFB8327C100130800002326D100DD
:10EA700083AB0700930610006FF04FBD8327C100E2
:10EA8000130800002326C10083AB07006FF01FE0CE
:10EA90008327C100130800002326D10083AB0700A1
:10EAA0006FF04FBA8327C1002326D10083AB070044
:10EAB00013D8FB41930608006FF08FA913060104D9
:10EAC0009385090013850A00EFE01FD56FF08F9B37
:10EAD000938B0C002326D100930C00006FF00FAB3A
:10EAE000130506006FF0DFAA938516006FF0CFC301
:10EAF000130A0D006FF04FA89307F0FF2324F100D5
:10EB00006FF00F99130F0600138505006FF09F83B8
:10EB10008327C10083AC07009387470063D40C00B0
:10EB2000930CF0FF83C61D002326F100938D050092
:10EB30006FE05FF93787018093070500032547B22F
:10EB40009306060013860500938507006FE09FDD9E
:10EB500083D7C50003AE450603D3E50083A8C501EE
:10EB600003A84502130101B893F7D7FF130700402C
:10EB7000232C8146231AF100138405009307010713
:10EB800093058100232A914623282147232E1146ED
:10EB9000130905002326C107231B6100232211034B
:10EBA000232601032324F100232CF1002328E10074
:10EBB000232EE10023200102EFE0DFD693040500BD
:10EBC000635C05028357410193F7070463880700DC
:10EBD0008357C40093E707042316F4008320C1473A
:10EBE00003248147032901471385040083244147F7
:10EBF0001301014867800000930581001305090097
:10EC0000EF00803FE30005FC9304F0FF6FF09FFBF3
:10EC1000B787018083A747B2130101FF2324810036
:10EC2000232291002326110093040500138405007C
:10EC30006386070003A78703630407080317C4005C
:10EC4000931707019376870093D707016388060817
:10EC5000832604016388060A13F617006308060278
:10EC60000326440123240400130500003306C0409A
:10EC7000232CC400638A06028320C1000324810080
:10EC800083244100130101016780000013F627006F
:10EC90009305000063140600832544012324B40077
:10ECA00013050000E39A06FC93F70708E38607FCC8
:10ECB000136707042316E4001305F0FF6FF0DFFB72
:10ECC00013850700EF0000770317C40093170701AF
:10ECD0009376870093D70701E39C06F693F6070126
:10ECE0006382060893F747006394070483260401B0
:10ECF00013678700931707012316E40093D70701D2
:10ED0000E39C06F413F6072893050020E306B6F407
:10ED10009305040013850400EF00D0720317C400AC
:10ED2000832604019317070193D707016FF0DFF2E1
:10ED300083250403638E0500930704046388F500AC
:10ED400013850400EF705FEA0317C4002328040250
:10ED5000832604011377B7FD232204002320D40067
:10ED60006FF01FF99307900023A0F40013670704C6
:10ED70002316E4001305F0FF6FF01FF0130101FFED
:10ED80001305600023261100EF10C03D130510008D
:10ED9000EF109FAC8397C500130101FE232C810067
:10EDA00023263101232E1100232A9100232821013B
:10EDB00093F687001384050093090500639C0610F1
:10EDC000371700001307078083A64500B3E7E70065
:10EDD0002396F5006356D01803278402630C070CB2
:10EDE0009397070193D70701B716000083A4090082
:10EDF000B3F6D70023A009008325C4016398061643
:10EE0000930610001306000013850900E7000700B1
:10EE10009307F0FF630EF5188357C400032784029D
:10EE20008325C40193F74700638E070083264400BF
:10EE3000832704033305D540638607008327C40373
:10EE40003305F540130605009306000013850900FD
:10EE5000E70007009307F0FF631EF51003A7090002
:10EE60008317C400630A07169306D0016306D70010
:10EE7000930660016314D70C8326040137F7FFFF64
:10EE80001307F77FB3F7E7002316F40023220400EB
:10EE90002320D4008325040323A09900638C05005C
:10EEA000930704046386F50013850900EF70DFD330
:10EEB00023280402130500008320C10103248101DB
:10EEC00083244101032901018329C10013010102A7
:10EED0006780000003A90501E30E09FC83A4050077
:10EEE00013970701135707011377370023A0250154
:10EEF000B3842441930700006314070083A74501EE
:10EF00002324F400634890006FF0DFFA3309A9006E
:10EF1000E35290FA832744028325C40193860400B8
:10EF20001306090013850900E7800700B384A44095
:10EF3000E34EA0FC8357C4001305F0FF93E70704DA
:10EF40008320C1012316F40003248101832441019D
:10EF5000032901018329C100130101026780000018
:10EF600003A7C503E34AE0E66FF0DFF403250405D9
:10EF70006FF05FEB8357C40037F7FFFF1307F77F8E
:10EF8000B3F7E700832604019397070193D707415E
:10EF900013D7C7002316F400232204002320D40033
:10EFA00093771700E38807EE2328A4046FF09FEE01
:10EFB00083A70900E38207E61307D0016388E7020D
:10EFC000130760016384E7028357C40093E70704D3
:10EFD0002316F4006FF05FEE37F7FFFF1307F77F9C
:10EFE00083260401B3F7E7006FF09FFA23A099008E
:10EFF000130500006FF05FEC130101FE232C81006C
:10F00000232E1100130405006306050083278503E2
:10F01000638007028397C500639607028320C101BE
:10F020000324810113050000130101026780000021
:10F030002326B100EF0000408325C1008397C5005F
:10F04000E38E07FC13050400032481018320C10122
:10F05000130101026FF01FD463080506130101FEBE
:10F06000B7870180232C81001304050003A547B254
:10F07000232E11006306050083278503638A070298
:10F080008317C400639C07008320C101032481010E
:10F0900013050000130101026780000093050400BE
:10F0A000032481018320C101130101026FF09FCE6F
:10F0B0002326A100EF0000388317C4000325C100F8
:10F0C000E38407FC6FF09FFDB787018003A507B2BB
:10F0D000B7F50080938585FF6F00902B1305000026
:10F0E00067800000B7150180938545A36F00502A03
:10F0F0001305000067800000130101FEB7F70080D0
:10F10000232E1100232C8100232A91002328210182
:10F1100023263101232441012322510123206101AF
:10F12000032445009387470E232EF5021307C52EAF
:10F13000930730002324E52E2322F52E2320052ECD
:10F1400093074000130905002326F40013068000EE
:10F150009305000023220406232004002322040038
:10F160002324040023280400232A0400232C040061
:10F170001305C405EF405F89370B018083248900A4
:10F18000B70A0180370A0180B7090180130B0B4AC7
:10F19000938A4A50130ACA589389495FB7070100F6
:10F1A000232064032322540323244403232634030B
:10F1B000232E84009387970023A6F4001306800073
:10F1C0009305000023A2040623A0040023A2040048
:10F1D00023A4040023A8040023AA040023AC0400F1
:10F1E0001385C405EF405F820324C900B7070200FE
:10F1F00023A0640323A2540323A4440323A63403BB
:10F2000023AE9400938727012326F40023220406CB
:10F2100023200400232204002324040023280400C4
:10F22000232A0400232C04001305C40513068000C0
:10F2300093050000EF404FFD8320C10123206403AC
:10F24000232254032324440323263403232E84003F
:10F250000324810193071000232CF9028324410128
:10F26000032901018329C100032A8100832A410067
:10F27000032B01001301010267800000130101FF4D
:10F2800023229100130680069384F5FFB384C40201
:10F290002320210113890500232481002326110046
:10F2A00093854407EFA09F9F1304050063000502A8
:10F2B0001305C50023200400232224012324A400D5
:10F2C0001386840693050000EF400FF48320C100ED
:10F2D0001305040003248100832441000329010055
:10F2E0001301010167800000130101FEB78701804F
:10F2F0002328210103A907B223263101232E11005F
:10F3000083278903232C8100232A91002324410190
:10F3100093090500638A070A1309092E9304F0FF75
:10F32000130A400083274900032489009387F7FFCD
:10F3300063D807006F00400813048406638E9706A5
:10F340000317C4009387F7FFE31807FEB707FFFF13
:10F35000938717002322040623200400232204009D
:10F36000232404002326F40023280400232A040075
:10F37000232C040013068000930500001305C40528
:10F38000EF408FE823280402232A040223220404E6
:10F39000232404048320C1011305040003248101F4
:10F3A00083244101032901018329C100032A81002B
:10F3B000130101026780000003240900630C0400AC
:10F3C000130904006FF01FF613050900EFF0DFD2F8
:10F3D0006FF09FF49305C01A13850900EFA01F8CEE
:10F3E00013040500630605021305C500232004006D
:10F3F000232244012324A4001306001A93050000CD
:10F40000EF408FE023208900130904006FF09FF183
:10F41000232009009307C00023A0F9006FF09FF795
:10F42000B787018003A507B2B7150180938545A36F
:10F430006F000076832785036384070067800000E0
:10F440006FF09FCB6780000067800000678000003E
:10F4500067800000B787018003A547B2B7F5008039
:10F460009385C50D6F008068B787018003A547B2FB
:10F47000B7F500809385050F6F004067130101FD0C
:10F4800023248102232E3101232861012326110226
:10F490002322910223202103232C4101232A5101FD
:10F4A000130B05009389050013040600EFA08FF6E7
:10F4B000930710006310F5029387F9FF1307E00F1D
:10F4C000636AF70013F7F90F2306E1001309100030
:10F4D0006F00C0029306C405138609009305C1009E
:10F4E00013050B00EF10802B9307F0FF13090500A5
:10F4F0006304F50A630E05080347C1009304000086
:10F50000130AF0FF930AA0006F0080028327040013
:10F51000938617002320D4002380E70093841400EF
:10F520009307C100B387970063F4240703C707005C
:10F53000832784009387F7FF2324F400E3D807FC94
:10F5400083268401930507001306040013050B00AE
:10F5500063C4D700E31C57FBEF10400AE31045FDDE
:10F560001309F0FF8320C102032481028324410296
:10F570008329C101032A8101832A4101032B01014F
:10F58000130509000329010213010103678000002C
:10F59000138909006FF01FFD8357C40093E7070428
:10F5A0002316F4006FF01FFC8317C6001397270182
:10F5B0006340070203274606B7260000B3E7D700DB
:10F5C000B72600003367D7002316F6002322E6068D
:10F5D0006FF0DFEA130101FEB7870180232C810061
:10F5E00003A447B2232E11001386050093050500DE
:10F5F0006306040083278403638007048317C6001F
:10F60000139727016340070203274606B726000029
:10F61000B3E7D700B72600003367D7002316F600FC
:10F620002322E60613050400032481018320C1017F
:10F63000130101026FF09FE42324A10013050400CD
:10F640002326C100EFF01FDF0326C10083258100C0
:10F650006FF0DFFA832786006388073083D7C50001
:10F66000130101FD23248102232C4101232A51018E
:10F67000232611022322910223202103232E31016C
:10F680002328610123267101232481012322910172
:10F690002320A10113F78700130A0600930A05002F
:10F6A000138405006306070803A705016302070822
:10F6B00013F7270083240A00630C070883274402FA
:10F6C0008325C401370B0080930900001309000053
:10F6D000134B0BC01386090013850A00630209044B
:10F6E0009306090063742B0193060B00E780070063
:10F6F0006352A02683278A00B389A9003309A94051
:10F700003385A7402324AA006300052083274402F1
:10F710008325C4011386090013850A00E31209FC3E
:10F7200083A9040003A94400938484006FF09FFA26
:10F730009305040013850A00EFF08FCD6314053A9A
:10F740008357C40083240A0013F72700E31807F641
:10F7500013F7170063160712832C84000325040097
:10F76000370B0080934BEBFF130C000013090000D4
:10F77000134BFBFF630E090E13F7072063080724E2
:10F78000138D0C00636E992D13F70748630A070861
:10F790008329440183250401130719009396190056
:10F7A000B386360193D9F601330DB540B389D9003C
:10F7B00093D919403307A7011386090063F6E900BE
:10F7C000930907001306070093F707406386072C89
:10F7D0009305060013850A00EFA04FCC930C05009B
:10F7E000630A052E8325040113060D00EFD09F87C1
:10F7F0008357C40093F7F7B793E707082316F4007D
:10F800003385AC01B387A941232894012320A400A8
:10F81000232A3401930C09002324F400130D09005A
:10F8200013060D0093050C00EFD09F95032784006D
:10F830008327040093090900B30C9741B387A701FC
:10F84000232494012320F4001309000003268A00D6
:10F85000330C3C01B309364123243A016386090A7B
:10F86000832C8400032504008357C400E31609F0A9
:10F8700003AC040003A94400938484006FF09FEF5D
:10F88000130B000013050000130C00009309000087
:10F890006380090E6306050E93070B00938B090026
:10F8A00063F43701938B07000325040083270401C9
:10F8B0008326440163F8A7000329840033892601C5
:10F8C0006340790F63C4DB1A832744028325C40194
:10F8D00013060C0013850A00E780070013090500D2
:10F8E000635AA006330B2B4113051000630C0B0465
:10F8F00003268A00330C2C01B389294133092641A0
:10F9000023242A01E31609F8130500008320C1020D
:10F910000324810283244102032901028329C101B6
:10F92000032A8101832A4101032B0101832BC1009A
:10F93000032C8100832C4100032D010013010103DE
:10F94000678000009305040013850A00EFF0CFEAFA
:10F95000E30005FA8317C40093E707042316F400B5
:10F960001305F0FF6FF09FFA130500006780000099
:10F9700083A9440003AC040093848400E38A09FE55
:10F98000138609009305A00013050C00EFA0DFB358
:10F99000630C051213051500330B85416FF0DFEF83
:10F9A00093050C0013060900EFD08FFD8327040098
:10F9B0009305040013850A00B38727012320F40070
:10F9C000EFF08FE3E30005F26FF0DFF88327040127
:10F9D00063E2A70483274401636EF90293060900DA
:10F9E00063F42B0193060B00B3C6F602032744020F
:10F9F0008325C40113060C0013850A00B386F602A2
:10FA0000E700070093090500E356A0F433093941E4
:10FA10006FF0DFE393890C00637499019309090087
:10FA20001386090093050C00EFD08FF5832784001F
:10FA300003270400B3873741330737012324F40039
:10FA40002320E400E39407FC9305040013850A00D7
:10FA5000EFF08FDAE31005F0330939416FF01FDF63
:10FA6000930C0900130D09006FF09FDB13860B0048
:10FA700093050C00EFD0CFF0032784008327040008
:10FA800013890B0033077741B38777012324E40000
:10FA90002320F4006FF01FE513850A00EFD05F808C
:10FAA000930C0500E31E05D48325040113850A0089
:10FAB000EF708F938317C4001307C00023A0EA00E0
:10FAC00093F7F7F76FF05FE993871900138B07003F
:10FAD0006FF0DFDC1307C0008317C40023A0EA0027
:10FAE0006FF09FE71305F0FF6FF05FE2130101FE77
:10FAF00023282101232631012324410123225101FE
:10FB000023206101232E1100232C8100232A910040
:10FB1000138B0500930A052E130A000093091000A9
:10FB20001309F0FF83A44A0003A48A009384F4FF1E
:10FB300063C604028357C4009384F4FF63FCF90096
:10FB40008317E4001305040063862701E7000B0018
:10FB5000336AAA0013048406E39E24FD83AA0A00E4
:10FB6000E3920AFC8320C101032481018324410123
:10FB7000032901018329C100832A4100032B0100CD
:10FB800013050A00032A81001301010267800000A7
:10FB9000130101FD23202103232E3101232C4101D8
:10FBA000232A5101232861012326710123261102F2
:10FBB0002324810223229102930A0500938B0500DE
:10FBC000130B052E130A0000930910001309F0FF10
:10FBD00083244B0003248B009384F4FF63C8040246
:10FBE0008357C4009384F4FF63FEF9008317E40095
:10FBF0009305040013850A0063862701E7800B0044
:10FC0000336AAA0013048406E39C24FD032B0B0033
:10FC1000E3100BFC8320C1020324810283244102F0
:10FC2000032901028329C101832A4101032B010118
:10FC3000832BC10013050A00032A8101130101036C
:10FC40006780000083D7C500130101F8232C8106CB
:10FC5000232E1106232A9106232821072326310764
:10FC60002324410713F7270013840500630C0702C0
:10FC70009387350423A0F50023A8F500930710000F
:10FC800023AAF5008320C1070324810783244107A9
:10FC9000032901078329C106032A810613010108EC
:10FCA000678000008395E5009304050063CC050898
:10FCB00013068100EF009066634405088327C100A6
:10FCC00037F90000130A00403379F900B7E7FFFF66
:10FCD0003309F900B7170000133919009389078019
:10FCE00093050A0013850400EF905FFB8317C4009F
:10FCF000630E050637F700801307470E23AEE402B4
:10FD000093E707082316F4002320A4002328A40067
:10FD1000232A440163180908B3E737018320C10788
:10FD20002316F400032481078324410703290107D4
:10FD30008329C106032A8106130101086780000098
:10FD40008357C40093F7070813090000638607046C
:10FD5000130A000493050A0013850400EF901FF4B2
:10FD60008317C40093090000E31605F813F7072072
:10FD7000E31A07F093F7C7FF93E72700130734044C
:10FD80002316F400930710002320E4002328E40046
:10FD9000232AF4006FF01FEF130A004093090000BC
:10FDA0006FF01FF48315E40013850400EF00905DED
:10FDB000631605008317C4006FF01FF68357C40055
:10FDC00093F7C7FF93E717009397070193D707416E
:10FDD0006FF09FF4130101F92324810613840500B9
:10FDE0008395E5002322910623202107232611066F
:10FDF000930406001389060063CA050413068100F4
:10FE0000EF00D051634405040327C100B7F7000099
:10FE10008320C106B3F7E70037E7FFFFB387E700AA
:10FE20000324810693B717002320F90093070040AD
:10FE300023A0F4003715000083244106032901069E
:10FE40001305058013010107678000008317C400B4
:10FE50002320090093F70708638407028320C10663
:10FE6000032481069307000423A0F400032901065C
:10FE70008324410613050000130101076780000079
:10FE80008320C106032481069307004023A0F400C9
:10FE9000032901068324410613050000130101070D
:10FEA000678000008327C52D6386070013050000C7
:10FEB00067800000130101FF9305000823248100DF
:10FEC0002326110013040500EF905FDD232EA42CE0
:10FED0006304050293070508232005001305450068
:10FEE000E31CF5FE130500008320C10003248100FC
:10FEF00013010101678000001305F0FF6FF0DFFEC2
:10FF0000130101FE232A9100232E1100232C8100CE
:10FF10009307F0019304050063EAB7020327C52D98
:10FF200013840500630407041314240033048700BA
:10FF3000032504002320C4008320C1010324810180
:10FF40008324410113010102678000008320C10165
:10FF500003248101930760012320F50083244101DC
:10FF60001305F0FF130101026780000093050008EC
:10FF70002326C100EF909FD223AEA42C13070500C7
:10FF8000630005020326C1009307050093060508D8
:10FF900023A0070093874700E39CD7FE6FF0DFF8AC
:10FFA0001305F0FF6FF05FF9130101FF23229100A9
:10FFB00023261100232481009307F00193040500F8
:10FFC00063EAB70A8327C52D1384050063840704F9
:10FFD00013972500B387E70003A70700630C070208
:10FFE00093061000630CD7069306F0FF6308D7044E
:10FFF0001385050023A00700E70007001305000094
:02000004800179
:100000008320C100032481008324410013010101E6
:100010006780000013850400EF00404813060400C9
:10002000032481008320C10093050500138504008B
:1000300083244100130101016F00C03F8320C100F0
:1000400003248100930760012320F50083244100ED
:100050001305100013010101678000008320C10017
:1000600003248100832441001305000013010101D2
:1000700067800000930760012320F5001305F0FF5F
:100080006FF01FF89307F00163EAB70C0327C52D43
:10009000130101FF23248100232291002326110054
:1000A000138405009304050063000706131524005C
:1000B0003307A70083270700638C07029306F0FF2E
:1000C0006386D708930610006386D70613050400DD
:1000D00023200700E7800700130500008320C100EC
:1000E0000324810083244100130101016780000083
:1000F0008320C100032481008324410013051000E4
:10010000130101016780000093050008EF901FB9FB
:1001100023AEA42C13070500630E05029307050008
:100120009306050823A0070093874700E39CD7FEAA
:100130006FF0DFF78320C100032481008324410096
:100140001305300013010101678000001305200032
:100150006FF0DFF81305F0FF6FF05FF81305F0FFA5
:1001600067800000130101FF23229100378701807F
:1001700023261100232481009307F001832447B232
:1001800063E8A70A83A7C42D13040500638207044C
:1001900013172500B387E70003A70700630A0702C8
:1001A00093061000630AD7069306F0FF6306D70490
:1001B00023A00700E7000700130500008320C1000B
:1001C00003248100832441001301010167800000A2
:1001D00013850400EF00802C130604000324810023
:1001E0008320C1009305050013850400832441008A
:1001F000130101016F0000248320C100032481004A
:100200009307600123A0F40013051000832441002C
:1002100013010101678000008320C10003248100D5
:1002200083244100130500001301010167800000D1
:100230009307600123A0F4001305F0FF6FF01FF88F
:10024000130101FF2320210137870180232611009C
:1002500023248100232291009307F001032947B250
:1002600063EEA702130405000325C92D938405003E
:1002700063080504131424003304850003250400D7
:10028000232094008320C1000324810083244100A3
:100290000329010013010101678000008320C100D0
:1002A00003248100930760012320F9008324410087
:1002B000032901001305F0FF13010101678000000D
:1002C0009305000813050900EF905F9D232EA92CCC
:1002D000630E0500930705001307050823A0070018
:1002E00093874700E31CF7FE6FF0DFF81305F0FF7C
:1002F0006FF05FF9130101FFB787018023248100AC
:1003000003A447B2232611008327C42D638C070062
:10031000130500008320C1000324810013010101A3
:10032000678000009305000813050400EF901F97F5
:10033000232EA42C630C0500930705082320050039
:1003400013054500E31CF5FE6FF09FFC1305F0FF5D
:100350006FF05FFC130101FF2322910037870180BA
:1003600023261100232481009307F001832447B240
:1003700063EEA70A03A7C42D130405006300070654
:10038000131524003307A70083270700638C070297
:100390009306F0FF6388D708930610006388D7069A
:1003A0001305040023200700E78007001305000061
:1003B0008320C10003248100832441001301010133
:1003C000678000008320C100032481008324410052
:1003D0001305100013010101678000009305000858
:1003E00013850400EF909F8B23AEA42C1307050008
:1003F000630E0502930705009306050823A0070076
:1004000093874700E39CD7FE6FF09FF78320C100DE
:1004100003248100832441001305300013010101EE
:1004200067800000130520006FF09FF81305F0FFB0
:100430006FF01FF8130101FF1387050023248100CB
:100440002322910013040500B78401809305060060
:10045000130507002326110023A004B4EF00101792
:100460009307F0FF630CF5008320C1000324810093
:1004700083244100130101016780000083A704B4B5
:10048000E38407FE8320C1002320F40003248100BD
:100490008324410013010101678000006F00900E6A
:1004A000130101FF23248100138405008395E500D7
:1004B00023261100EF00C07963400502832704055D
:1004C0008320C100B387A7002328F40403248100FC
:1004D00013010101678000008357C40037F7FFFF55
:1004E0001307F7FFB3F7E7008320C1002316F400DA
:1004F000032481001301010167800000130500003F
:10050000678000008397C500130101FE232C810042
:10051000232A91002328210123263101232E1100B3
:1005200013F7071013840500930405008395E50075
:100530001309060093890600631E070237F7FFFFC1
:100540001307F7FFB3F7E7002316F4000324810134
:100550008320C10193860900130609008329C10085
:1005600003290101138504008324410113010102C1
:100570006F0080339306200013060000EF008066B2
:100580008317C4008315E4006FF05FFB130101FFC4
:1005900023248100138405008395E50023261100A0
:1005A000EF0040649307F0FF6304F5028357C40033
:1005B000371700008320C100B3E7E7002328A40415
:1005C0002316F40003248100130101016780000059
:1005D0008357C40037F7FFFF1307F7FFB3F7E700B0
:1005E0008320C1002316F4000324810013010101BC
:1005F000678000008395E5006F00C031130101FEA4
:10060000232C8100232A910023282101232E11006D
:100610002326310113090500938405001304060005
:100620006306050083278503638A07140317C40044
:1006300083268401937787002324D400931607012F
:1006400093D60601638407088327040163800708A3
:1006500037260000B3F6C60093F9F40F93F4F40FB5
:100660006380060A0327040083264401B307F7408A
:1006700063DED70A83268400130617002320C400F4
:100680009386F6FF2324D400230037010327440177
:10069000938717006308F70C8357C40093F717007C
:1006A000638607009307A000638EF40A8320C101CC
:1006B00003248101032901018329C100138504005A
:1006C00083244101130101026780000093050400A7
:1006D00013050900EFE0CFD3631E05080317C4001C
:1006E0003726000093F9F40F9316070193D60601FD
:1006F000B3F6C6008327040193F4F40FE39406F6DF
:10070000832644063367C70037E6FFFF1306F6FF6C
:10071000B3F6C6002316E400032704002322D40600
:1007200083264401B307F740E3C6D7F493050400DA
:1007300013050900EFE05F8C631E05020327040028
:100740008326840093071000130617009386F6FF94
:100750002320C4002324D4002300370103274401AD
:10076000E31CF7F29305040013050900EFE0DF88AE
:10077000E30E05F29304F0FF6FF05FF3EFE09FCB21
:100780006FF0DFEA3787018093070500032547B242
:1007900013860500938507006FF05FE6130101FEE5
:1007A000232C8100232A9100B7770180232E11008A
:1007B00083A78766130405009384060063820502FD
:1007C000E78007009307F0FF6306F5028320C1016D
:1007D0000324810183244101130101026780000089
:1007E0001306000093054100E78007009307F0FF20
:1007F000E31EF5FC23A004009307A0088320C10199
:100800002320F40003248101832441011301010208
:1008100067800000130101FEB7870180232C81004F
:10082000232A9100232E110083A447B2B7770180B9
:1008300083A7876613040600630A05021386050072
:10084000930604009305050013850400E780070064
:100850009307F0FF630AF5028320C101032481019D
:100860008324410113010102678000009306060002
:10087000930541001306000013850400E78007007C
:100880009307F0FFE31AF5FC232004008320C10145
:10089000032481019307A00823A0F40083244101CD
:1008A0001301010267800000130101FF1387050097
:1008B00023248100232291009305060013040500E0
:1008C000B784018013860600130507002326110054
:1008D00023A004B4EF00C0659307F0FF630CF5009C
:1008E0008320C100032481008324410013010101FE
:1008F0006780000083A704B4E38407FE8320C1005F
:100900002320F4000324810083244100130101010A
:1009100067800000130101FF23248100232291003E
:1009200013040500B78401801385050023261100F8
:1009300023A004B4EF0080389307F0FF630CF500A8
:100940008320C1000324810083244100130101019D
:100950006780000083A704B4E38407FE8320C100FE
:100960002320F400032481008324410013010101AA
:1009700067800000130101FF2324810023229100DE
:100980002320210113840500232611009304050070
:10099000EFE04FC08327C40213090500638A0700F4
:1009A0008325C40113850400E7800700634405061E
:1009B0008357C40093F7070863960706832504034B
:1009C000638C0500930704046386F5001385040017
:1009D000EF608FA123280402832544046388050067
:1009E00013850400EF604FA023220404EFE09FA5CD
:1009F00023160400EFE05FA58320C10003248100DB
:100A0000832441001305090003290100130101019A
:100A1000678000008357C4001309F0FF93F70708AD
:100A2000E38E07F88325040113850400EF60CF9B54
:100A30006FF0DFF863840506130101FE232C8100AB
:100A4000232E110013040500630605008327850388
:100A5000638A07028397C500639C07008320C10156
:100A600003248101130500001301010267800000C7
:100A700013050400032481018320C1011301010235
:100A80006FF05FEF2326B100EFE0DF9A8325C1000E
:100A90008397C500E38407FC6FF09FFD13050000FA
:100AA0006780000063080506130101FEB787018017
:100AB000232C81001304050003A547B2232E110047
:100AC0006306050083278503638A07028317C40032
:100AD000639C07008320C1010324810113050000EA
:100AE00013010102678000009305040003248101C3
:100AF0008320C101130101026FF0DFE72326A1006B
:100B0000EFE05F938317C4000325C100E38407FC73
:100B10006FF09FFD1305000067800000130101FFC7
:100B2000138705002324810023229100130405006C
:100B3000B7840180930506001305070023261100E2
:100B400023A004B4EF00001D9307F0FF630CF50031
:100B50008320C1000324810083244100130101018B
:100B60006780000083A704B4E38407FE8320C100EC
:100B70002320F40003248100832441001301010198
:100B800067800000130101FF2324810023229100CC
:100B900013040500B7840180138505002326110086
:100BA00023A004B4EF00801E9307F0FF630CF50050
:100BB0008320C1000324810083244100130101012B
:100BC0006780000083A704B4E38407FE8320C1008C
:100BD0002320F40003248100832441001301010138
:100BE00067800000130101FF1387050023248100A3
:100BF000232291009305060013040500B7840180A9
:100C000013860600130507002326110023A004B451
:100C1000EF00001E9307F0FF630CF5008320C10076
:100C20000324810083244100130101016780000037
:100C300083A704B4E38407FE8320C1002320F400CB
:100C40000324810083244100130101016780000017
:100C5000130101FF13870500232481002322910043
:100C60009305060013040500B7840180138606006F
:100C7000130507002326110023A004B4EF00401C35
:100C80009307F0FF630CF5008320C100032481006B
:100C900083244100130101016780000083A704B48D
:100CA000E38407FE8320C1002320F4000324810095
:100CB000832441001301010167800000130101FF3B
:100CC0002326110023248100930500001306000051
:100CD0009306000013070000930700009308900399
:100CE0007300000013040500634C05008320C1005D
:100CF0001305040003248100130101016780000033
:100D000033048040EF20DFBC232085001304F0FF74
:100D10006FF0DFFD130101F723229108232611084C
:100D20009384050023248108930501001306000025
:100D300093060000130700009307000093080005C6
:100D400073000000130405006344050213850400CA
:100D500093050100EF00C0228320C10813050400A1
:100D600003248108832441081301010967800000DE
:100D700033048040EF20DFB5232085001304F0FF0B
:100D80006FF0DFFC1305100067800000130101F90C
:100D90009305810023261106EFF0DFF79307F0FF9C
:100DA000630EF5000325C1008320C1061355D5004D
:100DB0001375150013010107678000008320C10629
:100DC000130500001301010767800000130101FFF4
:100DD00023261100EF20DFAF8320C10093076001BD
:100DE0002320F5001305F0FF1301010167800000C7
:100DF000130101FF23261100232481009306000024
:100E000013070000930700009308E003730000003D
:100E100013040500634C05008320C1001305040082
:100E20000324810013010101678000003304804026
:100E3000EF201FAA232085001304F0FF6FF0DFFDD1
:100E4000130101FF232611002324810093060000D3
:100E500013070000930700009308F00373000000DD
:100E600013040500634C05008320C1001305040032
:100E700003248100130101016780000033048040D6
:100E8000EF201FA5232085001304F0FF6FF0DFFD86
:100E900037830180832743B4130101FF2326110008
:100EA000130805006398070213050000930500006E
:100EB0001306000093060000130700009308600D5E
:100EC000730000001307F0FF930705006304E504B7
:100ED0002322A3B43305F800930500001306000095
:100EE0009306000013070000930700009308600DAD
:100EF00073000000832743B43308F800631C050126
:100F00008320C1002322A3B413850700130101012C
:100F100067800000EF20DF9B8320C1009307C000A3
:100F20002320F5001305F0FF130101016780000085
:100F3000130101FF232611002324810093060000E2
:100F400013070000930700009308000473000000DB
:100F500013040500634C05008320C1001305040041
:100F600003248100130101016780000033048040E5
:100F7000EF201F96232085001304F0FF6FF0DFFDA4
:100F8000130101FF83A3450183A2850183AFC5013E
:100F900003AF050283AE050303AE050403A3850377
:100FA00003A8850483A8C50403A68505232681001C
:100FB0002324910003A4050183A485002322210199
:100FC00003A9050083A6C50503A7850683A7C50653
:100FD0002310250123119500232285002314750079
:100FE000231555002316F5012317E5012328D50104
:100FF0002326C50523246504232C0501232E150172
:101000002324C5022326D5020324C100232CE50294
:10101000232EF502832481000329410013010101DD
:1010200067800000930805009387050013080600F9
:10103000138506001383080063940628B7560180C1
:101040009386865863F6C50E370701006378E60C71
:101050001307F00F3337C700131737003355E60077
:10106000B386A60083C60600130500023387E60098
:10107000B306E540630CE500B395D70033D7E8002D
:101080003318D600B365B7003393D80093580801DE
:10109000B3D615031316080113560601935703011F
:1010A00033F7150313850600B305D602131707019E
:1010B000B367F70063FEB700B38707011385F6FF38
:1010C00063E8070163F6B7001385E6FFB3870701FE
:1010D000B387B74033F71703131303011353030107
:1010E000B3D717031317070133636700B306F6027C
:1010F00013860700637CD300330368001386F7FF71
:10110000636603016374D3001386E7FF13150501BB
:101110003365C500930500006F00400E37050001E0
:1011200013070001E36CA6F2130780016FF01FF3B1
:1011300063160600130710003358C7023707010073
:101140006370E80C1307F00F637407011305800048
:101150003357A800B386E60003C706001306000253
:101160003307A700B306E6406316E60AB3870741D4
:101170009305100093580801131608011356060131
:1011800013570301B3F61703B3D71703939606015A
:1011900033E7E600330EF60213850700637EC701CE
:1011A000330707011385F7FF636807016376C701FB
:1011B0001385E7FF330707013307C741B3771703E9
:1011C00013130301135303013357170393970701B5
:1011D00033E36700B306E60213060700637CD3001F
:1011E000330368001306F7FF636603016374D300DB
:1011F0001306E7FF131505013365C500678000007E
:101200003707000113050001E364E8F413058001CA
:101210006FF01FF43318D80033D5E7003393D800AC
:10122000B397D70033D7E800935808013366F70027
:10123000337715039317080193D7070193550601D8
:1012400033551503131707013367B700B386A70299
:1012500093050500637ED700330707019305F5FF6B
:10126000636807016376D7009305E5FF330707013D
:10127000B306D74033F716031316060113560601BB
:10128000B3D61603131707013385D702B367C70018
:101290001387060063FEA700B38707011387F6FFD5
:1012A00063E8070163F6A7001387E6FFB38707012A
:1012B00093950501B387A740B3E5E5006FF09FEB79
:1012C00063E6D5183707010063F4E6041307F00F4F
:1012D000B335D700939535003757018033D5B60025
:1012E000130787583307A7000347070013050002B9
:1012F0003307B700B305E5406316E5021305100098
:10130000E3EEF6EE33B5C800134515006FF01FEF9E
:101310003707000193050001E3E0E6FC9305800137
:101320006FF09FFB3358E600B396B6003368D800E1
:1013300033DEE700935E0801B376DE03B397B700B0
:1013400033D7E8003313B6003366F700931708016C
:1013500093D7070113570601335EDE039396060108
:1013600033E7E600338FC70313050E00637EE70102
:10137000330707011305FEFF636807016376E70182
:101380001305EEFF330707013307E741B376D703B1
:101390003357D70393960601338EE702931706015E
:1013A00093D70701B3E7F6001306070063FEC701F2
:1013B000B38707011306F7FF63E8070163F6C70168
:1013C0001306E7FFB387070113150501B70E0100E8
:1013D0003365C5009386FEFF3378D50013560501AB
:1013E000B376D30013530301B387C741330ED8023A
:1013F000B306D60213570E01330868023308D8002B
:1014000033070701330666026374D7003306D6013B
:10141000935607013386C60063E6C702E39CC7CE36
:10142000B70701009387F7FF3377F700131707011A
:10143000337EFE00B398B8003307C7019305000060
:10144000E3FEE8DA1305F5FF6FF0DFCC930500004B
:10145000130500006FF09FDA930E0500138305005B
:101460001308060093870600639A06223757018007
:101470001307875863FCC50CB7060100637ED60AC4
:101480009306F00F63F4C60093078000B356F6008E
:101490003307D70003470700B307F700130700021D
:1014A000B308F740630CF700B3151301B3D7FE0080
:1014B00033181601B3E5B70033951E0193560801A2
:1014C000B3F7D50213160801135606011357050189
:1014D000B3D5D5029397070133E7E700B305B6020A
:1014E000637AB70033070701636607016374B700C7
:1014F000330707013307B740B377D7021315050148
:10150000135505013357D7029397070133E5A70019
:101510003307E602637AE5003305050163660501DA
:101520006374E500330505013305E54033551501C6
:101530009305000067800000B706000193070001D3
:10154000E366D6F4930780016FF05FF4631606003C
:101550009306100033D8C602B70601006376D8128E
:101560009306F00F63F4060193078000B356F8006A
:101570003307D70003460700B30503413306F600DF
:1015800093070002B388C7406386C7083318180161
:10159000B357C300B31513011353080133D6CE005C
:1015A0003366B6009315080193D5050133951E01E6
:1015B000B3D6670233F7670293570601B386D502A5
:1015C000131707013367F700637AD7003307070162
:1015D000636607016374D70033070701B306D7407A
:1015E00033F766021316060113560601B3D66602D8
:1015F00013170701B386D502B365C70063FAD50098
:10160000B385050163E6050163F4D500B3850501E3
:10161000B385D5409356080133F7D50293170801D7
:1016200093D7070113560501B3D5D5021317070148
:101630003367C700B385B702637AB7003307070182
:10164000636607016374B70033070701B305B7404A
:1016500033F7D5021315050113550501B3D5D5028E
:10166000B385B7029317070133E5A700637AB50086
:1016700033050501636605016374B5003305050193
:101680003305B5406FF09FEAB706000193070001EC
:10169000E36ED8EC930780016FF05FEDE3ECD5E8E3
:1016A000B707010063F8F6049308F00FB3B7D8004A
:1016B000939737003757018033D8F60013078758C0
:1016C0003307070183480700B388F8009307000237
:1016D00033881741639A170363E46600E3ECCEE4B2
:1016E0003385CE40B305D340B3BEAE00B385D541FC
:1016F0006FF05FE43707000193070001E3ECE6FABF
:10170000930780016FF01FFBB3571601B3960601D4
:1017100033EED700335F1301B3D71E0133950E01AB
:10172000935E0E01B31503013353DF03B3E7B70034
:1017300093150E0193D5050113D707013316060142
:10174000B376DF03338F65029396060133E7E60035
:1017500093060300637EE7013307C7019306F3FF97
:101760006368C7016376E7019306E3FF3307C701A8
:101770003307E7413373D7039397070193D70701E3
:101780003357D703131303013363F300B385E50223
:1017900093070700637EB3003303C3019307F7FF8A
:1017A0006368C3016376B3009307E7FF3303C301A4
:1017B00093960601370F0100B3E6F600B305B34078
:1017C0001303FFFFB3FE66001357060193D606010D
:1017D00033736600B3876E0233836602B38EEE0204
:1017E000B386E602B38E6E0013D707013307D70125
:1017F00063746700B386E60113530701B306D30091
:10180000370301001303F3FF337767001317070152
:10181000B3F76700B307F70063E6D500639ED50012
:10182000637CF5003386C740B3B7C700B387C701F1
:10183000B386F64093070600B307F5403335F5004D
:10184000B385D540B385A540B398150133D50701BD
:1018500033E5A800B3D505016FF0DFCD8327050080
:10186000832E4500032F85008326C50003A70500AE
:1018700083A2450083AF850003A3C500130101FFC8
:10188000732620003788000013D606011308F8FFDE
:10189000139E06019315030193D8F60133760601D2
:1018A00093560301135E0E0193D50501B3F60601AD
:1018B0001353F301631E060133E8D7013368E801CF
:1018C0003368C80163120808639CC60A6F00800071
:1018D000639A0601336857003368F8013368B8002B
:1018E00063160804130510006396C6026394E702AA
:1018F00063925E026310FF03631EBE00638468028E
:10190000639A060033E5D7013365E5013365C50108
:101910003335A000130101016780000073601800D7
:101920006F000006130500006FF0DFFE3785000032
:101930001305F5FF6310A604B3E7D701B3E7E7018A
:10194000B3E7C7016388070213150E01135505415C
:10195000E35605FCB78700009387F7FF13051000D7
:10196000E39AF6FA336757003367F7013367B70036
:10197000E30207FA9395050193D50541E3D005FAF3
:10198000130510006FF01FF9832F05000328450091
:10199000032E850083A205000325C50083A845000A
:1019A00083AE850083A6C500130101FFF327200045
:1019B000B7870000135605019387F7FF93150501BC
:1019C0001393060113D706013376F60093D505016C
:1019D0001355F501135303013377F70093D6F6013E
:1019E0006310F602B367F801B3E7C701B3E7B700C6
:1019F000638A070C736018001305E0FF6F00400650
:101A0000631AF700B3E71201B3E7D701B3E7670042
:101A1000E39207FE631A060AB367F801B3E7C7014A
:101A2000B3E7B70093B71700631A070033EF12014B
:101A3000336FDF01336F6F00630A0F06639C07008B
:101A40006394A6006352C702630E05041305F0FFFA
:101A50006F0000011305F0FF638406001385060084
:101A600013010101678000006356E600E31A05FEDA
:101A70006FF0DFFDE36AB3FC639E6502E3E6CEFD33
:101A8000631EDE03E3E208FD63141801E3EEF2FBDC
:101A9000E36E18FD63141801E3EA5FFC1305000010
:101AA0006FF01FFC130510006FF09FFBE39807FE1B
:101AB0006FF09FF9E3EC65FA6FF05FFEE368DEFB21
:101AC0006FF0DFFDE300C7F4E31C07F693070000A7
:101AD0006FF0DFF5832F050003284500032E8500F6
:101AE00083A205000325C50083A8450083AE8500B9
:101AF00083A6C500130101FFF3272000B78700006C
:101B0000135605019387F7FF9315050113930601FB
:101B100013D706013376F60093D505011355F50169
:101B2000135303013377F70093D6F6016310F602DF
:101B3000B367F801B3E7C701B3E7B700638A070CDF
:101B400073601800130520006F004006631AF70049
:101B5000B3E71201B3E7D701B3E76700E39207FEEB
:101B6000631A060AB367F801B3E7C701B3E7B70022
:101B700093B71700631A070033EF1201336FDF01C9
:101B8000336F6F00630A0F06639C07006394A6001F
:101B90006352C702630E05041305F0FF6F000001D6
:101BA0001305F0FF6384060013850600130101018D
:101BB000678000006356E600E31A05FE6FF0DFFD64
:101BC000E36AB3FC639E6502E3E6CEFD631EDE03BB
:101BD000E3E208FD63141801E3EEF2FBE36E18FD87
:101BE00063141801E3EA5FFC130500006FF01FFCAB
:101BF000130510006FF09FFBE39807FE6FF09FF94D
